:100000000C94780F0C94970F0C94970F0C94970FF7
:100010000C94E9290C94970F0C94970F0C94442B93
:100020000C94970F0C94970F0C94970F0C94970FB8
:100030000C94970F0C94970F0C94970F0C94970FA8
:100040000C94970F0C94970F0C94970F0C94970F98
:100050000C94970F0C94970F0C943A300C94970FC4
:100060000C94970F0C94970F0C94970F0C94970F78
:100070000C94970F0C94970F0C94970F0C944622A6
:100080000C94970F0C94970F0C94970F0C94970F58
:100090000C94970F0C94970F0C94970F0C94970F48
:1000A0000C94970F3D130915D614231507123E150E
:1000B000C714C814F3108011B21EEE14C714C7146D
:1000C000BB1F681309100915D614231507123E1516
:1000D0005B14C814AA138011B21EEE145511C71474
:1000E000BB1F6813C7140915D614231507123E1534
:1000F0002012C814F6118011B21EEE145B11C71441
:10010000BB1F6813C7140915D614231507123E1513
:100110008212C814F9118011B21EEE14B714C7145C
:10012000BB1F681315110915D614231507123E15A8
:10013000C714C814FD118011B21EEE146413C71445
:10014000BB1F681315110915D614231507123E1588
:100150004911C81496138011B21EEE147115C714FC
:10016000BB1F681315110915D614231507123E1568
:100170004F11C814D9138011B21EEE14F510C71414
:10018000BB1F68131511C714C714C7140712C7146F
:100190005615C71406118011B21EC714C714C71410
:1001A000BB1FC714C7140915D614231507123E1513
:1001B000C714C8140C138011B21EEE140713C71411
:1001C000BB1F6813C7140915D614231507123E1553
:1001D000B611C8143E138011B21EEE146111C7147B
:1001E000BB1F6813C7140915D614231507123E1533
:1001F000BE11C81442138011B21EEE14C714C714E6
:10020000BB1F6813C7140915D614231507123E1512
:10021000C311C814A40F8011B21EEE142B14C714FE
:10022000BB1F6813C7140915D614231507123E15F2
:10023000C714C814990F8011B21EEE144613C714C8
:10024000BB1F6813C7140915D614231507123E15D2
:100250008B11C81420148011B21EEE149315C7140C
:10026000BB1F6813C7140915D614231507123E15B2
:100270009711C81466158011B21EEE149C14C71491
:10028000BB1F6813C71488117D1417130712DC11E4
:10029000A211E811EC108011B21EC7147211C7141C
:1002A000BB1FC7149CACCCB6F400C111214191A175
:1002B00031B171F19CACCCB6F4367491A1C111216D
:1002C0004131F17100030205000305010406020437
:1002D000C0C1C2FFC4C5C618808182C38485868719
:1002E0007071728374757677303132733435363786
:1002F00010111213141516170304050A08060BFF34
:100300000209070D010C00FF464B3A3A494A483AA8
:100310003A3A3A3A4C4F3A3A3A3A3A3A3A3A3A3A16
:100320003A3A3A3A3A4D3A3A66304E745A00000038
:1003300000000000000000000000000000000000BD
:1003400000000000000000000001540003FC000257
:10035000A80550000FF0000AA000000550000FF0A3
:10036000000AA00000000000000000000015470087
:100370003FFE002AA0005FFF07A0057807FEF03EC1
:1003800000F03FFFBD2AAA0AF555FFD400502B40CC
:10039000BFC2F007C0BCFF007CABC0A05F80001FE5
:1003A000FFFFFFFFFFFF800FFF000FFF400FFFFF6A
:1003B000FF2FFFFFFFFFFCFFFFFCF00000F000003D
:1003C000F00000FFFFFCFFFFFCFFFFFFFFFFFFFF50
:1003D000003FFF003FFF407FFFFFFF2FFFE0FFFFD9
:1003E000FCFFFFFCC003FCC003FCD007FCFFFFFCCC
:1003F000BFFFE01FFFFFFFFFFFFF8000FF0000FFC8
:100400004000FFF0002FF000FFFFD0FFFFFC000BCB
:10041000FC0003FC0007FC00FFFC00FFE0FFFFFF07
:10042000FFFFFFFF0000FF0000FF40003FFFFF0A4B
:10043000FFFFFFFFFCFFFFFC0003FC0003FC0007C5
:10044000FCFFFFF0FFFE80FFFFFFFFFFFFFF003F0D
:10045000FF003FFF003FFF0000FF0000FFFFFCFF29
:10046000FFFCC003FCC003FCC003FC0003FC000352
:10047000FCFFFFFFFFFFFFFF003FFF003FFF002AE1
:10048000FF0000FF0000FFFFFCFFFFFCC00000C0FA
:1004900000008000000000000000001FFFFFFFFFC1
:1004A000FFFF8000FF0000FF4000FFF0002FF00082
:1004B000FFFFD0FFFFFC000BFC0003FCFF07FCFF6D
:1004C000FFFCFFFFE0FFFFFFFFFFFF00003F00001A
:1004D0003F00003FFFFFFFFFFFFFFFFFFCFFFFFCB0
:1004E000C00000C00000C00000FFFFFCFFFFFCFFD9
:1004F0000000FF0000FF5555FFFFFFFFAAAAFF0005
:1005000000FF00000003FC0003FC5557FCFFFFFC4C
:10051000AAABFC0003FC0003FC000000000000FF8D
:100520000000FF0000FFFFFFFFFFFFFF000000FFD4
:10053000D000FFFC000BFC0007FCFFFFFCFFFFE00E
:10054000000000FFFFFFFFFFFF00003F0001FF0072
:100550001FF8FFFF80FFF800FFFFFCFFFFFCD0004B
:1005600000FD0000BFD0000BFFFC00BFFCFFFFFF41
:10057000FFFFFF000000000000000000000000007E
:100580000000FFFFFCFFFFFC0003FC0003FC000376
:10059000FC0003FC0003FCFFFFFFFFFFFF0AFF500E
:1005A000000FFF05FFA0FFFFFFFFFFFFFFFFFCFFA6
:1005B000FFFC000000000000000000FFFFFCFFFF48
:1005C000FCFFFFFFFFFFFF2BFF50002BFF00002B66
:1005D000FFFFFFFFFFFFFFFFFCFFFFFC00000050DD
:1005E0000000FF5000FFFFFCFFFFFC1FFFFFFFFFAD
:1005F000FFFF8000FF0000FF4000FFFFFF2FFFFF15
:10060000FFFFD0FFFFFC000BFC0003FC0007FCFF1A
:10061000FFFCFFFFE0FFFFFFFFFFFFFF003FFF00CA
:100620003FFF407FFFFFFF2FFFFEFFFFFCFFFFFCB0
:10063000C00000C00000C00000C0000000000017A3
:10064000FFFF7FFFFFFF8000FF0000FF4000BFFFB4
:10065000FF2BFFFFFFFF50FFFFF0000BFC0FF6FC2E
:100660000AFF6CFDBFF4FFDBFCFFFFFFFFFFFFFF96
:10067000003FFF003FFF407FFFFFFF2FFFFEFFFF18
:10068000FCFFFFFCFF0000FFD000EFFD00C2FFFCFD
:10069000002FFC17FFF57FFFFFFF80BFFF003FFF2C
:1006A000403FBFF02F2BF00A003F50403FF4C00BFB
:1006B000FCC003FCD007FCFFFFF8FFFFA0FF000019
:1006C000FF0000FF5555FFFFFFFFAAAAFF0000FF34
:1006D0000000000000000000555554FFFFFCAAAACE
:1006E000A8000000000000FFFFFFFFFFFF00000068
:1006F000000000000000FFFFFFFFFFFFFFFF50FFB3
:10070000FFF4000BFC0003FC0007FCFFFFF8FFFFF9
:10071000A0FFFFFFFFFFFF0000000000000000003F
:10072000FFFFFFFFFFFFFFD000FFFD0000BFD00075
:100730000FFC007FE0FFFE00FFE000FFFFFFFFFF78
:10074000FF000000000000000000FFFFFFFFFFFFB0
:10075000FFFFFCFFFFFC017FA03FF00002BF50FF46
:10076000FFFCFFFFFCFF5000FFFF5000AFFF000049
:100770003F005FFFFFFFA0FFA0000017FC17FFFC7A
:10078000FFE800F00000FFD4002BFFFC002BFCFF73
:10079000FFD0FFFFFD0000BF00000F00007FFFFF44
:1007A000FEFFFFE0000000000000D55554FFFFFCF5
:1007B000EAAAA8000000000000FF0000FF0000FF00
:1007C0000007FF007FFF07FFFFFFFEFFFFE007FFBF
:1007D000FC7FFFFCFFE3FCFE03FCE003FC0003FCEA
:1007E0000003FCFFFFFFFFFFFFFF0000FF0000FF13
:1007F0000000FF0000FF0000FFFFFCFFFFFC000304
:10080000FC0003FC0003FC0003FC0003FC140000DC
:100810003FD4002BFFD4002BFF00002B0000000072
:100820000000000000000000000000D40000FFD421
:10083000002BFFC0002BC0FF0000FF0000FF0000E6
:10084000FF0000FF0000FFFFFFFFFFFF0003FC00B1
:1008500003FC0003FC0003FC0003FCFFFFFCFFFFA4
:10086000FC001F0001FF001FFFFFFFFFFF2FFFFF26
:1008700002FF00002F00000000000000FFFFFCFF4F
:10088000FFFCFFFFFC000000000000000000000073
:100890000000000000000000000000000000000058
:1008A0000003FC0003FC0003FC0003FC0003FC004D
:1008B00003FC0003FC00000000000000000000003A
:1008C0000000000000000000000000000000000028
:1008D0000000000000000000000000000000000018
:1008E0000000000000555555FFFFFFAAAAAA00000E
:1008F00000000000000000000000554154FFC3FC50
:10090000AA82A8000000000000555500FFFF00AAC1
:10091000AA00000000000000FFFF00FFFF00000031
:1009200000000000000000000000000000000000C7
:10093000000000000FF00FFFFF0FFFFF000FF00F90
:10094000FFFF0FFFFF000FF03FC000FFFFC0FFFFE2
:10095000C03FC000FFFFC0FFFFC03FC000005554B4
:1009600007FFFF0FE02FFFFFFFAFEAAF0FF40F020B
:10097000FC0200540040FF40C02FC0FFFFFCEAAF64
:10098000E8F57FC0FFFE0001540003FC0002A8014F
:1009900000017F017FFE3FFE803E8000000140019C
:1009A0007FC07FFE80FE800080000003FC0003FC0F
:1009B0000000000101551F1FFFFF3E03FF3FDFE066
:1009C0000AFA00000003FFFD40EAAFF04002FCF528
:1009D00000FCBFF5F802FFD0FFFAB0000000FFFFF7
:1009E00000FFFF0000000000000000000000000009
:1009F00000000000000000000000000000000000F7
:100A000000000000000000000007FF01FFFF0FFAD8
:100A1000007E0000A80000000000000000FF400071
:100A2000FFFD0002BFC00002F40000A800000000AB
:100A30000000F400003F40000BFD5500BFFF000226
:100A4000AF00000000000000007C0007F055FF80B0
:100A5000FFF800EA0000000000003D0F000BDF007F
:100A600015FF003FFF002AFF0007EF003E0FF07C5C
:100A700000F7E000FF5400FFFC00FFA800FBD000DF
:100A8000F0BC0000000F00000F00155F003FFF00EA
:100A90002AAF00000F00000FF00000F00000F55436
:100AA00000FFFC00FAA800F00000F00000000007C2
:100AB00000000F00000F00005B0007CF01FA0F00DD
:100AC000000B400000C00000C00000940000CF40B8
:100AD00000C2BD0080000000000500000F00000FF4
:100AE00000000F00000F00000F00000F500000F08A
:100AF0000000F00000F00000F00000F00000F00046
:100B00000000000702F50F000BCF0000A700000F48
:100B100000000F00000B400000C17E00CF80006885
:100B20000000C00000C000008000000000000000C5
:100B30000000000100017F017FFE3FFE803E80003B
:100B4000000140017FC07FFE80FE80008000000029
:100B5000000000000017FFFF7FFFFFFF8001FF0084
:100B60001FFF41FFBFFFFF2BFFFFFFFF50FFFFF401
:100B7000FF8BFCF803FC8007FCFFFFF8FFFFA000E1
:100B8000000007FC007FFD55FFFFFFAAAAAA000096
:100B9000000000000003FC0003FC5557FCFFFFFCB5
:100BA000AAABFC0003FC0003FC1FF0007FF000FF79
:100BB0008000FF0001FF401FFFFFFF2FFFF8001F15
:100BC000FC01FFFC1FFBFCFF83FCF803FC8003FC23
:100BD0000003FC1FF000FFF000FF8000FF003FFF5C
:100BE000407FFFFFFF2FFFE0003FD0003FFC000BE6
:100BF000FCC003FCD007FCFFFFFCBFFFE000007F50
:100C00000007FF007FF807FF807FFD55FFFFFFAA69
:100C1000AAAAFF0000FF0000FF0000FF0000FF5530
:100C200054FFFFFCFFAAA8FFFFFDFFFFFFFF00FF2F
:100C3000FF00FFFF00FFFF00FFFF002F003FD0007D
:100C40003FFC000BFC0003FC4007FCFFFFFCFFFF28
:100C5000E01FFFFFFFFFFFFF807FFF00FFFF00FFA0
:100C6000FF00FFAA002FFFFFD0FFFFFC800BFC005E
:100C700003FC4007FCFFFFFCFFFFE0550000FF0006
:100C800000FF0000FF0001FF001FFFFFFFFFFFF854
:100C9000000000000000155554FFFFFCFAAAA880D0
:100CA00000000000001FFFD0FFFFFFFF80BFFF001C
:100CB0003FFF407FFFFFFF2FFFE27FFFD0FFFFFCE2
:100CC000E00BFCC003FCD007FCFFFFFCFFFFE01FB4
:100CD000FFF5FFFFFFFF80BFFF003FFF407FFFFFEB
:100CE000FF2FFFFF003FD0403FFCC00BFCC003FCC8
:100CF000C007FCFFFFFCFFFFE06FFFF9F4550FFC9E
:100D00000A8FFCFFF3FC054FFCAA0FE7FFF6BFFFBD
:100D1000E4C1547CCA80FC3FFCFCC540FCC2A8FC7A
:100D20007FFF6C00000700000F00000F00000B00A9
:100D30000000000000000000400000C01500C7E8EF
:100D4000009E0000000000000000000000000007FE
:100D500000007F0007F8007F8007F8003F80003820
:100D60000000400000F40000BF40000BF40000BF92
:100D700040000BF00000B0000FF0000FF0000FF08B
:100D8000000FF0000FF0000FF0000FF00FF0000F59
:100D9000F0000FF0000FF0000FF0000FF0000FF068
:100DA000003400003F40000BF40000BF40000BF493
:100DB0000000BF00000B0000700007F0007F8007FC
:100DC000F8007F8000F8000080000017FC007FFC26
:100DD00000FF8001FF001FFF41FFBFFFF82BFF80D6
:100DE000000000000000555154FFF3FCAAA2A80027
:100DF00000000000002FFFF902AA8F00000F000082
:100E00000B000000000000000000BFFFE0CAAA00C5
:100E1000C000008000000000000000000000000092
:100E20000000003FC0003FC0003FC0003FD0003F77
:100E3000FF000BFF1FFFD0FFFFFCFF8BFCFF03FC3D
:100E4000FF03F8FFFFFCFFFFFC0FFFFF0FFFFF009A
:100E5000001F00003F00003F00003F00000BFFFFAD
:100E6000FCFFFFFCF80BFCC003FCD007FCFFFFFC01
:100E7000FFFFE000007F0003FF0003FE0003FC0013
:100E800003FD0003FF0000BFFFFFD0FFFFFC000BCE
:100E9000FC0003FC0007FC000FFC000FE000000159
:100EA00000001F00003F00003F00002F0FFFFF0F5A
:100EB000FFFFFFFFD0FFFFFCE00BFCC003FCD007EF
:100EC000FCFFFFFCFFFFFC00007F0003FF0003FEB0
:100ED0000003FC0003FD0003FF0000BFFFFFD0FF85
:100EE000FFFC3FCBFC3FC3FC3FC3FCFFC3FCFFC385
:100EF000FC400000F40000FC0000FC0000FC0000CE
:100F0000FC0000E000000000000000000000000005
:100F10000000000000000000000000400000F4009D
:100F200000FC0000FDFFF4FCAAA0FC0000E00000B3
:100F300000000000000000000000000000000000B1
:100F40000000000000400000F40000FC0000FDFF75
:100F5000FDFCAAA8FC0000E0000000000000150055
:100F600007E800AA000000000000000000000040A8
:100F70000000F40000FC0000FDFFFDFCAAA8FC003E
:100F800000E0000000000000150007E800AA0000D3
:100F9000AF400002BD00000000400001F4000FFC63
:100FA000000FFDFFF7FCAAA0FC0000E0000000001D
:100FB00000C01500C7E8002A0000AF400002BD00D5
:100FC000000000400001F4000FFC000FFDFFF7FCE3
:100FD000AAA7FC000FE0000B000000C01500C7E846
:100FE000002A00006F4000C2BD0080000000001514
:100FF00000003F00000000000500000F000000009E
:101000000000555550FFFEA000BF00555F00FFFFD8
:1010100000001600000000000FF0000FF0000FF0BD
:10102000000FF5000FFF15FFF03FAFF00FF5FC0FBD
:10103000FFA85FF000FFF0000FF0000FF0000FF0CE
:1010400000FD4000FFFD40FC2BFDFC002FFD0002D9
:10105000FFC000FFC0000005FC05FFFCFFA0FCE096
:1010600000FC0001FC000FFC000FFC000000000071
:10107000000000000000070001FE007F800FE0007C
:101080000001FC007FFC1FE0FCFF00FC0BD0FC001B
:10109000BFFC0000FC00000100000F00003F00004A
:1010A0003F00003F00003F00003EF001F0C17FF034
:1010B000DFFA00E00550DFFFF0EA03F0000A00006D
:1010C000000500007F0003FF0003F80003FD00019E
:1010D000FF0003FAFFFF40FFFFF0A00FF0001FE04A
:1010E00057FF50FFFFF0AA03F017FFFF3FEAAAFEE9
:1010F0000054FC00FCFF01FD3FFFFF0BFE8FFFFFD4
:10110000FFABFEAA00FF0000FF0001FF00FFFE0092
:10111000FFF80000000114001FFC007FFC00FCFD34
:10112000403F3FFFFF0ABFFF5FF500FFFFF0800277
:10113000FC0003F8517FE0FFFE00EA8000001FD4AE
:1011400001FFFD07F82F0FF00F0FF00F0FF00A024D
:10115000FC001FFD00FFFFD0F00BF4E003FCC00318
:10116000FC8003FC000FF000001500003F07FFFFAC
:101170003FFFFFFE003FFC002ABF00000003FC0110
:101180005FFCFFFFFCFEA3FC0003FC0003FC00036C
:10119000FC0000FC005FFF0FFEFE3F80FCFE00FC39
:1011A000FD00FC3F4000FC0000FFD400FEFFC0FC3F
:1011B0000BF0FC02FCFC01FC0007E0000014000145
:1011C000F80013F007F3C0FE83F0A002FF00000A4E
:1011D0000155001FFFD07E02FCFC00FCFC07E0FF75
:1011E000FFFCAAAAA800001F0001FE0173F05FE344
:1011F000F0F803F50000BF00000AFFFF40FEAFF467
:10120000FC02FCFC00FCFC01FCFC03F0A80000005C
:1012100000500000F0007CF51FE0FF3E00000000E1
:10122000000000000000FC0000FC5555FCFFFFFC26
:101230000000FC0000FC00000000005F0001FE0157
:10124000F3F05FA3F0F802FF00002B000000FFFDA9
:1012500040AAAFF40002FC0001FC555FF8FFFE80DD
:101260000000000003FF0010AA45F0003F800028A6
:1012700001FF0002AA000000FFFFD0AAABFC0000A3
:10128000FC0005F8FFFFFCAAAAA80000000000006F
:1012900000000005FFFF3FFFFFFE00003C000000D4
:1012A000000000001F00003FFFFFFFFFFFE80000FD
:1012B00000000000000000001FE0003FC0003FD021
:1012C000000FF00003FC0003FC001FF07F8000FF14
:1012D0000000FF00003FC0000FF0000FF0007F8013
:1012E000000000FF07F0FF0F007E0BD3F007F3FDB7
:1012F0000F80FF00002FFFFFFCFFFFFC000000003D
:101300000000000000FFFFFCFFFFFC0017FF01FFD3
:10131000EA0FE8000FC0000FD40002FFD5002BFF3A
:10132000FF50FCAFFDFC000BFC0000000007FC5F61
:10133000FEFCFA80FC400000F40000FC0000FDFF11
:10134000F4FCAAA0FC0000E0000000000000000087
:10135000000000000000000000000000000000008D
:1013600000000003FC0003FC0003FC0003FD00037D
:10137000FF0000BF07FFD03FFFFC3F8BFC3F03FC9B
:101380003F03F8FFFFFCFFFFFC0FFFFF0FFFFF0015
:10139000001F00003F00003F00003F00000BFFFF68
:1013A000FCFFFFFCF80BFCC003FCD007FCFFFFFCBC
:1013B000FFFFE000000700003F00003F00003F008B
:1013C000003F00003F00000BFFFFD0FFFFFCE00BE1
:1013D000FCC003FCC003FCF00FFCF00FE0000001B8
:1013E00000001F00003F00003F00002F0FFFFF0F15
:1013F000FFFFFFFFD0FFFFFCE00BFCC003FCD003AE
:10140000FCFFFFFCFFFFFC00000100001F00003F8D
:1014100000003F00003F00003F00000B555540FF1B
:10142000FFF4EFEFFC0FC3FC4FC3FCFFC3FCFFC393
:10143000FC000003007FFF03FFFF03FE0303FD0327
:1014400003FFC000BFC0FC0000FFFFFCFFFFFCFC6F
:101450000000FC000000000000000000007F00030E
:10146000FF0003FE0003FC0003FD0003FF0000BFBC
:10147000FD03F4FFC3FF2FC0BF0FC03F1FC07FFF9E
:10148000FFFFFFFFF803FFFF03FFFF00000700005F
:101490000F00000F00000F000002FFFFFCFFFFFC29
:1014A000F80000F00000F40000FFFFFCFFFFFC006C
:1014B000000000000000001500FF3F00FF3F00009B
:1014C00000000000000000000000400000FFFFFCE2
:1014D000FFFFFC0000000000000000000000000012
:1014E000000000000000001500FF3F00FF3F000368
:1014F000F40003FF0000BF00003F40007FFFFFFF3C
:10150000FFFFF800FFFF00FFFF00000000000100E8
:10151000003F00003E000000FFFFFCFFFFFC1FF447
:1015200000FEBF40E00BFC0000BC0000000000001B
:10153000000000000000003FFF003FFF000000002F
:101540000000000000000000000000FFFFFCFFFFA3
:10155000FC00000000000000000700003F00003F0A
:1015600000000F00003F00003F00000BFFFFFCFAEF
:10157000AAA8D40000FFC000E80000F55554FFFF02
:10158000FC00003F00003F00001F00003F00003F44
:1015900000003F00000BFFFFFCFFFFFCE00000C06D
:1015A0000000C00000FFFFFCFFFFFC000007000080
:1015B0003F00003F00003F00003F00003F00000BE5
:1015C000FFFFD0FFFFFCE00BFCC003FCD007FCFFDB
:1015D000FFFCFFFFE0003FFF003FFF0007FE000FA2
:1015E000F0000FF4000FFF0002FFFFFFFCFFFFFC05
:1015F00002FD0000FF0001FF00FFFF00FFF80000F8
:10160000007F0007FF000FF8000FF0000BF4003F11
:10161000FF003FFFFFF400FFFF0002FF0000FF009C
:1016200001FE00FFFFFCFFFFFC00003F00003F0049
:10163000000700003F00003F00003F00000BFFFFDD
:10164000FCFFFFFCFE0000E00000D00000FC0000FA
:10165000FC000000001F0000FF0000FE0000FC0076
:1016600000FC0000FF0000BFFD0FD0FFCFFC2FC229
:10167000FC0FC0FC0FD1FC0FFFFC02FFE0000003D9
:1016800001555703FFFF02AAAB0000030000000052
:101690000000FC0000FD5540FFFFF4FEABFCFC0128
:1016A000FC003FFC003FE000003F00003F00000066
:1016B00000000000000000003F00003FFFFFD0FFDF
:1016C000FFFC000BFC0003FC0007FCFFFFFCFFFF1E
:1016D000E000003F00003F000000000000000000AC
:1016E00000003F00003FFFD000FFFD0002FFD000E0
:1016F0003FFC01FFE0FFFE00FFE00000003F0000B4
:101700002A00000000000000000000001500003F5B
:10171000FFFFD0AAAFFC0007FC03FFF0000BFC5555
:101720005FFCFFFFE000003F00002B000000000016
:101730000000000000001700003F4001FCF41FE81B
:10174000BFFE000FF0007FFD00F82FD48002FC00E8
:10175000003F00003F0000000000000000150000F6
:101760003F00003FFD03F4FFC3FC2FC0BC1FC03C83
:10177000FF807CFFFFFCFFFFF800003F00003F0000
:10178000003F00003F00003F00003F00003FC0015D
:10179000FCC01FFCC1FFFCDFFFFCFFE3FCFE03FC01
:1017A000E003FC00000000000301400F7FFFFFFE8C
:1017B000AAA8F00000A00000000000C00000F00196
:1017C00040FFFFFD2AAABF00000F00000A00000032
:1017D000000000555555FFFFFFAAAAAA000000000F
:1017E0000000000000000000555554FFFFFCAAAAAD
:1017F000A8000000000000000000F00000FC000055
:10180000FFFFFD2BEAAF0000030000020000000014
:10181000000F00001F1FFFFFFAABE8E00000800090
:1018200000FD4000FFFD40FC2BFDFC002FFD0002F1
:10183000FFC000FFC0000005FC05FFFCFFA0FCE0AE
:1018400000FC0001FC000FFC000FFC1FFFFFFFFF6E
:10185000FFFF800FFF000FFF400FFFFFFF2FFFFF75
:10186000FFFFD0FFFFFCC00BFCC003FCC007FCFF68
:10187000FFFCFFFFE03000003000003000002000DF
:1018800000300418355D80300C902000083BAEBC61
:10189000359D9C318C9C2AAAA83BAEBC359D9C31C1
:1018A0008C9C2AAAA8300018355580300090200062
:1018B00008300418355D8030009020000830001892
:1018C0003555803000002000000057C007FFC402DB
:1018D000FFC000028000FFC005FFD402FFE0002E21
:1018E000000001F41557F82D1000028000300000B0
:1018F00030000030000020000007FFF40B503C05D2
:101900007FF40A00283FFFFC000F00157D402AAA43
:10191000800007FC00783C07897C280028003C00F8
:10192000557D55AABEAA003C00000000555555AA99
:10193000BEAA003C003FFFFC30000C30000C300021
:101940000C3FFFFC31554C32AA8C30000C3FFFFCA1
:1019500031554C32AA8C33FFCC30000C30000C30A7
:10196000000C35555C31554C32AA8C30000C355585
:101970005C31554C32AA8C33FFCC35555C2AFFA81C
:10198000000000000000000000000000555400AA04
:10199000BC00003C00003C00557C00AAA8000000F0
:1019A00000003C00003D55002AAA00000000000095
:1019B000001555003EAA003C00003C00003C000021
:1019C0003C00003C00003C00557C00AABC00003CF0
:1019D0000001414403C7E007E3C0228280003C00CD
:1019E000003D55003EAA003C00003C00557D55AA34
:1019F000AAAA000000000000000000000000000093
:101A0000000000003FFF3C0000000000003FC0005D
:101A10000000001540002A800017D7D42BEBE83FC8
:101A2000FFFC02828007F4D01F7DF40F3DF0020A14
:101A3000803C0078001E8007A0142800281F47F46F
:101A40003C343C2F8AF80002080000001440002AB1
:101A5000000000000007FFD03E00BC20000800008E
:101A60000034001C2F55F802AA80000000024C60D0
:101A7000017F50006E40020820003C0003FFC000C0
:101A80003C000000000000000003D800000000003F
:101A900000003C00003C00003C000028000000006A
:101AA0000000F0000000000000000078001E800729
:101AB000A0002800001FFFF43C1E3C3DF57C0AAA54
:101AC000A005003C3FFFFC00003C0000001F01FCA3
:101AD0003C1FBC3DF83C0A80281F00F43C143C3DF0
:101AE0007D7C0A82A0007F00078F003FFFFC000A78
:101AF000003FF0F43CF03C3CF57C282AA01FFFF4AA
:101B00003C3C3C3C3D7C280AA03C00003C1FFC3D8A
:101B1000F8002A80001FD7F43C3C3C3D7D7C0A82C3
:101B2000A01FF4F43C3C3C3D7D7C0AAAA0000000D0
:101B30000141400282800000000000000141440297
:101B400082A0000000001D0001E2D00E002C000069
:101B50000001414003C3C003C3C0000000040004EF
:101B60000B407800B7800008001F00003C1F3C3D80
:101B700078000A800006AAA431AA4C24AA4C02AA22
:101B80000007FFFC3E0F002F5F5402AAA83FFFFC96
:101B90003C3C3C3D7D7C0A82A01FFFF43E00BC3DE6
:101BA000007C0A00A03FFFFC3C003C2F55F802AA35
:101BB000803FFFFC3C3C3C3C283C2800283FFFFC8D
:101BC0003C3C003C28002800001FFFF43C003C3C4B
:101BD0000F7C080AA03FFFFC003C00157D542AAA98
:101BE000A83C003C3FFFFC3C003C0000001400F41B
:101BF0003C003C3FFFF82800003FFFFC003C001782
:101C0000C3D42800283FFFFC00003C00003C00003B
:101C1000283FFFFC0B40001F55542AAAA82FFFFCA9
:101C200002D000157D542AAAA81FFFF43C003C3DB9
:101C3000557C0AAAA03FFFFC3C3C003D7C000AA06A
:101C4000001FFFF43C053C3D57FC0AAAA03FFFFCE7
:101C50003C3D003D7EF40AA0281FF4343C3C3C3C53
:101C60003D7C080AA03C00003FFFFC3C0000000057
:101C7000003FFFF400003C15557C2AAAA03FFF401E
:101C80000000B41555E02AAA003FFFF800078015B0
:101C900057D02AAAA83D417C02BE8017EBD4280069
:101CA000283FD400003FFC3FE8000000003C01FC5E
:101CB0003C1E3C3DE03C2A00281555543EAABC3C45
:101CC000003C0000002D000002B400000AD000001B
:101CD000281400143C003C3FFFFC00000001E00021
:101CE0001E00000B400000A00000003C00003C0073
:101CF000003C0000282D000002D000000000000081
:101D0000000051F400F33C00F774002AA83FFFFCE8
:101D100000F03C00F57C002AA0007FF400F03C00BD
:101D2000F03C002020007FF400FC3C157D7C2AAABA
:101D3000A8007FF400F33C00F73C002A20057D5406
:101D40003EBEA83D28000A0000007D1400F33C00C0
:101D5000F77C002AA03FFFFC00780000F554002A21
:101D6000A80050003CFFFC0000000000000000F450
:101D700000503C3CFFF80000000FFFFC0007D000C3
:101D8000382C0000081400003FFFFC000000000099
:101D90000000FFFC002D00007D5400AAA800BFFC3D
:101DA00000F80000BD54002AA8007FF400F03C00B9
:101DB000F57C002AA000FFFC007AD000F5F0002A94
:101DC00080007FD000F0F0007FD400AAA800FFFCC4
:101DD00000780000F400002800007D3C00F33C0087
:101DE000F37C00A0A015F5502AFABC00007C00008E
:101DF000A000FFF400003C00557C00AAA000FF40BA
:101E00000000B40055E000AA0000FFFC0001E00063
:101E100055F400AAA800F47C002BA0007EF400A0DA
:101E20002800FD14000F3C005F7C00AAA000F07C9D
:101E300000F3BC00FE3C00A028000000057D503AE5
:101E400082AC000000000000555555AAAAAA000067
:101E50000000000035415C0ABEA00000003F41FCCC
:101E60003CBE3C3D007C2A00A83FFFFC003C00003B
:101E70003C00002800010101FF02EB0202D76802CA
:101E8000D10102C08007C128282828140005C200FB
:101E900000000002CB170BB4E577F1FFFF4FF1FF15
:101EA000FF4F02B064011101FF03C7A6E90236200B
:101EB000023A1102B80902D01F0120012902B9E338
:101EC00001FF02B923027200013900000000000185
:101ED0000101020203030405060708090A0B0C0EA0
:101EE0000F1012141517191B1D1F212325272A0057
:101EF00011241FBECFEFCDBFDFE7DEBF10E4A0E0AF
:101F0000B0E4E0EDFEE700E00BBF02C007900D92E9
:101F1000AE30B107D9F72DE7AEE0B0E401C01D92B5
:101F2000A63EB207E1F70E943D3C0C94663F0C943C
:101F300000009091317D81E098279093317D8093CE
:101F400007408093064008951092317D81E0809390
:101F500007408093054080930640089581E0809378
:101F6000E57D10927A4210927B428093CF69E1E343
:101F7000F2E411921586138E11A617AA82E4EF33AC
:101F8000F807B9F710928642109287421092884261
:101F900010928A4210928B421092C9691092CA69BB
:101FA00010927742109278421092794280E18093A9
:101FB00089421092F5691092CD6908958091794215
:101FC000813019F087E792E4089588E792E4089554
:101FD0008031910508F0C097E1E3F2E427E0289F03
:101FE000B001299F700D112490E080E0DC01A60F64
:101FF000B71FA457BD4B258D30E1239FA0011124AD
:10200000248D242B2C93019632968730910571F7FD
:1020100008950895CF93DF93DC01EB013EE04991F1
:102020004D933A95E1F7DF91CF910895CF93DF93E8
:10203000342FDC01EB01231BA30FB11DC30FD11DF6
:1020400049914D932A95E2F7DF91CF910895242F7E
:10205000DC01261BA60FB11D1D922A95EAF70895F3
:10206000CF93DF93342FDC01EB01231BA30FB11DB2
:10207000C30FD11D4C9158815D9349932A95D2F796
:10208000DF91CF910895CF93DF93DC01022E000CF6
:10209000330B51E0E42FF0E02E173F071CF4DF91E3
:1020A000CF91089580E06115710521F0EB01CE0F0D
:1020B000DF1F8881EA0FFB1F9081C091CF699C0FC1
:1020C000980F908380918942981730F0981B9083E5
:1020D0005093CF694F5FDECF1092CF69FBCF0F9344
:1020E000FC0131E0021714F40F91089590E061159E
:1020F000710531F0DB01A20FB11D27FDBA959C914E
:1021000080E04115510531F0DA01A20FB11D27FD24
:10211000BA958C91981B8091CF69981B97FF0FC03F
:1021200080918942980F3093CF69309731F0DF0169
:10213000A20FB11D27FDBA959C932F5FD3CF1092AC
:10214000CF69F3CFCF93DF93242FEC01C60FD11DBE
:10215000261B498149932A95E2F71A92DF91CF9184
:102160000895CF93DF93DC011092CF692417A4F078
:10217000E42F042E000CFF0B90E06115710521F097
:10218000EB01CE0FDF1F9881EA0FFB1F80818917BB
:1021900031F081E08093CF69DF91CF9108954F5F57
:1021A000E5CFAEE7B2E48D919C911197E0E8F2E4BF
:1021B000208131812D933C93A2E8B2E42D913C9192
:1021C000119720833183E4E8F2E4208131812D935B
:1021D0003C931082118208950E94D11080937A421C
:1021E00090937B4208950C94D1100E94D110E1E3AA
:1021F000F2E4292F22952F7022A39F7091A3982F8C
:1022000092959F7090A38F70878F0895E1E3F2E419
:1022100082A1829591A1892B90A19295278D922BD5
:10222000EAE7F2E49083818308958295837090E0D9
:102230009C01220F331F227095958795822B9091D8
:102240007D42292F22952F7030E096E1929FF00178
:10225000939FF00D1124E65DFF4B9589EAE2F0E4CF
:1022600044E0840290011124458949130CC0DF0128
:10227000A20FB31F4D915D916D917C91452B462B23
:10228000472B09F0848B769641E4EA38F40761F72E
:1022900008956DE472E48BE592E40C940A106BE50A
:1022A00072E48DE492E40C940A106DE472E489E621
:1022B00092E40C940A1069E672E48DE492E40C94C2
:1022C0000A10E1E3F2E4968D858D8295807F248D5E
:1022D000822B8093F3699093F4691092A34110923A
:1022E000A4410895E1E3F2E4858D20E1829FC001DD
:1022F0001124248D822B8093A3419093A4410895AF
:1023000082958F708093CB6985E08093F5690895FD
:1023100010928A420895E1E3F2E4858D90E1899F6D
:1023200090011124848D822B80938A420895E1E3E9
:10233000F2E480918A42982F9F70948F82958F70DB
:10234000858F0895E1E3F2E4AAE8B2E48C91958DDB
:1023500040E1949F90011124948D922B9C93982F8F
:102360009F70948F82958F70858F089580918A4297
:102370008093884280EA8093070408958091884280
:1023800080938A42089580918A42909188429093E6
:102390008A428093884280EA8093070480910240B9
:1023A000811109C088ED9DE1809303409093044022
:1023B00081E08093024008950E94DE0FFC0190812D
:1023C000911103C08DE0808308959150908308950A
:1023D0000E94DE0FFC0190819F5F90830E94DE0FC0
:1023E000FC0120812E3008F010820895109279426D
:1023F000089581E080937942089590917742809189
:102400007842981303C081E08093CF690895CF93F9
:10241000C82F0E94DE0FDC01EC91F0E0EF5CFD4B79
:10242000C295CF70C48F0E94DE0FFC019081911184
:1024300004C08DE08083CF91089591509083FBCFAD
:10244000CF93DF930E94DE0FDC01EC91D0918742A5
:10245000C0918642ED30B1F480911040982F9F7B5F
:10246000953B11F0873F49F4C0935A42D09386427E
:10247000C0938742DF91CF910895D0935A42C09381
:102480004D42F8CF80910F408D3079F5809110400A
:10249000853F61F0982F9F70973039F582958F7046
:1024A000982F977F973009F18B30F9F0D0938642BF
:1024B000C09387420E94DE0FDC01EC91F0E0EF5CFC
:1024C000FD4BC58F0E94DE0FDC01EC91F0E0EF5C6C
:1024D000FD4BD48F0E94DE0FDC01EC91F0E0EF5C4D
:1024E000FD4B858D80934D42C5CFF0E0EF5CFD4BF9
:1024F000D58F0E94DE0FDC01EC91F0E0EF5CFD4B2C
:10250000C48FB8CFCF93DF930E94DE0FDC018C9194
:10251000C09186428D3001F59091104080915A42D1
:10252000292F2F7B253B11F0973F49F48093874259
:1025300080938642C0935A42DF91CF910895909143
:10254000874220914D422093864280938742909308
:102550005A42C0934D42F0CF20910F40D091874214
:1025600090E02D3099F520911040253F61F0322FF9
:102570003F70373059F522952F70322F377F373023
:1025800029F12B3019F18F5C9D4BFC01858D8093D7
:1025900087420E94DE0FDC01EC91F0E0EF5CFD4B26
:1025A000848D809386420E94DE0FFC0190914D4203
:1025B000E081F0E0EF5CFD4B958F0E94DE0FDC01C7
:1025C000EC91F0E0EF5CFD4BD48FC3CF8F5C9D4B63
:1025D000FC01858D809387420E94DE0FDC01EC9127
:1025E000F0E0EF5CFD4B848D809386420E94DE0F0D
:1025F000DC01EC91F0E0EF5CFD4BD58F0E94DE0F2B
:10260000DC01EC91F0E0EF5CFD4BC48F95CF809145
:10261000304280937A42089580913042E1E3F2E4BF
:10262000982F92959F7090A38F70878F08958091B7
:10263000327D9091337D892B91F08091327D909104
:10264000337D01978093327D9093337D81E090912B
:10265000A241911101C080E08093CF6908958091DB
:10266000CD69823099F71092CD691092A2411092F3
:1026700030428091254290E0E5CF089580E180933B
:10268000894208958AE0809389420895E1E3F2E463
:1026900082A1829591A1892B90A19295278D922B51
:1026A000909328408093294082E08093F5690895B3
:1026B000E1E3F2E4968F982F92959F70958F8F703B
:1026C000848F1092F569089583E08093F5690895E9
:1026D000CF93DF93CDB7DEB72E97CDBFDEBF829508
:1026E0008F70E82FF0E0E850FD4FE491DE01119685
:1026F0009E01215F3F4FBD0181E08E0F0E2E000C29
:10270000FF0BEF5CFD4B948D9D93E0E08E300CF45D
:10271000E82FA217B30781F78DE492E40E940A1014
:102720002E96CDBFDEBFDF91CF91089580912742D5
:102730002AE0829FC00111242091417D3091427D89
:102740008217930720F081E08093CF69089510925B
:10275000CF69089584E08093F5690895F894809195
:10276000086A8823B9F0E091066AF0E0EA50F64979
:1027700080819091066A9F5F9093066A9091066AA5
:102780009F709093066A9091086A91509093086A9E
:102790007894089580E0FCCF9091240895FFFCCFB9
:1027A0008093220808952EE0FC0111922A95E9F702
:1027B000089581E392E40E94D3138FE392E40E9490
:1027C000D3138DE492E40C94D313ECE8F2E48DE39C
:1027D00097E2DF019C011D9221503040E1F70895FE
:1027E000CF93DF93DC01FC013B966B3061F41B96C9
:1027F0008C911B9792919183EA17FB07D9F78083FD
:10280000DF91CF9108958C91ED0199819993CE1725
:10281000DF07D9F71B968C93F3CF9C014097C097A5
:1028200068F0211582E0380749F0C901805F9240C5
:10283000419720F081E0203F334008F080E0089588
:1028400080912F42882331F00E94D11080937A42E8
:1028500090937B420895CF93DF938091A341909111
:10286000A441009731F08D3F910589F0DF91CF9120
:102870000895C091F369D091F469CE010E940D14BE
:102880008823A1F3CE01DF91CF910C94E80F209122
:102890004F4280914E4230E1839FC0011124922B20
:1028A00020914D42822B80932C7D90932D7D81E051
:1028B00080930640DBCF0E94DE0FDC01EC91ED300F
:1028C000A1F49091104080915A42292F2F7B253BF3
:1028D00011F0973F39F4909187429093864280930C
:1028E0008742089590914D42F8CFF0E0EF5CFD4BA8
:1028F000848D80938642858DF2CF8091327D909138
:10290000337D892B51F08091327D9091337D0197F9
:102910008093327D9093337D08958091CD6981308D
:10292000D9F78091B2418111F7CF82E08093CD69D0
:102930008091254290E0ECCF8EE0815078F4809138
:102940002F42882351F08091CC698D3031F48091F1
:102950004D4280935A4280933E420895E82FF0E022
:10296000EF5CFD4B948D20819223948FE6CFCF9323
:10297000DF93ADE4B2E4C9E6D2E43EE04C91588185
:102980005D9349933A95D1F7DF91CF9108950895DA
:10299000CF9382958F70E82FF0E0E850FD4FC491FF
:1029A0000E94DE0FFC01C083CF91089582958F7045
:1029B000E82FF0E0E850FD4FE491AAE8B2E421E00E
:1029C00030E002C0220F331FEA95E2F78D919C910F
:1029D0001197822B932B8D939C9308952091C96915
:1029E0003091CA6982958F70E82FF0E0E850FD4F72
:1029F000E49181E090E002C0880F991FEA95E2F728
:102A00008223932321E0892B09F420E02093CF69CE
:102A1000089582958F70E82FF0E0E850FD4FE49123
:102A2000AAE8B2E481E090E002C0880F991FEA951D
:102A3000E2F7809590952D913C91119782239323F5
:102A40008D939C93089582958F70E82FF0E0E85065
:102A5000FD4FE49181E090E002C0880F991FEA9554
:102A6000E2F720918A4230918B428223932321E026
:102A7000892B09F420E02093CF690895CF93C82FC4
:102A80000E94DE0FC295CF70EC2FF0E0E850FD4FB2
:102A9000E491DC018C910E2E000CFF0B8E171F06AB
:102AA00019F481E08093CF69CF910895CF93DF939C
:102AB000ADE4B2E4CBE5D2E43EE04C9158815D93C5
:102AC00049933A95D1F7DF91CF91089580912F42A4
:102AD000811106C00E94D11080937A4290937B426C
:102AE0000895E1E3F2E482A1829591A1892B90A15E
:102AF0009295278D922BE2E8F2E420813181209398
:102B0000844230938542A0E8B2E42D913C91119724
:102B100020833183EEE7F2E4208131812D933C93D1
:102B20009083818308958EE0815078F480912F42C4
:102B3000882351F08091CC698D3031F480914D42E1
:102B400080935A4280933E420895E82FF0E0EF5C74
:102B5000FD4B948D2081922B948FE6CFE0E4F4E03E
:102B600081818D608183E0E0F4E0818180648183F4
:102B7000E0E6F9E084E0818381E380830895809337
:102B800064098091630987FFFCCF08951F93CF9359
:102B9000DF93C0E0D4E010E41E830E94BF151D83C4
:102BA000DF91CF911F91089527E731E0829FF001D7
:102BB000839FF00D1124E75FF54920E08181928128
:102BC0009695969530E4839FA0011124942B9283CF
:102BD00090818695869530E4939FA0011124842BE3
:102BE00081839695969590832F5F33962D3731F795
:102BF000089527E731E0829FF001839FF00D1124B3
:102C0000E75FF5492DE781819081990F990F382F62
:102C10003295369536953370932B90839281880F39
:102C2000880F392F3295369536953370832B8183F3
:102C3000990F990F9283215033962111E4CF089573
:102C4000E9E0FAE68DE190E1DF019C011D9221505F
:102C50003040E1F70895E9E0FAE69191DF0111973C
:102C600098279C939AE7E632F907B9F7089527E782
:102C700031E0829FF001839FF00D1124E75FF54959
:102C80009F0122513D4F8191DF01119786768C93F0
:102C9000E217F307C1F7089527E731E0829FF001BB
:102CA000839FF00D1124E75FF549629FD001639F78
:102CB000B00D1124A75FB549CF0189589E4F2191CE
:102CC0002D93E817F907D9F7089570E027E731E069
:102CD000482F429FC001439F900D112447E751E0C8
:102CE000875F95490C945F3FFF920F931F93CF939B
:102CF000DF93182FF62E8AE20E94C61589E1810F14
:102D00000E94BF1589E18F0D810F0E94BF158BE2D4
:102D10000E94C61580E00E94BF158CE70E94BF1577
:102D20008CE20E94C61587E791E0189FE001199F89
:102D3000D00D1124C75FD549F89E8001F99E100D72
:102D400011240C0F1D1FC017D10731F4DF91CF9153
:102D50001F910F91FF90089589910E94BF15F3CFA5
:102D6000CF93DF938F773CE0839FC00111248B5872
:102D7000974EC62FC695E7E7F1E04E9FD0014F9FD3
:102D8000B00D1124A75FB54933E0C39FE0011124C2
:102D90008A1B9B0B60FF30C0AE014D5F5F4FCA0FB7
:102DA000DB1FA40FB51F3CE0841B950BFC01EA0F51
:102DB000FB1F2636F1F0E491E22748814A7A4883E6
:102DC0004C9145754C93F0E0AF0155954795542FC4
:102DD00055754881452B4993EE0FFF1FEA7A4C91B8
:102DE000E42BED93315011F788E0860FDF91CF91FE
:102DF0000895E491E676E1CFAC0FBD1F3CE08C1B5B
:102E00009D0BFC01EA0FFB1F263641F0E491E227FF
:102E1000EC93315011963111F4CFE6CFE491E67680
:102E2000F7CFFF920F931F93CF93DF938C01D42F93
:102E3000F22EC0E0F801EC0FF11D8081811107C076
:102E4000862FDF91CF911F910F91FF9008952F2D25
:102E50004D2F0E94B016682FCF5FECCFFF920F93DB
:102E60001F93CF93DF938C01D42FF22EC0E0F80193
:102E7000EC0FF11D8491811107C0862FDF91CF9156
:102E80001F910F91FF9008952F2D4D2F0E94B01686
:102E9000682FCF5FECCF9C0180E0F901E80FF11DB6
:102EA0009081992311F08F3F09F408958F5FF5CF3A
:102EB000EF92FF920F931F93CF93DF93CDB7DEB7BF
:102EC0006097CDBFDEBF89839A836B837C834D83FC
:102ED0005E832F83388709871A87E8E3F7E7A0E83E
:102EE000B7E78FEA98E71082118212821C9211963E
:102EF0001C92119712961C921297E55BFF4FA55BEF
:102F0000BF4F8E179F0779F76AE089E00E944C1641
:102F1000CE0101967C0110E000E0F7014191519152
:102F20007F012FEF2F5F822F022E000C990BFC01E7
:102F3000E40FF51FE491ABE0B0E0AC0FBD1FA80FAC
:102F4000B91FEC93E111EECFB801675E7F4F880F98
:102F5000991F880F991F681B790B2FEF49E0CE014D
:102F60000B960E9411170E5C1F4F0A3F1105A9F620
:102F700089E00E94D4156096CDBFDEBFDF91CF916E
:102F80001F910F91FF90EF90089599E1899F802DF7
:102F9000112461E0282F260F30E0A901440F551FAE
:102FA000240F351F275F3549F901E15DF24F90810C
:102FB000492F440F440FD901A05DB24F9C919295C7
:102FC000969596959370942B90839C91492F440FDE
:102FD000440F329690819295969596959370942B86
:102FE0009C93408194E0499FA00111244360408359
:102FF0002A55314FF90110826F5F683159F60895F3
:10300000CF93DF930E94201680E090E8A1E0BB27D9
:103010009858AF4FBF4FC9E0DAE6ABBFFC0127912C
:1030200029930196A11DB11D22E7C730D207A9F748
:1030300080E090E0A1E0BB27AC01BD0158586F4F84
:103040007F4FC7E0D2E76BBFFA01279129934F5F0B
:103050005F4F6F4F7F4F28E7CF3AD207A1F78855D0
:103060009148AF4FBF4FCFEAD8E7ABBFFC012791E4
:1030700028830196A11DB11D23962AE7C632D207E7
:10308000A1F7DF91CF910895BF92CF92DF92EF9297
:10309000FF920F931F93CF93DF93362F9AE2899F6E
:1030A000800111240B581C4F83E0689F700111248C
:1030B000B0E0A0E085E1B82E50E097E7C92EDD240E
:1030C000D3948A2FAA32B10561F487E0830FDF9190
:1030D000CF911F910F91FF90EF90DF90CF90BF9015
:1030E0000895FD01E00FF11FE4916B2D0E94113E48
:1030F000BA01680F711D6C9DE0016D9DD00D7C9D26
:10310000D00D1124CE0DDF1DC90FD11DC75FD549CC
:10311000E227E8831196D5CFCF92DF92EF92FF920C
:103120000F931F93CF93DF93D62E92E1899FE001F7
:103130001124C35DDC4F83E0689F8001112430E0DF
:1031400020E089E0C82E50E097E7E92EFF24F394B1
:10315000822F2231310559F483E08D0DDF91CF911B
:103160001F910F91FF90EF90DF90CF900895F9019C
:10317000EC0FFD1FE4916C2D0E941D3EBA01680FFB
:10318000711D6E9DD0016F9DB00D7E9DB00D1124FF
:10319000A00FB11FA90FB11DA75FB549EC932F5F19
:1031A0003F4FD6CF1F93CF93DF93EC01142FFE0137
:1031B0008491811105C0862FDF91CF911F910895D1
:1031C00020E0412F0E94441863E0680F2196EFCF62
:1031D00080E10C94C61581E10C94C615382F262F7A
:1031E000562F5695569543E0852F642F0E941D3E1D
:1031F000982F990F990FE82FE91BE50FA7E7B1E08A
:103200008A9FB0018B9F700D1124E60FF72FF11DDF
:10321000832F8695849FE00DF11D1124E75FF5490A
:10322000317087E0831B220F2670821B21E030E083
:1032300001C0220F8A95EAF78081822B808308954E
:10324000CF92DF92EF92FF92CF93DF93EC01862F24
:103250008150990BFC01EC53FD4FE491633008F46D
:1032600021979E01ABE7B4E10E947E3E6B017C0199
:10327000AFE1B5E00E947E3EAE2FA40FBB27BB1F7F
:103280009D012C0F3D1FD695C795D695C7952C0F40
:103290003D1FDC01CB0153E1B695A7959795879526
:1032A0005A95D1F7820F931F63E1F694E794D79470
:1032B000C7946A95D1F78C1991098730910540F42C
:1032C0008F5FDF91CF91FF90EF90DF90CF900895C7
:1032D0000797F3CF823021F4637081F48DE1089574
:1032E0008150990B67E070E00E943F3E62E070E021
:1032F0000E943F3E9FE1981B892F08958CE108951D
:103300008D3010F08C500895811101C08CE008952B
:10331000CF93DF931092317D85E080931842ECE1EA
:10332000F0E4C5E3DDE7A5EEB9E6119219921D922E
:1033300080E4E832F807C9F710922C7D10922D7DB9
:10334000DF91CF91089560E089E00E946516809139
:103350002C7D80FF07C020E049E060ED86EC98EF0F
:103360000E942E1780912C7D81FF07C020E049E04C
:103370006AEA8CEC98EF0E942E1780912C7D82FFD8
:1033800006C020E049E06CE984E30E94B016809119
:103390002C7D83FF06C020E049E064E983E30E94BE
:1033A000B01680912C7D84FF06C020E049E06CE8D7
:1033B00082E30E94B01680912C7D85FF06C020E03C
:1033C00049E064E881E30E94B01680912C7D86FF7D
:1033D00006C020E049E06CE780E30E94B0168091CF
:1033E0002C7D87FF07C020E049E06EE481ED98EF77
:1033F0000E942E1780912C7D90912D7D90FF07C00B
:1034000020E049E060E387ED98EF0E942E1780915D
:103410002C7D90912D7D91FF06C020E049E068E26F
:1034200087E40E94B01680912C7D90912D7D92FFB3
:1034300007C020E049E062E08BED98EF0E942E1774
:1034400080912C7D90912D7D88279370892B39F464
:1034500020E049E060E380EE98EF0E942E1789E0BB
:103460000E94D41561E089E00C9474160F931F93A9
:10347000CF93DF938091317D882331F101EF19E6FD
:1034800025E33DE7CCE1D0E4EAE8F1E465EE79E656
:10349000D9011B969C91D8018E918D01B4E08B9F30
:1034A000A0011124892F8370842B8295807F4B8506
:1034B000840F868B96959695978B2150310921978D
:1034C00032976017710721F7DF91CF911F910F910C
:1034D00008951F93CF93DF93182F88E1EAE8F1E472
:1034E000A4E1BDE701900D928A95E1F760E0812F9C
:1034F0000E94651660E081E0810F0E946516CAE8AF
:10350000D1E485E020E0412F682F8E890E94441885
:10351000412F682F8F890E948C18229791E4C2371F
:10352000D90781F780912C7D90912D7D837099270B
:10353000892B49F420E048E061E088E5DF91CF91F4
:103540001F910C94B016DF91CF911F910895EAE876
:10355000F1E4A4E1BDE791918D91981306C081E457
:10356000E13AF807C1F781E0089580E00895DC01B1
:103570001E96FB013E963E912291321305C0A8177C
:10358000B907C9F781E0089580E00895FC01108231
:1035900011821282138214820895DC011596FB01B8
:1035A00035963E912291231728F0321728F0A8175C
:1035B000B907B9F781E0089580E008956F927F928E
:1035C0008F929F92AF92BF92CF92DF92EF92FF9233
:1035D0000F931F93CF93DF938B01DB011D921D92FD
:1035E0001D921C921397EC0122963C01BEE06B0EDB
:1035F000711CC12CD12C7601C394A991B0E0A70114
:1036000096010E94943EF80180809180A280B38050
:10361000DC01CB01880D991DAA1DBB1D8083918300
:10362000A283B383AAE0B0E00E94943E6B017C01C8
:103630006C167D0611F7DF91CF911F910F91FF90CE
:10364000EF90DF90CF90BF90AF909F908F907F9042
:103650006F900895AC0190E070E0292F092E000CC6
:10366000330B261737070CF00895240F351FF90187
:1036700010829F5FF2CF4F925F926F927F928F92F4
:103680009F92AF92BF92CF92DF92EF92FF92CF9331
:10369000DF9300D000D0CDB7DEB7F894BE016F5FE6
:1036A0007F4F84EC91E40E94DE1A7894C980DA801E
:1036B000EB80FC808CE3882E912CA12CB12CC701CF
:1036C000B601A50194010E94533E60931E42CA01B7
:1036D000B901A50194010E94533E60931D42C701A8
:1036E000B60120E13EE040E050E00E94533ECA01B6
:1036F000B90128E130E040E050E00E94533E609381
:103700001C4280911C420E94801980932A42C7016A
:10371000B60120E831E541E050E00E94533E6901E6
:103720007A01C982DA82EB82FC82CA01B9016C5546
:103730007C498F4F9F4F22E0660F771F881F991F8C
:103740002A95D1F721EB3AE342E050E00E94533E44
:10375000215F3F4F4F4F5F4F82EAC80E8FEDD81E5B
:1037600084E2E81EF11CC20ED31EE41EF51E62E0C8
:1037700056954795379527956A95D1F7C21AD30A7A
:10378000E40AF50AA4E1B0E0A70196010E94943E84
:103790002B013C012AE8421A29E0520A610871080B
:1037A000C301B20129E83CE140E050E00E94533EF1
:1037B00049015A01ADE6B1E00E94943EC61AD70A0B
:1037C000E80AF90AC301B20124E232E740E050E01E
:1037D0000E94533EC21AD30AE40AF50AA8EEB3E0E7
:1037E000A70196010E94943E29E837E740E050E0A7
:1037F0000E94533E29013A018EE1289FC0181124EE
:10380000A9E5B2E00E94943E28EE33E040E050E0AB
:103810000E94533EC21AC09222422EE04216510428
:103820006104710490F58CE6881A82E1980AA10877
:10383000B10821E0421A51086108710880921F42C4
:103840009092204240922142409122426091214236
:1038500080911F42909120420E94201980932B4218
:1038600081E0809313402496CDBFDEBFDF91CF91DE
:10387000FF90EF90DF90CF90BF90AF909F908F9090
:103880007F906F905F904F9008958BE6881A82E149
:10389000980AA108B1082DE0421A51086108710880
:1038A000CDCF2F923F924F925F926F927F928F92E5
:1038B0009F92AF92BF92CF92DF92EF92FF920F93BF
:1038C0001F93CF93DF93CDB7DEB72997CDBFDEBF70
:1038D000C0901F42D090204220E3C21A28EFD20AA3
:1038E0000D2C000CEE08FF0830912142232E022CF3
:1038F000000C330829823A8291012330310548F4C3
:10390000245F3F4F29833A8331E0C31AD108E1088D
:10391000F10810912242ADE6B1E0A70196010E94A4
:10392000943E4601570122E0B694A7949794879459
:103930002A95D1F7860E971EA81EB91EC701B6019B
:1039400020E931E040E050E00E94533E820E931E99
:10395000A41EB51EC701B60124E630E040E050E0E9
:103960000E94533E821A930AA40AB50A29813A8119
:103970002F5F3F4FC901880F991F820F931F65E08A
:1039800070E00E942B3E2EE129803A80229DC001EA
:10399000239D900D1124810F911D17FD9A95FB0118
:1039A000E80FF91F9F0150E040E060E070E0CB01BC
:1039B000E9833A834B835C836D837E838F8398870F
:1039C0009401A50160E070E080E090E0A980BA80F9
:1039D000C12CD12CE12CF12C00E010E00E94563FCC
:1039E0002A5E36494A4051096109710981099109E4
:1039F000E0E8AE2EF1E5BF2ECC24C3940E949F3E9A
:103A000059016A017B018C01A0911C4240911D4229
:103A100040901E420A2E000CBB0B20E13EE00E94AB
:103A20008D3E042C000C550866087708DC01CB019C
:103A3000840D951DA61DB71D3CE34302A001112472
:103A4000840F951FA11DB11D1C012D01612C712C2E
:103A500043013A82AB835C826D827E828F8298863C
:103A60009C01AD0160E070E080E090E00E94563F74
:103A700029014A01698779831C01F8941092CE6963
:103A8000A6EC6A2EA1E47A2E8AE0A82EB12CC12CD5
:103A9000D12CE12CF12C00E010E09201A401698509
:103AA0007981C1010E94F73EF30121933F01920108
:103AB000A40169857981C1010E94F93E29014A0169
:103AC000698779831C0122ED31E426153705E1F67B
:103AD00064EC71E48CEF91E40E940A1078942996CA
:103AE000CDBFDEBFDF91CF911F910F91FF90EF907F
:103AF000DF90CF90BF90AF909F908F907F906F900E
:103B00005F904F903F902F900895FC0195E020E04A
:103B10008191980FDF0111979A3060F49C9390E0A7
:103B2000211101C09E5F2F5F2E3011F09111F0CF57
:103B3000892F08959A509C9391E0F2CFCF938031D2
:103B400008F04AC0E82FF0E0E855F24E0C94753EBC
:103B5000B81DC51DDD1DEE1D341E4B1EEC1D611E66
:103B6000671E7A1E8B1E931E9B1EA31EAB1EAF1ECE
:103B70008091C3412EE0829FC00111246DE472E464
:103B80008C539E4BCF910C940A108091C341CEE090
:103B90008C9FC00111246DE472E48C539E4B0E94F3
:103BA0000A10E091C341CE9FF0011124ED54FE4B69
:103BB000118A128ACF910C943B1B8091C3413EE045
:103BC000839FC00111246DE472E480529E4B0E94D9
:103BD0000A1081E080931340CF9108958091C341F2
:103BE000811126C09091B34120914E4280E1289FDF
:103BF0009001112480914D42806C822B8923809307
:103C0000B3418091B3418F7339F78091C969909125
:103C1000CA699F7D8093C9699093CA698091C96977
:103C20009091CA699F7E8093C9699093CA69D4CFE5
:103C300023E040E06EE472E485EB91E40E9416100C
:103C40009091B84191709093B8412091B741809183
:103C5000B6413AE0239F800D1124911103C0809357
:103C60002E7DBACF8195FBCF8091C3412EE0829FFC
:103C7000C00111246DE472E484509E4B0E940A102E
:103C800080910B4282FD04C081E080931B42A4CF4F
:103C900010921B42A1CF24E040E06DE472E48EEB71
:103CA00091E40E94161089EB91E40E94C61A80915B
:103CB000B3419091B44194608093B3419093B441E7
:103CC0008BCF8091B3419091B4419B7FF5CF4091D0
:103CD000B3415091B4412091C341255F81E090E010
:103CE00002C0880F991F2A95E2F78095909584234A
:103CF0009523E2CF4091B3415091B4412091C3410B
:103D0000255F81E090E002C0880F991F2A95E2F7B5
:103D1000842B952BD1CF4091B3415091B441209148
:103D2000C341285FDBCF4091B3415091B441209112
:103D3000C341285FE6CF4091B3415091B4412091F7
:103D4000C3412A5FCBCF4091B3415091B441209100
:103D5000C3412A5FD6CF81E08093C3413DCF10920B
:103D6000C3413ACF7F928F929F92AF92BF92CF92F0
:103D7000DF92EF92FF920F931F93CF93DF93082F61
:103D800002950F70C02FD0E0E090F369F090F469D5
:103D900020EFE22223E0F222E02AFD2AE092F369FA
:103DA000F092F469C7010E940D14182F882381F046
:103DB000C701DF91CF911F910F91FF90EF90DF909E
:103DC000CF90BF90AF909F908F907F900C94E80F12
:103DD0008091A3419091A4418B3F910509F469C062
:103DE0008D3F910541F5CC54DD4FFE01C49180E03B
:103DF000C7FD8BE0FC2FFF709F2E00E02C2F207161
:103E0000822EDBE0D81B90E0FC01E45EFF4B7F01DB
:103E1000FC2FF0727F2E9C012B5C32486901C0742C
:103E2000FC01EB51F6495F01901213C081E08093D1
:103E3000074080930540DF91CF911F910F91FF9034
:103E4000EF90DF90CF90BF90AF909F908F907F903A
:103E50000895882069F06D2F8CE190E40E94F013A2
:103E6000E12FF0E0EF5CFD4B848DF70180831F5F55
:103E7000772069F06D2F85E39DE70E94F013E12F15
:103E8000F0E0EF5CFD4B848DF60180831F5FCC2357
:103E900071F06D2F85EE99E60E94F013E12FF0E0AE
:103EA000EF5CFD4B848D8170F50180831F5F0F5F98
:103EB000BBCF802FDF91CF911F910F91FF90EF909B
:103EC000DF90CF90BF90AF909F908F907F900C9499
:103ED0009E1D8230A1F038F08430E9F1C8F08530C1
:103EE00009F442C008956091C3418EE0689FB0011B
:103EF00011246C537E4B8DE492E40C940A10609173
:103F0000C3418EE0689FB001112460527E4BF3CF15
:103F10008091C341811117C08091B3418F7080930C
:103F20004D428091B34182958F7080934E42809133
:103F3000B4418F7080934F428091B44182958170DB
:103F400080935042089523E040E065EB71E48EE4F5
:103F500092E40C9416106091C3418EE0689FB0010A
:103F6000112464507E4BC7CF24E040E06EEB71E437
:103F70008DE492E4EECF6F927F928F929F92AF92F8
:103F8000BF92CF92DF92EF92FF920F931F93CF9346
:103F9000DF93182F12951F708DE492E40E94D313C3
:103FA0008091A3419091A4418B3F910509F4B9C040
:103FB0008D3F910509F440C0892B79F5112359F003
:103FC0008091F3699091F469807F9370812B809345
:103FD000F3699093F4690091F3691091F469C80151
:103FE0000E940D148823C9F00031110510F0005310
:103FF000110987E0809FE001819FD00D1124C457F3
:10400000DD4BADE4B2E467E04991542F52955F7007
:104010004F704D935D936A95B9F7DF91CF911F91E2
:104020000F91FF90EF90DF90CF90BF90AF909F9057
:104030008F907F906F900895153001F580912C7DC1
:1040400090912D7D90934F429C0194E03695279559
:104050009A95E1F72F7020934E428F7080934D42D6
:104060008091317D8823C9F21330B8F21530A9F25E
:1040700081E08093074080930540CFCFE12FF0E0AF
:10408000EC55FD4FC4910BE0C7FF00E02C2F2F70C3
:10409000822ED0E0912C3C2F3071732E802F90E037
:1040A000DC01A45EBF4B7D01BC2FB0726B2E9C0166
:1040B0002B5C32486901C074DC01AB51B6495D012B
:1040C000891471F2772069F0ED2FF0E0EF5CFD4B81
:1040D000D7018C91848FDF5F602F8CE190E40E9488
:1040E000F013662069F0ED2FF0E0EF5CFD4BD60198
:1040F0008C91848FDF5F602F85E39DE70E94F01332
:10410000CC2369F0ED2FF0E0EF5CFD4BD5018C91F5
:10411000848FDF5F602F85EE99E60E94F013939401
:10412000CFCF812FDF91CF911F910F91FF90EF9013
:10413000DF90CF90BF90AF909F908F907F906F90C7
:104140000C94691F6EE084EC91E40E942A1B6EE0DF
:1041500080EE91E40E942A1B6EE08CEF91E40E94B5
:104160002A1B6EE082ED91E40E942A1B6EE08EEE27
:1041700091E40E942A1B6EE08AE092E40E942A1BCE
:1041800064E085EB91E40E942A1B89EB91E40E9494
:10419000C61AE3EBF1E4108A808191818064808308
:1041A0009183808191819160808391834AE050E086
:1041B00069E070E081EF91E40E945F3F88E08093C6
:1041C0000B420C94511C6F927F929F92AF92BF92C0
:1041D000CF92DF92EF92FF920F931F93CF93DF93D3
:1041E000EAE2F0E480E691E0DF019C011D922150BB
:1041F0003040E1F7E3E4FDE782EADF011D928A95B2
:10420000E9F740E058EFDF0120E066E0A62E00E08D
:1042100014E176E1B72E99249394FA013491319602
:10422000D4913196C4913196E49111963C931197B3
:104230001796CC9317971896EC931897303108F08F
:1042400051C0822F6A2D0E94113E909F6001919F64
:10425000D00C11240D2C000CEE08FF08813009F45D
:1042600056C0823009F458C060E070E880E09927B9
:10427000C60ED71EE81EF91E1296CD92DD92ED9263
:10428000FC921597632F70E06D2E712C2630D0F4C0
:104290009C92B69E7001B79EF00C1124C301880F4A
:1042A000991F880F991F8E0D9F1D865D9F4B12963B
:1042B000CD90DD90ED90FC901597FC01C082D182ED
:1042C000E282F3821696DC931697B69EC001B79EE3
:1042D000900D1124865D9F4BF301E80FF91F208B91
:1042E000FC01C58B2F5F4C5F5F4F1996223109F09F
:1042F00094CFDF91CF911F910F91FF90EF90DF90BE
:10430000CF90BF90AF909F907F906F90089560E0A6
:1043100070E081E09927ACCF60E070E881E09927F8
:10432000A7CFE62FE69527E0AC01249FC001259F8B
:10433000900D11248F5C9D4BE80FF92FF11DE55A6C
:10434000FF4F808160FD82958F700895CF92DF923C
:10435000EF92FF929C01892F992782958F7066E1D9
:10436000689FA001699F500D1124FA01E65DFF4B83
:10437000948984E0989FF0011124E40FF51FE65D15
:10438000FF4BC080D180E280F38080E090E0C114D8
:10439000D104E104F10449F1C9019F70B701A601FC
:1043A000480F591F611D711D6BBFFA01A791AC0128
:1043B000569547955695479570E060E0505F6F4F72
:1043C0007F4F4C0D5D1D6E1D7F1D6BBFFA01479128
:1043D00050E0880F991F8670992702C05595479520
:1043E0008A95E2F78A2F942F9370FF90EF90DF90D9
:1043F000CF9008958091086A8823E1F30E94AE135C
:1044000090ED980F9A3030F09FE9980F963020F495
:1044100099EA980F892F08959FEB980F963010F422
:1044200099ECF7CF803231F390E0F4CF8A3310F07B
:104430008755089580530895F894E6EFF9E6108AB9
:10444000118A128A78940895F8949091086A9031AC
:10445000B1F0E091076AF0E0EA50F649808380917C
:10446000076A8F5F8093076A8091076A803110F036
:104470001092076A8091086A8F5F8093086A789427
:1044800008958091240886FFFCCF08951F920F9213
:104490000FB60F9211240BB60F928F93EF93FF93E9
:1044A000E091076AF0E080912008EA50F6498083A5
:1044B0008091076A8F5F8093076A8091076A8F7087
:1044C0008093076A8091086A8F3028F48091086A87
:1044D0008F5F8093086AFF91EF918F910F900BBED1
:1044E0000F900FBE0F901F901895CF93DF93EC01A4
:1044F000FE018491811103C0DF91CF9108950E9444
:10450000CC132196F5CF813408F0875F8F70089522
:1045100047E0489F9001499F300D11242F5C3D4B8F
:10452000BC016C5F7F4F8617970710F080E00895FD
:1045300050E040E0FA01E55AFF4FE20FF31FE0813F
:10454000E11109C04F5F5F4F4730510599F7019660
:10455000295F3F4FE8CF81E008959C01ADECBCECB2
:104560000E947E3EDC01CB0123E1B695A79597958D
:1045700087952A95D1F70895482F282F392FADEC2C
:10458000BCEC0E947E3E23E19695879577956795D2
:104590002A95D1F7842F2AE0629F8019112408956B
:1045A00082EC8093304281E08093A2418093CD6978
:1045B0008091254290E08093327D9093337D0895E1
:1045C00027E731E0829FD001839FB00D1124A75FC0
:1045D000B549629FF001639FF00D1124E75FF54933
:1045E0008EEE92E001900D920197E1F7089597E029
:1045F000899FB001112430E020E0A901460F571F28
:10460000FA01E053F64944575D4BDA019C919083DF
:104610002F5F3F4F2730310581F7089527E0829FB4
:10462000C001112430E020E0A901480F591FFA0110
:10463000E053F64944575D4B6081FA0140816413B1
:1046400007C02F5F3F4F2730310571F781E0089594
:1046500080E008950F931F93CF938C01562F44232E
:10466000D9F06A30C8F4C0E0222319F0FC0120839D
:10467000C1E0852F90E00E94BC22F801EC0FF11DF3
:10468000805D8083E1E0EC0FE00FF12FF11D1082DF
:10469000CF911F910F910895252F30E0ADECBCEC28
:1046A0000E947E3E23E196958795779567952A959A
:1046B000D1F7605DF8016083DBCF1F93CF93DF9369
:1046C000CDB7DEB72597CDBFDEBF182F6091224250
:1046D00020E041E0CE0101960E942A2380912B42E6
:1046E00024E08202C00111242FEF40E0612F8954A1
:1046F00096400E942E172FEF40E0682F8DE20E9417
:10470000B016682F8091F14280FF21C02FEF40E06A
:10471000CE0101960E9411172FEF40E0682F8DE225
:104720000E94B016E091214294E0E902F0011124C8
:104730002FEF40E0682FCF01895796400E942E1737
:104740002596CDBFDEBFDF91CF911F910895809157
:10475000214224E08202C00111242FEF40E089575A
:1047600096400E942E172FEF40E0682F8DE20E94A6
:10477000B0162FEF40E0682FCE0101960E9411176E
:10478000DFCF1F93CF93DF93CDB7DEB72597CDBF94
:10479000DEBF182F80911B42813009F040C060912C
:1047A0002A4220E241E0CE0101960E942A232FEF07
:1047B00040E0612FCE0101960E9411172FEF40E0DB
:1047C000682F8AE30E94B016182F60911D4220E0E6
:1047D00040E0CE0101960E942A232FEF40E0612F96
:1047E000CE0101960E941117682F80911B428130E3
:1047F00079F480911C422FEF40E08C30ACF080E5E2
:104800000E94B0162FEF40E0682F8DE40E94B01692
:104810002596CDBFDEBFDF91CF911F9108956091A6
:104820001C4220E240E0BFCF81E4EACFCF92DF928A
:10483000EF92FF921F93CF93DF937C01EB01142F34
:104840000E94BC22805D8A839701ADECBCEC0E9483
:104850007E3E6B017C0133E1F694E794D794C794D4
:104860003A95D1F7C6018A309105D8F0A701960193
:104870000E94943E23E196958795779567952A95B2
:10488000D1F7605D6883C6010E94BC22805D898388
:104890001B82DF91CF911F91FF90EF90DF90CF901F
:1048A00008951883892B79F71983F2CF0F931F93FB
:1048B000CF93DF93EB0197FF2FC000271127081B31
:1048C000190B873F9F4F1CF58DE28883C8010E941A
:1048D000BC22805D8A832DEC3CECD8010E948D3E89
:1048E000DC01CB0123E1B695A795979587952A958D
:1048F000D1F7009721F00E94BC22805D898383E478
:104900008B831C82DF91CF911F910F91089580E2DC
:1049100088838DE28983DACF20E2288329838C0182
:10492000D5CFCF92DF92EF92FF92CF93DF937C01AE
:10493000EB010E94BC22805D8B839701ADECBCEC47
:104940000E947E3E6B017C0133E1F694E794D7949C
:10495000C7943A95D1F796012A30310588F0A7011E
:104960000E94943E23E196958795779567952A95C1
:10497000D1F7605D6883C6010E94BC22805D05C0DE
:1049800080E38883C114D104B1F78A838EE28983DE
:1049900086E58C831D82DF91CF91FF90EF90DF90B1
:1049A000CF90089585E08093A0001092A4008FEF2F
:1049B0008093850689E48093080681E08093000651
:1049C00080930A0680910D0680FFFCCF209110068F
:1049D0003091110684E0369527958A95E1F750E0ED
:1049E00040E060E070E686E090E00E94533E109266
:1049F000000681E080930D06C901089520910611FB
:104A000030910711A0910411B091051181E08093BC
:104A1000A00092E4909308068093000680930A0613
:104A200080910D0680FFFCCF8091100690911106B9
:104A300044E0969587954A95E1F7281B390B0E942B
:104A40007E3EDC01CB01985FAF4FBF4F1092000656
:104A50005CE0B695A795979587955A95D1F70895F7
:104A6000E62FE69527E0829FC00111248F5C9D4BC5
:104A7000E80FF92FF11DE55AFF4F808160FD829507
:104A80008F70089527E0289FD001299FB00D112431
:104A900030E020E0F901EA0FFB1FE457FD4B908165
:104AA000492F4F70FB01408392959F7091832F5F38
:104AB0003F4F6E5F7F4F2730310561F708958F922A
:104AC0009F92BF92CF92DF92EF92FF920F931F932C
:104AD000CF93DF93CDB7DEB76897CDBFDEBFD42EBF
:104AE0008E010F5F1F4FAE01435F5F4F780120E2E1
:104AF000D7012D937D011B961C921B974A175B07CC
:104B0000B9F7382F4C0120E072E0CC24C39483E045
:104B1000B82E882D831B8617D8F4D401ED914D0152
:104B2000822F90E0E7FD54C0E03618F4E03488F1BD
:104B3000E054800F911FDC01EC93F4018081982FE9
:104B40009D7F9C3219F08A3309F040C02C3008F365
:104B500085E020E04D2D682FD8018D918D010E94B8
:104B600044184D2D682FF80183850E948C180E156E
:104B70001F0579F76896CDBFDEBFDF91CF911F91FA
:104B80000F91FF90EF90DF90CF90BF909F908F900C
:104B90000895E03238F0EA3349F4840F951FDC01C0
:104BA0007C9314C0F0E0E85FFC4FE491EE3251F0EA
:104BB000EA3B99F3EC3209F0BCCF840F951FFC015E
:104BC000B08204C0840F951FFC01C0822F5FBECF4E
:104BD000EAE3AFCF2F923F924F925F926F927F9214
:104BE0008F929F92AF92BF92CF92DF92EF92FF92FD
:104BF0000F931F93CF93DF93CDB7DEB7A697CDBFAB
:104C0000DEBF8C014B018430910510F40E94F72225
:104C10009E012F5F3F4F79013E013DE0630E711C05
:104C2000570180E2D5018D935D011B961C921B9765
:104C30006A167B06B9F787E0809F9001819F300D4F
:104C40001124F901EE56FD4B8081803109F08BC0B3
:104C500085E090E0682FF901E80FF91FE457FD4B5C
:104C60004081411103C00197A8F76FEF6F5F90E09B
:104C7000462F50E087E0809FD001819FB00D112426
:104C8000AF5CBD4B292F092E000C330B24173507C1
:104C90000CF10430110508F047C0402F440F4F5F5E
:104CA000CE0149960E945F25A696CDBFDEBFDF915B
:104CB000CF911F910F91FF90EF90DF90CF90BF9019
:104CC000AF909F908F907F906F905F904F903F90AC
:104CD0002F900895FA01E21BF30BEA0FFB1FE65A2F
:104CE000FF4F808187FD1EC0803280F48823C1F091
:104CF0007EEF780F7230B0F079EF780F753090F06A
:104D000072EF780F7F3070F08E3160F4E9E1F0E0FF
:104D1000EC0FFD1F2E0F3F1FF90180839F5FB2CF65
:104D20008AE0F4CF82E0F2CF8BE0D4018C9380E272
:104D300011968C9320E0822F022E000C990BFC011F
:104D40003296E80DF91D8417950714F01082ACCF48
:104D500069E170E06C0F7D1F860F971FDC018C915D
:104D600080832F5FE8CF6E01B9E1CB0ED11CB60175
:104D7000C8010E9442255090F142E1E0B3E04B2E81
:104D800053FC03C0E3E0442443949091EF42929596
:104D90009C70A091F042AF70FA2F898D2A8D482F18
:104DA0003AE0239F400D11245B8D5523F1F024E65A
:104DB000241B422F51E09830D1F4622F220F770B41
:104DC0002A2F30E02F5F3F4F261737070CF452C0D1
:104DD00051E06217730721F49DA151E0953018F05E
:104DE00098E04A3024F090E002C09830C9F32EA138
:104DF000222311F02DE22983943009F414C1983054
:104E0000D9F191115FC1EE87A83008F0D8C09601A2
:104E10002A1B3109D90171E01B968C91853008F469
:104E200070E0772473947F0E2DE030E0872D072CFF
:104E3000000C990BD901A81BB90BAC0DBD1D6C91D1
:104E4000670F70E06A3010F060E071E08E0D9F1D1A
:104E5000605DDC016C937A947110E8CF713009F0D9
:104E6000DFC081E38A83552309F4ACC041508DE251
:104E70008A87A9C051E0B7CF513009F04FC081E017
:104E80008A0F982F941BD601A91BB10997FDB395E2
:104E900091E01C962C91253008F490E01EA2042E7F
:104EA000000C550B6DE070E06701C40ED51E282F75
:104EB000082E000C330B3901641A750A77FC0CC0FC
:104EC000DB01A21BB30BAC0DBD1D5896FC91F90F75
:104ED00090E0FA3010F091E0F0E02E0D3F1DF05D13
:104EE000D901FC93815019F7EE870430110508F0C1
:104EF0001FC1000F0F5F85E020E0402F682FD70112
:104F00008D917D010E944418402F682FF701838501
:104F10000E948C18AE14BF0479F7C6CE8F5F8A0F3B
:104F20008A3064F5F1E0D601A81BB10987FDB3957D
:104F30001C969C91953008F4F0E0082E000C990B1B
:104F4000D601A81BB90B9D01235F3F4F1901BC017E
:104F50001816BCF0F13049F14F5FD301A40FB11D19
:104F6000EC9352FEC2CF435014160CF0BECFD301C7
:104F7000A40FB11D47FDBA954C92F5CFF52F8AE0ED
:104F8000DCCFD101DD901D01DF0EB9E0F52FBD159D
:104F900010F4D52EF1E09701280F391FA0E3CA2E97
:104FA000DC0CD901DC920197D3CF81E38A836C0FAB
:104FB0007D1F80E3DB0112968C934E5FCECF70E0B5
:104FC000F7E02FCF4F5F242F042E000C330BADECF6
:104FD000BCEC0E947E3EDC01CB0133E1B695A79587
:104FE000979587953A95D1F720E3280F2B8720E3F3
:104FF000240F36EF839F200D11242C87442309F4BE
:1050000074CF8A81803309F070CF433609F06EC0C7
:1050100041E02F2FFF0F330B2F5F3F4F59E35EC04F
:10502000552389F224CFA83008F03FC0B6016A1B8F
:105030007109DB0161E01B968C91853008F460E01A
:1050400071E07F0F2DE030E0872F072E000C990BC9
:10505000D901A81BB90BAC0DBD1DAC91A60F60E02A
:10506000AA3010F061E0A0E08E0D9F1DB0E35B2E32
:105070005A0EDC015C92715039F7613001F581E321
:105080008A835523A1F04150141614F48DE28A87C7
:105090004E5F23E0842F622F0E941D3E291B491B77
:1050A000620E711CD301EC938ECFF7E0C8CF4F5F37
:1050B000842F63E00E941D3E21E0290FF0CF55238D
:1050C000B9F3E2CF442309F410CF983009F099CF17
:1050D0000CCF8E0D9F1DDC015C934F5F842F042E3F
:1050E000000C990B28173907A4F7FFCE81E38A83B8
:1050F0005523E1F04150242F042E000C330BADEC6E
:10510000BCEC0E947E3EDC01CB0123E1B695A79565
:10511000979587952A95D1F720E3280F2B87405D37
:10512000F6EF8F9F400D11244C87DFCE4F5FE3CF0A
:1051300080E09CE22EE2D7013D917D01D401A80FD1
:10514000B11D3C9341E0480FD7011B963C913E13A3
:1051500010C0D401A40FB11DE13049F42C938E5F2F
:10516000AE14BF0441F7880E911CF401EFCD9C935F
:10517000F6CF842FF5CFCF93DF93CDB7DEB72E9741
:10518000CDBFDEBFBE016F5F7F4F90E00E94422522
:105190008E8581111AC09B81911111C029818D8545
:1051A000222369F09AE03C85899F300D1124832FDA
:1051B000223028F02B85399F200D1124822F2E9626
:1051C000CDBFDEBFDF91CF91089580E0F8CFF89496
:1051D000E5EAF1E411861086128613861486158698
:1051E000789408958F708A3010F0895A0895805D00
:1051F0000895CF93C82F82958F700E94F2280E9445
:10520000CC138C2F8F700E94F228CF910C94CC136A
:105210001F93CF93DF9327E0289FE001299FD00DB4
:105220001124CD56DD4B16E08A9182958F700E9435
:10523000F2280E94CC1388818F700E94F2280E946D
:10524000CC13115088F7DF91CF911F9108950F93E0
:105250001F93CF93DF938C01EC012E968A918F7070
:105260000E94F2280E94CC130C171D07B9F7DF919A
:10527000CF911F910F9108950F931F93CF93DF93B9
:105280008C01EC0125968A918F700E94F2280E9471
:10529000CC130C171D07B9F7DF91CF911F910F9118
:1052A0000895CF93C82F892F0E94F228803311F0E0
:1052B0000E94CC138C2F82958F700E94F2280E943E
:1052C000CC138C2F0E94F228CF910C94CC131F93F7
:1052D000CF93DF93D82F162FC42F82958F700E9403
:1052E000F22820E04C2F612F0E94B016182F8D2F2E
:1052F0000E94F22820E04C2F612FDF91CF911F9167
:105300000C94B0161F93CF93DF9320E046E060E645
:1053100089EC9AEF0E942E17CFE1D1E116E0988137
:10532000412F682F892F0E946729C03191E1D90749
:1053300021F4DF91CF911F910895C83111F41F5FBF
:1053400088E72197ECCF9091AF419830BCF4E09181
:10535000AD41F0E0EB55FE4B80838091AD418F5F16
:105360008093AD418091AD4187708093AD41809134
:10537000AF418F5F8093AF4181E0089580E0089551
:10538000E091AD41E81BFF0B3197E770FF27EB552C
:10539000FE4B80810895F8948091AF411816BCF4BB
:1053A000E091AE41F0E0EB55FE4B80819091AE4133
:1053B0009F5F9093AE419091AE4197709093AE41B4
:1053C0009091AF4191509093AF41789408958FEFB1
:1053D000FCCF1F920F920FB60F9211240BB60F92B3
:1053E0002F933F934F935F936F937F938F939F93ED
:1053F000AF93BF93CF93DF93EF93FF938091CE69E9
:105400008F5F8093CE698091CE6983708093CE69DF
:105410008091B3419091B44186FF28C084EC91E41F
:105420000E94851D882349F08091B3419091B44139
:1054300082608093B3419093B4418091B341909145
:10544000B44190FF13C064EC71E480EE91E40E94DB
:10545000B71A882359F08091B3419091B44181608B
:105460008093B3419093B441109211408091B34125
:105470009091B44187FF28C082ED91E40E94851D80
:10548000882349F08091B3419091B4418860809322
:10549000B3419093B4418091B3419091B44191FF55
:1054A00013C062ED71E48EEE91E40E94B71A882376
:1054B00059F08091B3419091B44184608093B3419D
:1054C0009093B441109211408091B3419091B441B6
:1054D00092FF19C089EB91E40E94851D6EEB71E487
:1054E00089EB91E40E94CD1A882369F089EB91E45D
:1054F0000E94C61A8091B3419091B441806180931B
:10550000B3419093B4418091B3418F73D9F08091AE
:10551000C9699091CA6990628093C9699093CA6978
:105520008091C9699091CA6990618093C96990938B
:10553000CA6981E08093E57D80911140813011F44A
:10554000109211408091CE69811186C080911140E6
:10555000823049F08091347D882329F08091347D18
:1055600081508093347D80911E428F5F80931E42D4
:1055700080911E428C330CF46FC081E08093134005
:1055800010921E4280911D428F5F80931D420E94A7
:10559000FE24E82F8FEE8E0FEA52893114F4E9E1F0
:1055A000E81B0E2E000CFF0BE553F14EE4918091A9
:1055B0002E7DE80FE093460180911D428C330CF460
:1055C0004BC010921D4280911C428F5F80931C4201
:1055D00080911C428831D4F110921C428091224269
:1055E0008F5F80932242C091224260911F4270914E
:1055F0002042809121420E946A190C2E000CDD0B82
:105600008C171D06BCF491E09093224280912142B8
:105610008F5F80932142809121428D305CF0909386
:10562000214280911F4290912042019680931F4217
:1056300090932042409122426091214280911F42EA
:10564000909120420E94201980932B4280911C420D
:105650000E94801980932A4281E080935301FF9138
:10566000EF91DF91CF91BF91AF919F918F917F91FA
:105670006F915F914F913F912F910F900BBE0F90C3
:105680000FBE0F901F9018951F920F920FB60F929A
:1056900011242F933F934F938F939F9381E0809397
:1056A00012408091B241813089F58091084081504B
:1056B0008093084080910840811128C08091264243
:1056C000809308404EB180912F7D9091307D880F5E
:1056D000991F21E030E04F3F11F430E020E0822BB1
:1056E000932B80932F7D9093307D80912F7D90918F
:1056F000307D892B59F41092B241109202408FEF05
:105700008FB99DE090936B0480936C0481E080934B
:105710000B0A9F918F914F913F912F910F900FBE48
:105720000F901F901895CF93DF9300D000D0CDB786
:10573000DEB780911340813009F04EC00E94D22420
:105740002091417D3091427D820F931F96958795E0
:105750008093417D9093427D209127424CE251E01D
:10576000BA01EAE02E9F6019710911249B01369558
:10577000279536952795BA01621B730B6817790731
:1057800088F582E1898385E18A8386E18B831C82A7
:105790006FEF80E00E9465162FEF40E062EECE01D1
:1057A00001960E94111781E00E945D2380E60E940D
:1057B000C123E0EEF1E48EEE91E42191211138C095
:1057C0008E179F07D1F780E00E94F91561E080E015
:1057D0000E947416109213402496CDBFDEBFDF9155
:1057E000CF910895B901660F771FFA01E61BF70BF9
:1057F000E817F90720F482E1898384E1C5CF620FBD
:10580000731FFA01E61BF70BE817F90720F482E192
:10581000898383E1B9CF220F331F220F331F421B2D
:10582000530B4817590710F481E1F2CF80E1F0CF14
:105830002FEF40E068EC87E00E94B016C4CF0895D7
:10584000CF92DF92EF92FF920F931F93CF93DF934C
:105850008091114081118CC0D12CC2E0CC2ED4E7B4
:10586000ED2ED4E0FD2E11E08091F5698230F1F546
:10587000809128409091294080937C4290937D4272
:10588000D09210400E94DE0FFC01808180930F4077
:1058900080917C4290917D422091024021110AC06A
:1058A0008C3FF1E19F0739F5E0920340F09204400C
:1058B000109302400E94A6219C01369527953695AB
:1058C0002795D22E7091CF6970932F421092CF6995
:1058D0004091F569423009F4FEC1A0F4442331F14E
:1058E000413009F49EC11092F5693EC080917A4220
:1058F00090917B42C1CF883C20E19207D9F6C092BB
:105900000240D8CF443009F4F6C108F4E7C145306D
:1059100051F720917A4230917B422F5F3F4F209385
:105920007A4230937B4280FDDECF9ECF40917A4217
:1059300050917B42FA013196E0937A42F0937B4298
:10594000682F6370623031F1633009F459C16130FE
:10595000C1F0F901FF27EE0FFF1FEC55FF4F4591F6
:105960005491822FFA0109958091F56981117CCFBC
:10597000DF91CF911F910F91FF90EF90DF90CF902B
:1059800008956093F5698093F1699093F26970933B
:105990001B40EACFD22FD695D695D695C22FC77089
:1059A000EFEFEC0FE73078F4F0E0E752F34D0C94B2
:1059B000753E2A2D132DE02C182D212D242D272D59
:1059C0002DE060E005C00E94DE0FFC016081262F03
:1059D0002093CC69D150DF3108F03EC0ED2FF0E0CC
:1059E000EC50F34D0C94753E322D362D3A2D422D50
:1059F0004A2D4E2D542D5A2D602D682D6C2D722D53
:105A00007C2D912D962D9B2DA12DA72DAF2DBA2D3F
:105A1000B82DC12DC92DCF2DD82DDD2DE32DE72D8E
:105A2000ED2DF12DF52D0E94DE0FFC012081C9CF57
:105A3000609177422091784226170CF0C9CF2DE073
:105A4000C7CF22E062E0C4CF2CE063E0C1CF2DE0FD
:105A50006DE0BECF22E0B5CF422F81E392E40E94F9
:105A6000271082CF422F8FE392E4F9CF422F8DE4AB
:105A700092E4F5CF462F6FE372E481E392E40E9453
:105A8000301072CF462F61E372E48FE392E40E94FC
:105A900016106ACF462F6DE472E4EFCF462F6FE306
:105AA00072E48DE492E4F3CF462F6DE472E48FE369
:105AB00092E4E5CF462F6DE472E481E392E4E7CF10
:105AC000462F6FE372E481E392E40E9443104CCFCF
:105AD000462F6DE472E4F7CF1093CF69462F70E044
:105AE00060E0F1CF022F262F4FE352E461E372E42E
:105AF000CB010E946F1038CF1093CF69C73061F48B
:105B0000809189428A3041F480913E428B3020F06E
:105B1000895080933E4228CF022F262F50E040E04C
:105B2000E5CF022F262F4DE452E4E0CF462F6DE45F
:105B300072E4CB01CACF462F61E372E48DE492E4B4
:105B4000C4CF1093CF69462F70E060E0F7CF022FEB
:105B5000262F4DE452E461E372E4CA01CACF1093E8
:105B6000CF69022F262F50E040E06DE472E4C0CFF1
:105B70001093CF69022F262F4DE452E470E060E0CD
:105B8000ECCF462F70E060E08FE392E40E94B1100A
:105B9000EBCE462F70E060E08DE492E4F7CF022F69
:105BA000262F4DE452E461E372E490E080E0A1CF5F
:105BB000022F262F4FE352E4F6CF462F70E060E02D
:105BC00081E392E4E3CF462F6DE472E4F9CF422FF4
:105BD00081E392E40E94A210C7CE422F8FE392E4A9
:105BE000F9CF422F8DE492E4F5CFC1E3D2E4C20FA6
:105BF000D11D261B4A9149832A95E1F71882B4CE1C
:105C0000822F86958F7327FD805421702713B0CE85
:105C1000480F511D87FD5A9540937A4250937B421D
:105C2000A3CE40917A4250917B424F5F5F4F4093A9
:105C30007A4250937B421092F56960911B409C011F
:105C4000217033276217130609F092CE2091F16973
:105C50003091F2693695279536952795BC01E6E097
:105C6000660F771FEA95E1F76627262B372B81FF12
:105C700005C020937A4230937B4276CE8091824257
:105C80009091834280938442909385428091804298
:105C900090918142809382429093834280917E4290
:105CA00090917F42809380429093814240937E42C4
:105CB00050937F4220937A4230937B42C9010E94E5
:105CC000A621892B09F050CE0E94D11080937A42F0
:105CD00090937B4249CE0E94581346CE20917A423F
:105CE00030917B422F5F3F4F20937A4230937B422B
:105CF0000E94581339CE882351F080917A429091B6
:105D00007B42019680937A4290937B42ECCD109235
:105D10007A4210927B428091317D882319F0109352
:105D20001140E1CD1092E57D1093CF69C0921140F2
:105D30001092347DD8CD0F931F93CF93DF93182FFC
:105D4000D62FC1E001E0DC1728F4DF91CF911F913D
:105D50000F910895111105C08091EF4281608093E9
:105D6000EF420E94D022109211400093E57D0E94E4
:105D7000202C809111408130D1F7CF5FE4CF4F923A
:105D80005F926F927F928F929F92AF92BF92CF92CB
:105D9000DF92EF92FF920F931F93CF93DF93CDB7D4
:105DA000DEB72E97CDBFDEBF0091F64210E0102F78
:105DB000002700271F708091F542082B48010093AF
:105DC0001740109318404EEE642E42E4742ECE011C
:105DD00001965C0107966501F3012191D6012D938F
:105DE0006D01A817B907C9F7E0901540F09016406B
:105DF000E016F10668F5F801EE19FF097F0180E071
:105E00000E94C029823009F05AC0EA94EF2809F0B4
:105E100056C0043011050CF452C081E00E94C02924
:105E200063E08232C1F485E00E94E02261E083E019
:105E30000E94E02263E080E00E949B2E0E94361ABE
:105E400081E00E94691A63E081E00E949B2E0EC0EF
:105E5000E01AF10AD4CF81E00E94E02265E083E0FD
:105E60000E94E0226BE085E00E94E02269E081E090
:105E70000E947416D5018D915D01F30181933F015C
:105E8000AC15BD05B9F780911740909118408093EB
:105E90001540909316402E96CDBFDEBFDF91CF9177
:105EA0001F910F91FF90EF90DF90CF90BF90AF9038
:105EB0009F908F907F906F905F904F90089580910A
:105EC000EF4281FF14C0809114408111CFCF63E075
:105ED00081E00E94E02265E083E00E94E0226BE026
:105EE00085E00E94E02281E080931440BFCF1092B1
:105EF00014400430110534F5119501951109000F76
:105F0000111F0A5F1F4FFF24F3948F2D0F2C000CDD
:105F1000990B0817190780F455245394442443948B
:105F200083E0E82EF12C052D052C000C110B8016BA
:105F3000910660F4682D88CF60E08F2D0E94651671
:105F4000F394E3CF93E0892E912CE6CF8091EF423A
:105F500081608093EF420E94D022109211404092C3
:105F6000E57D0E94202C809111408130D1F70E9464
:105F7000361AC701801B910B880F8F5F0E94691A28
:105F80005394D1CF20912C42022E000C330B2F5F63
:105F90003F4FAC01249FC001259F900D349F900D71
:105FA0001124019708F40895EFECF7E03197F1F729
:105FB00000C00000F6CF1F93CF93DF9383E090E003
:105FC0000E94C22FC0E4D4E018E01E8383E090E07A
:105FD0000E94C22F1D8381E090E0DF91CF911F913D
:105FE0000C94C22FEF92FF921F93CF93DF930E94E6
:105FF000DB2FC5E7DEE1FE0114911123F1F03196AC
:10600000849122968F3F29F484E690E00E94C22F6B
:10601000F2CF84910E94C6157E01F7018FEFE81A36
:10602000F80A8E2D8C1B811720F01150C10FD11D45
:10603000E2CF84910E94BF15F0CFDF91CF911F91E5
:10604000FF90EF90089520912C42022E000C330B0C
:106050002F5F3F4FAC01249FC001259F900D349FBF
:10606000900D1124019708F4089552E05A95F1F724
:1060700000C0F8CF1F920F920FB60F9211240BB6EB
:106080000F92BF92CF92DF92EF92FF920F931F93E6
:106090002F933F934F935F936F937F938F939F9330
:1060A000AF93BF93CF93DF93EF93FF9380EA8093F7
:1060B000010488E080936B048FEF80936C04DFB160
:1060C0008FB9DD2309F492C0ED2EF12C97012150F8
:1060D00031092D233F21232B09F088C090911140D5
:1060E000923049F4109211408FB99DE090936B0467
:1060F00080936C0455C010E000E08FE1B82ECC24F2
:10610000C394D12CC02FB0920204C601002E01C04E
:10611000880F0A94EAF78093010485E090E00E94DA
:1061200023308EB190E0809590958E219F21892B10
:1061300031F40F5F1F4F0530110521F7C5E080E0F6
:10614000D69509F049C0CC0FCC0FCC0FC80FC83280
:1061500008F044C0D6E910EA80911A4281111093E8
:1061600007048EE591E00E942330D150A9F78C2FCF
:106170000E94A329882359F081E08093B24124E64C
:1061800032E32093034030930440809302408FE138
:106190008093010410921140809119428093347DC4
:1061A000FF91EF91DF91CF91BF91AF919F918F912F
:1061B0007F916F915F914F913F912F911F910F911F
:1061C000FF90EF90DF90CF90BF900F900BBE0F909D
:1061D0000FBE0F901F9018958F5FB2CF8FEF8FB9C2
:1061E0009DE090936B0480936C04D1CF8FEF7CCFB4
:1061F000CF92DF92EF92FF92CF93DF93A3E4BDE7BC
:1062000026E036E1D7964C91D7974F3F61F150E0A9
:10621000DC968C91DC9790E0D6966C91D6976130A5
:1062200069F5DD966C91DD97EC01CC0FDD1FCC0F8D
:10623000DD1F349FF001359FF00D1124CE0FDF1FBD
:10624000C65DDF4BD896CD90DD90ED90FC90DB974E
:10625000C882D982EA82FB82E65DFF4B8E0F9F1FC8
:10626000EC01288B658B2F5F1996223159F6DF914F
:10627000CF91FF90EF90DF90CF900895349FB001C1
:10628000359F700D1124EB01C65DDF4BC80FD91F80
:1062900048894213E8CFFC01EE0FFF1FEE0FFF1FEE
:1062A000E60FF71FE65DFF4B108211821282138208
:1062B000DACF1F93CF93DF93CDB7DEB76C97CDBF07
:1062C000DEBF11E060E0812F0E9465161F5F17306E
:1062D000C9F780912C7D81FD37C080912D4282309D
:1062E000F1F1833069F0813079F520E046E061E03A
:1062F00089E50E94B01670E060E082E090E022C084
:1063000020E042E061E084E50E94B01620E044E035
:1063100061E08AE50E94B01620E046E061E089E590
:106320000E94B01670E060E082E090E00E94EA25F2
:1063300070E060E081E090E00E94EA2570E060E0BB
:1063400090E080E00E94EA2566E081E00E947416F9
:106350006C96CDBFDEBFDF91CF911F91089520E0F5
:1063600046E061E081E40E94B016E7ECF2E467E108
:106370008291811102C06150D8F76F5F89F420E0EB
:1063800045E065E08DEC9AEF0E94D21885E00E940E
:10639000371620E046E061E081E40E94B016D4CFD9
:1063A000E62FF0E0E155FD4BCE010196DC01229194
:1063B0002D932A2F281B2617D4F345E00E945F2532
:1063C000E8CF7F928F929F92AF92BF92CF92DF924F
:1063D000EF92FF920F931F93CF93DF93CDB7DEB76A
:1063E0006597CDBFDEBF4C017A01CA0140968B0193
:1063F000041B150B6817790710F000E110E040E36B
:10640000BE016F5F7F4FC7010E9416248DE28C830F
:106410001D822FEF40E06EEBCE0101960E94111716
:1064200040E3BE016F5F7F4FC7010197800F911F4F
:106430000E9416242FEF40E06EEDCE0101960E94DF
:1064400011178E0C9F1CC12C8AE3782EAC2CB12C1A
:10645000A016B10688F06596CDBFDEBFDF91CF9163
:106460001F910F91FF90EF90DF90CF90BF90AF9072
:106470009F908F907F900895BE016F5F7F4FC50101
:10648000880D991D0E94EA25DC2CD694D394C0FC7B
:1064900021C040E2BE016F5E7F4FC5018E0D9F1D82
:1064A0000E9416247C8A1D8A20E04D2D61E0CE01D9
:1064B00041960E94111720E04D2D62E2CE01019617
:1064C0000E94111720E04D2D6AE88CE70E94B0165B
:1064D000C394BCCF20E04D2D62E9CE0101960E940D
:1064E0001117F6CF8130A9F028F08230F9F083300F
:1064F00059F1089588ED94E184BF909368008AE98A
:1065000090E08093260A9093270A88E08093020601
:10651000089588ED9CE184BF9093680085E391E045
:106520008093260A9093270A8AE0F0CF88ED25E22F
:1065300030E084BF2093680080ED91E08093260ACC
:106540009093270A8BE0E2CF88ED2DE230E084BF04
:10655000209368008BE692E08093260A9093270AA6
:106560008CE0D4CF84EF91E00E94C22F81E380932E
:10657000600980912C420C94723283E00E94723246
:10658000E0E2F8E087E594E08087918783E0878305
:106590008681806C868380E8858384E690E00C9415
:1065A000C22FCF93DF93109260090E94BD328CE01E
:1065B0000E94CC1383ED9AEF0E947522C9E0DAE6BF
:1065C000899182958F700E94F2280E94CC13FE015F
:1065D000319780818F700E94F2280E94CC138AE745
:1065E000C632D80769F78AE00E94CC1389ED9AEF8A
:1065F0000E94752284E00E94CC13DF91CF910C940D
:10660000B2320F931F93CF93DF93109260090E94D1
:10661000BD328CE00E94CC138AE00E94CC1387EF3D
:106620009AEF0E947522D0E0C0E0CE010E9488223D
:106630008823E1F0CE01C031D10508F0C0960E9458
:10664000512980E20E94CC1310E000E0C8018C0FB9
:106650009D1F0E94082980E20E94CC130F5F1F4FEC
:106660000430110599F78AE00E94CC132496C03CAF
:1066700043E0D407D1F681E40E94CC138AE30E9460
:10668000CC1380E20E94CC1381E392E40E9427297C
:1066900080E20E94CC1380E20E94CC1382E40E942C
:1066A000CC138AE30E94CC1380E20E94CC138FE3C8
:1066B00092E40E94272980E20E94CC1380E20E948B
:1066C000CC1383E40E94CC138AE30E94CC1380E2B3
:1066D0000E94CC138DE492E40E9427298AE00E9454
:1066E000CC1383E50E94CC138AE30E94CC1380E292
:1066F0000E94CC13CDE0D0E001E010E020918A426E
:1067000030918B42C8010C2E02C0880F991F0A9449
:10671000E2F782239323892B09F055C080E30E947E
:10672000CC13219758F78AE00E94CC138DE40E9485
:10673000CC138AE30E94CC1380E20E94CC138BE539
:1067400092E40E94272980E20E94CC1380E20E94FA
:10675000CC138EE40E94CC138AE30E94CC1380E217
:106760000E94CC1389E692E40E94272980E20E94CD
:10677000CC1380E20E94CC1387E40E94CC138AE3FE
:106780000E94CC1380E20E94CC13809187428F70CC
:106790000E94F2280E94CC13809186428F700E9442
:1067A000F2280E94CC138AE00E94CC1389ED9AEF64
:1067B0000E94752284E00E94CC13DF91CF911F913B
:1067C0000F910C94B23281E3AACFCF9388E790E087
:1067D0000E94C22FC0E08091B241813019F08C2F0D
:1067E000CF91089582E390E00E94C22F7299F3CF77
:1067F0008FEF0E942B166BE080E00E9474160E94BF
:10680000D1328FEF0E942B166BE080E00E9474164D
:10681000C1E0E1CF2F923F924F925F926F927F92B1
:106820008F929F92AF92BF92CF92DF92EF92FF92A0
:106830000F931F93CF93DF93CDB7DEB76C97CDBF88
:10684000DEBF8091E94220E1829FC00111242091A6
:10685000E84222952F70822B20E032E04901881A0D
:10686000990AAC01405351094B8F5C8FD12CC12C3C
:10687000F12CE12C512C4FEA642E4DE7742E2FEFB2
:1068800031E0D901A81BB90BA98FBA8F0E9420163D
:106890006FEF80E00E9465166FEF89E00E94651639
:1068A0006FEF8AE00E946516B6E05B9EC00111247E
:1068B0002FEF40E061E0895296400E942E17E1E1FF
:1068C000E51520F1E52DF0E0E859FB4C0C94753E00
:1068D0007A34D034E634C435CE35DD35A8350A35C2
:1068E000BA3454351435913643361037C534F6343E
:1068F0008634023706E31BEF27E23BEF43E15BEF11
:1069000062E27BEF89E09BEF0E9458176BE080E02A
:106910000E94741680EA8093020480915000897F5F
:10692000846080935000809150008160809350007B
:106930008895809150008E7F809350008091347DA7
:10694000811150C3109211406C96CDBFDEBFDF9114
:10695000CF911F910F91FF90EF90DF90CF90BF905C
:10696000AF909F908F907F906F905F904F903F90EF
:106970002F90089502E31BEF2FEF3BEF4DE15BEF0C
:106980006EE97BEF87ED9BEFBFCF02E31BEF2CEDB2
:106990003BEF47E15BEF6CE27BEF8EE09BEFB4CF28
:1069A00002E31BEF2CE73BEF41E85BEF64E87BEF92
:1069B00087E89BEF0E94581780912D420E94C517CF
:1069C00087E00E94691A0E945931A0CF02E31BEFB1
:1069D00023EC3BEFA90165E47BEF8AE49BEF0E9487
:1069E000581780911A420E94C51790CF02E31BEFFF
:1069F00026E13CEF40E15CEF62EE7BEF85EE9BEF42
:106A00000E945817809128420E94C5178091294200
:106A10008E5FE9CF02E31BEF23EC3BEFA9016EE8A9
:106A20007BEF89E89BEF70CF02E31BEF23EC3BEF9A
:106A3000A901B901C9010E94581734EFA32E32E40D
:106A4000B32E212C44244394322C34E03E8B07E0B7
:106A500010E020E241E0632DCE0101960E942A233E
:106A6000D5018C9190E0002E02C0959587950A94EF
:106A7000E2F720E080FF26E6442D6E89CE010196E4
:106A80000E941117339401501109BE89B05EBE8B6C
:106A90000F3F1007F1F64394F8E02F0E21E0A21A01
:106AA000B1084F12D1CF32CF8114910409F449C0FB
:106AB00081E040E1C416D1040CF480E09601215F2E
:106AC0003F4FA98DBA8D2A173B0708F4826002E375
:106AD0001BEF23EC3BEFA901823061F1833071F1B0
:106AE000B901813049F589E99BEF0E9458172FEFD2
:106AF00040E06CE583E49AEF0E942E1740E2BE016D
:106B00006F5F7F4FC4010E9416242FEF40E064E8BE
:106B1000CE0101960E9411178114910431F0A60153
:106B2000B4018B8D9C8D0E94E13168E081E00E9470
:106B30007416ECCE64E97BEFC901D7CF64E97BEF33
:106B4000D2CF02E31BEF23EC3BEFA901B901F4CF55
:106B500002E31BEF26E73BEF41E75BEF6CE67BEFE1
:106B600087E69BEF0E94581780911942883751F0B1
:106B7000803F21F08C3321F480E035CF82E033CFA9
:106B800083E031CF81E02FCF02E31BEF23EC3BEF1B
:106B9000A90160E47BEF8BE39BEFB6CE02E31BEF32
:106BA00021E63BEF4BE55BEF65E57BEF80E59BEF97
:106BB0000E94581780912C4216CF2FEF40E061E6DB
:106BC0008DEA9AEF0E942E1720E042E061E084EE09
:106BD00098EF0E942E1720E043E061E084E099EFF7
:106BE0000E942E1720E044E061E084E299EF0E94C9
:106BF0002E1720E045E061E084E499EF0E942E1713
:106C00000E9482290E94D2242091417D3091427DB0
:106C1000820F931F969587958093417D9093427D37
:106C2000BE016F5F7F4F0E9491242FEF40E062ED25
:106C3000CE0101960E9411170E94FE24BE016F5FD3
:106C40007F4F815191400E9456242FEF40E062EA2D
:106C5000CE0101960E94111720E046E061E080E835
:106C600099EF0E942E1720E048E061E084E699EF5A
:106C70000E942E1702E31BEF23EC3BEFA901B901A1
:106C80008FEA9BEF41CE20E042E04F0D61E088E0CB
:106C90000E94B0160CE61AEF82E0B82E20E04B2DD1
:106CA00069E0C8010E942E17035F1F4FB394B7E03D
:106CB000BB12F4CF0AE010E0B12CBAE0AB2EE4E056
:106CC000BE1223C080912742BE016F5F7F4F8A9D15
:106CD000C00111240E94912442E04B0D20E06CE69B
:106CE000CE0101960E941117B3940F5F1F4FF5E07C
:106CF000BF12E5CF02E31BEF2FEB3BEF4BEB5BEF5C
:106D000066EB7BEF83EB9BEFFFCDF801E75EFD4B7E
:106D1000808140E3BE016F5F7F4F90E00E941624A8
:106D2000DBCF02E31BEF23EC3BEFA90168EC7BEF29
:106D300089EA9BEFEE2011F083EA9BEF0E9458173F
:106D400028E0E29EC001112426E1289F8001299FAE
:106D5000100D1124065D1F4B412C8E2D880F880FBE
:106D6000880F8150888F4394888D840D0E94F2286B
:106D700020E0442D62E00E94B01618013CE03E8BFA
:106D8000B12CA12C20E0442D6E898CE70E94B01616
:106D9000F10181919191A191B1911F01892B8A2BD0
:106DA0008B2B49F1F801EA0DFB1D808929E0289F12
:106DB000F0011124ED5BF248908126E6911120E06C
:106DC00037E0839FC0011124442D6E89665F885B84
:106DD00097400E942E174FEFA41AB40A5E89545CA4
:106DE0005E8B84E0A816B10469F60A5E1F4F98E036
:106DF0004912B9CF8BCD26E6442D6E89645F80E5BC
:106E00009AEFE7CF02E31BEF23EC3BEFA9016AE027
:106E10007CEF84E09CEF0E94581780912E42E3CDD6
:106E200043EC5BEFA3E4AA2EADE7BA2EF5019A017D
:106E300086A9882311F029EE3BEF39966E167F065E
:106E4000B9F78F2D0F2C000C990B069669E0689FFF
:106E5000F001699FF00D1124ED5BF24881818F3FB5
:106E600039F0808140E45BEF882311F041ED5BEF66
:106E700002E31BEF66EB7BEF83EB9BEF0E9458175F
:106E800020E041E068E085EB9AEF0E942E1720E0B9
:106E900041E06AE885EB9AEF0E942E171FE181E03E
:106EA00020E042E0682F8BE10E94B0161150C1F73C
:106EB00020E042E068E78EE00E94B01620E041E06A
:106EC00068E78CE70E94B0168F2D66E00E941D3E99
:106ED0009D5F988F8795882787958F5F8F8B02E7B7
:106EE00018EF1E8AD501D6968C91412C813011F075
:106EF000F6E64F2EBE89B63088F53B2EE3E03E0E17
:106F0000242D432D6AE0C8010E942E17D501D79683
:106F10008C91242D432D61E48F3FB1F10E94F22822
:106F2000242D432D62E40E94B016282EF50184AD75
:106F30008F5F0E94F2286FE0620D242D432D0E9486
:106F4000B016282ED501DE968C910E94F22860E1C1
:106F5000620D242D432D0E94B0161AC03E88BDEF4D
:106F60003B0E20E0432D68E78CE70E94B016242DED
:106F7000432D6AE8C8010E942E17F50187A98F3FAB
:106F8000C9F4242D432D63EC87E59AEF0E942E1758
:106F900020E0488D6F8988E00E94B016FE89FF5F6F
:106FA000FE8B29E0A20EB11C095F1F4FFC3009F0D7
:106FB00099CFACCC0E94F228242D432D64EC0E9482
:106FC000B016282ED501DC968C918F5F0E94F22896
:106FD0006EE0620D242D432D0E94B016282EF5017F
:106FE00086ADB3CF8091B341857029F48091B241D1
:106FF000882309F492CC0E94CB29182F0E94E533F4
:10700000813009F41FEF0E94E72831E1351508F1BE
:10701000E52DF0E0E25FF74C0C94753E20384B38DC
:107020006738E0381B3A383AB9389138ED399D382D
:10703000A138853A413AA13A043A76382938923A49
:10704000103109F450C300F5112339F0183009F458
:1070500063C2133011F0173081F50E9420166BE0E7
:1070600080E00E94741681E0809313400E94932B6D
:107070000E94361A87E00E94691A62E087E00E9447
:1070800074160E94593160CC183109F429C31032AA
:1070900001F711E09BC01031C1F048F4112309F44D
:1070A00095C083E01830A9F680932D4206C01831B0
:1070B00051F0103271F610922D428091B3418570DB
:1070C00009F4E4CBCACF81E0EFCF82E0EDCF1831F5
:1070D00049F0103221F01111BCCF1EE077C01092A0
:1070E0001A42EBCF81E080931A42E7CF1031B1F022
:1070F00048F4112391F3183009F0ABCF81E080936D
:107100002942DBCF183131F0103209F0A2CF1092B2
:107110002842D3CF81E080932842CFCF10922942DA
:10712000CCCF183139F0103209F4E6C2111191CFE9
:10713000512CC3CFEAE05E2EC0CF183171F010326F
:1071400021F0111186CF17E041C040E1C41AD108E7
:10715000D7FEB3CFD12CC12CB0CFC6010F96A98DCD
:10716000BA8D8A179B0708F0A8CFB0E1CB0ED11CCF
:10717000A4CF1031C9F048F41123F9F01830B1F060
:10718000809119428093347D64CF183159F08CE39B
:107190001032B1F7809319428091EF42877F80933C
:1071A000EF42EECF88E7F6CF80EFF4CF8FEF8093FA
:1071B00019428091EF428860F2CF7EE0572EE0CFF7
:1071C000183149F0103221F0111143CF512E75CFF3
:1071D0000E94013372CF20E044E062E08FE59AEF35
:1071E0000E942E1761E084E00E94741685E0E9E0B9
:1071F000F0E4DE01519601900D928A95E1F710922C
:1072000060090E94BD320E94E5138AE00E94CC13FF
:107210008EED9AEF0E9475220E941C2257E0652E87
:107220007E01E1E1EE0EF11C60E3762E10E080912C
:10723000086A882361F00E94AE13F701E10FF11D87
:107240009081891719F0123008F073C01F5F0E94F7
:10725000CB298F3F11F4143051F70E94AE138A30BE
:1072600009F069C0DD24D394798A7A8A7B8A00E0A8
:1072700010E08091086A882369F00E94AE13082FFD
:1072800080ED800F8A3008F076C0F701E10FF11D24
:1072900000831F5F0E94CB298F3F31F4003249F7F2
:1072A000F3E0DF1609F494C0012F10E05701A00E9F
:1072B000B11ED12CC12C8501AE14BF0409F070C0E1
:1072C000B0E1CB16D10418F0E0E3CE1AD1086C9CE3
:1072D00080016D9C100D11240F5C1D4B94E0B92EA4
:1072E00085E0C82ED12C0E94FA21A82EA29420EF6E
:1072F000A2220E94FA21F601E45AFF4FE00FF11F8B
:107300008A298083F1E0CF1AD1082EEFC2162FEF21
:10731000D20649F7BA94095F1F4FB110E1CF0E941E
:10732000AE138A3009F49ECF0E94CB298F3FB9F368
:1073300099CF10E08CCF0E94CB298F3F09F48DCFDD
:1073400082E09BEF0E9475220E94E5130E94AE0F1F
:1073500083EF9AEF0E9475220E94B2320E9420169B
:107360006BE080E00E94741681E08093134083E01C
:107370000E94A329E9CA8FE9800F863008F485CFDF
:107380008FEB800F863038F4F701E10FF11D80E2BA
:10739000800F80837ECF0A3309F07CCFD52C7ACF43
:1073A000D5018E914D010E94162290E098012A1974
:1073B0003B09220F331F220F331F02C0880F991F72
:1073C0002A95E2F7C82AD92A540176CF0E94AE1333
:1073D0008091086A8111FACFB9CF103109F486C1C2
:1073E00048F4112309F4A4CE183009F032CEB1E1EB
:1073F0005B2E63CE183121F0103209F46ECE29CE07
:10740000E12C1BE0512E59CE103109F472C148F421
:10741000112309F481C0183009F01BCEFFE05F2E64
:107420004CCE183129F0103209F013CE12E0CECE36
:10743000A6E05A2E42CE1031B1F050F41123A9F03B
:1074400083E0183069F080912C420E94723201CEA4
:10745000183129F01032B9F710922C42F4CF81E0A4
:1074600080932C42F0CF82E0FBCFEEE05E2EEBCF9C
:10747000112309F451C0103209F0EBCDF12C1CE0BE
:10748000A5CE103171F1D8F4112309F439C11830A7
:1074900009F0DFCD8F2D0F2C000C990BFC01ED5D59
:1074A000FD4B208121502083209127422F3108F469
:1074B00004CE8E5D9D4B2EE1FC012083FECD183164
:1074C00049F0103209F0C5CDFA94F7FEF6CD94E0FC
:1074D000F92EF3CDF39434E03F150CF0EECDF12C02
:1074E000ECCD8F2D0F2C000C990BFC01ED5DFD4BAD
:1074F00020812F5F2083209127422F3108F4DDCD9A
:107500008E5D9D4BDC011C92D8CD183109F4FAC078
:10751000103229F011119DCD88E0582ECECD81E09A
:10752000E826CBCD183149F0103221F0111191CD60
:1075300018E04CCE10922E42C0CD81E080932E42B6
:10754000BCCD103109F46EC078F4112309F4DDC00C
:10755000E3E4FDE7183009F07CCD16AA3996BDE7C3
:10756000EF3AFB07D1F7A9CD1831C1F1103209F07C
:1075700070CDFA94F7FE02C07BE0F72E8F2D0F2C12
:10758000000C990B019710F48BE090E049E02F2D4F
:107590000F2C000C330B2A5F3F4F429FD001439FBB
:1075A000B00D1124AD5BB2489C012A5F3F4F429F52
:1075B000F001439FF00D1124ED5BF24818963C91C9
:1075C000208532137ACD019797FF02C08BE090E0BF
:1075D000FA94F7FEDCCF6BE0F62ED9CF8F2D0F2C6F
:1075E000000C990B069629E0289FF001299FF00DC9
:1075F0001124ED5BF248208539E0F3944BE04F1500
:107600000CF4F12C8F2D0F2C000C990B0696389F43
:10761000F001399FF00D1124ED5BF248808582174F
:1076200061F34BCD8F2D0F2C000C990B069629E0A2
:10763000289FF001299FF00D1124ED5BF248408551
:107640002081211139C003E41DE7F80186AD8413C0
:1076500020C083E49DE7DC01DE965C91DE97541741
:10766000A1F037A9D7962C9132130FC023E43DE740
:10767000D901DE966C91DE97561302C0D6961C9205
:10768000275F3F4F6216730699F7099668167906C9
:1076900011F739966E167F06C9F681E0D801DE969D
:1076A0009C91DE97941302C0D6968C93075F1F4F70
:1076B000E017F10799F701CDE3E4FDE726AD2413C8
:1076C00001C016AA39966E167F06C1F729E0289FD9
:1076D000F001299FF00D1124ED5BF2481082EDCCF2
:1076E00057E0552EEACC43E0542EE7CC35E0532E3C
:1076F000E4CC24E0522EE1CCD12CC12C19E066CD93
:1077000015E064CDF12C1DE061CDE12CF12C1BE0E6
:107710005DCD1F93CF93DF9382E080932C428091C5
:107720002C420E94723280917C008E7F98ED94BF33
:1077300080937C008091630083FDFCCF90917C005E
:1077400088ED9B7F84BF90937C0090917C00926039
:1077500084BF90937C0090917C00916084BF909353
:107760007C00809141018111FCCF82E08093470130
:1077700014E01093400110924601C1E0C093520101
:1077800081E680935001C0930A0A1092010A809109
:10779000090A8E7F8093090A86E08093000A80910F
:1077A000000A81608093000ADFEFD093010480E833
:1077B000809304040E94AE15D09362048DE0809300
:1077C0006B04D0936C04DFB910930106109200068D
:1077D0000E94E72887E380931E428BE380931D423B
:1077E00010921C428CE080932A42D5E0D093224232
:1077F00083E08093214285EE97E080931F4290932F
:107800002042409122426091214280911F429091FA
:1078100020420E94201980932B42C0931340C093B2
:107820002D4210922E421092CE69C0931B421092AC
:107830001A4288E78093194284E6809323428CE1C0
:10784000809324428CE380932542D093264288E1A2
:1078500080932742C0932842C09329420E94D22499
:107860008093417D9093427D809119428093347D35
:107870007894DF91CF911F9108950E94893B84E60F
:1078800090E00E94C22F0E94F22F0E94201661E019
:107890008AE00E9474160E94932B0E9459310E9424
:1078A000A2200E94E7280E94E5130E94AE0F0E94CA
:1078B000E32080EAF82E92E0E92EDD24D394D1E093
:1078C00018E0CFEF2EEFC22E0DE030E8B32E8091FE
:1078D0001140813009F423C108F48CC08230B9F71B
:1078E0001092E57D1092347DEAE2F0E4148A7696F7
:1078F00081E4EA38F807D1F710936B04C0936C0465
:10790000CFB980912842813071F40E9400186BE059
:1079100080E00E94741690912942990F990F80E09F
:107920009C5F0E94C22F0E9420166BE080E00E94A4
:1079300074160E94E8180E94E728D0920004C092B2
:1079400004048AE090E00E94233010936B04C093FB
:107950006C0400937704CFB980915000897F8460D4
:1079600080935000809150008160809350008895F2
:10797000809150008E7F8093500080911140823022
:1079800059F30E94EB18C09300040E94EB18B092C8
:1079900004040E94F83082E390E00E94C22F7399A1
:1079A00006C00E94E5130E94AE0F0E94E320809162
:1079B000B241813009F4AEC0D093E57D10927A4295
:1079C00010927B421092F569D093CF691092CD69E5
:1079D000D093317D0E94361A0E94A3190E9459311A
:1079E000D09313400E94932BCFB900936B04C093A4
:1079F0006C046DCF8091234290E080931940909366
:107A00001A4080911240813021F080910240811112
:107A10004AC08091CD69811116C00E94CB298F3F49
:107A200091F0E82FF0E0E053FD4FE491E093304215
:107A3000D093A241D093CD698091254290E080936C
:107A4000327D9093337D0E94202C809102408130C2
:107A500061F48091034090910440009709F457C06D
:107A600001978093034090930440809105408130BA
:107A700079F4809124422091194030911A40820F6C
:107A8000932F911D8093194090931A4010920540B6
:107A90008091194090911A400197809319409093DA
:107AA0001A40109212408091194090911A40892BEF
:107AB00009F0A7CF809106408823B9F020912C7D52
:107AC00030912D7D80910040909101402817390719
:107AD00051F00E94A31980912C7D90912D7D80936F
:107AE0000040909301401092064080910740882307
:107AF00059F00E94361A87E00E94691A62E087E016
:107B00000E947416109207400E94932BE0CE1092B0
:107B10000240ABCF82E390E00E94C22F48CF109288
:107B20000240EAE2F0E4148A769681E4EA38F80743
:107B3000D1F780912C7D81FD4AC00E9459310E946D
:107B4000361A87E00E94691A62E087E00E94741684
:107B500067E08BE00E94E022F092020480915000E6
:107B6000897F846080935000809150008160809371
:107B700050008895809150008E7F809350000E9425
:107B8000932B8091347D811105C08091EF4283FF5A
:107B9000E09211408091B2418130A1F410921140E5
:107BA000E091AE41F0E0EB55FE4B8081833041F433
:107BB0000E94CB290E94E533811102C00E940A3441
:107BC0000E94A31980911140813041F280CE8091B2
:107BD0002E42882309F4B1CF81E00E94C02983326C
:107BE000B9F482E00E94C029823291F480E00E94C0
:107BF000C0298D3109F4A1CF80E00E94C0298531D0
:107C000009F49BCF80E00E94C0298D3009F495CF04
:107C100080E00E94C029823209F49ACF0E94BF2ED0
:107C200097CF991B79E004C0991F961708F0961B0F
:107C3000881F7A95C9F78095089587FB082E062638
:107C400087FD819567FD61950E94113E0EF4919527
:107C500007FC81950895AA1BBB1B51E107C0AA1F11
:107C6000BB1FA617B70710F0A61BB70B881F991FDD
:107C70005A95A9F780959095BC01CD01089597FB81
:107C8000072E16F4009407D077FD09D00E942B3EF2
:107C900007FC05D03EF4909581959F4F089570950F
:107CA00061957F4F0895A1E21A2EAA1BBB1BFD010F
:107CB0000DC0AA1FBB1FEE1FFF1FA217B307E407CB
:107CC000F50720F0A21BB30BE40BF50B661F771F23
:107CD000881F991F1A9469F7609570958095909503
:107CE0009B01AC01BD01CF010895EE0FFF1F0024E1
:107CF000001C0BBE0790F691E02D0994A29FB001E5
:107D0000B39FC001A39F700D811D1124911DB29FCF
:107D1000700D811D1124911D08950E947E3EB7FFB4
:107D20000895821B930B08950E947E3EA59F900D9F
:107D3000B49F900DA49F800D911D11240895DF9391
:107D4000CF931F930F939A9DF02D219FF00D8B9D44
:107D5000F00D8A9DE02DF10D039FF00D029FE00DC7
:107D6000F11D4E9DE00DF11D5E9DF00D4F9DF00D3E
:107D70007F936F93BF92AF925F934F93D5010E9411
:107D80007E3E8B01AC01D7010E947E3EEB01E80FE5
:107D9000F91FD6010E94EE3E2F913F91D6010E941D
:107DA0007E3EC60FD71FE81FF91FAF91BF910E94FB
:107DB000EE3E2F913F910E947E3EC60FD71FE81FD7
:107DC000F91FD6010E947E3EE60FF71F9801BE0103
:107DD000CF010F911F91CF91DF9108950E947E3EB8
:107DE000460F571FC81FD91F08F43196089568948D
:107DF00001C0E8948F929F92CF93DF930E94053F3A
:107E0000DF91CF919F908F90089588249924F40159
:107E1000E401B0E49F93AA279A158B049C04ED0516
:107E2000FE05CF05D007A10798F4AD2FDC2FCF2F8B
:107E3000FE2FE92D982C892E982F872F762F652FCE
:107E4000542F432F322F2227B85031F7BF9127C02C
:107E50001B2EBF91BB27220F331F441F551F661FC8
:107E6000771F881F991F881C991CEE1FFF1FCC1FAE
:107E7000DD1FAA1FBB1F8A149B04EC05FD05CE0560
:107E8000DF05A007B10748F08A189B08EC09FD0937
:107E9000CE09DF09A00BB10B21601A94E1F62EF494
:107EA0009401AF01BE01CD01000C08952A0D3B1DC8
:107EB0004C1D5D1D6E1D7F1D801F911F0895DC01EF
:107EC00001C06D9341505040E0F70895F894FFCF02
:0E7ED000FF0001C800010101055058343100C7
:108000000106B5064E70F858985684D84C5B8C4BD8
:108010004C3B1C427070384BAE783C0670B958CE61
:108020008CA08D08849B76761908AE58FC58F3997D
:108030009E990AB5960D9E1596BD966262C6CA5067
:108040001C231908AE58FC58E21BE2371100EE5C05
:10805000981C45028CA08411008D08580CA0B5A274
:108060007B9BCBC313E3DB4B43CB3B434B535BBD0E
:10807000B25100E30E1C5016B523110CAE0E93C482
:108080008370FA70A033F0B80E6150F86550C4F0F8
:108090007C30147C3050BCE0C8CCF73008C8CC66CB
:1080A000EBE0D5884FA550F0D44FA550D43FA8F0B1
:1080B000EECBA550AEB87C58AE8CA74C3344983C60
:1080C000A883B5BC84634C6100431300A550EED473
:1080D000D3B87C588C33A3B070E0A550EED433B83D
:1080E0007C588CC378A84E703868F828EEE8B5BC88
:1080F0008860A04E70B85860434C3748ED04711C3E
:10810000EC1F0C1B919CCC9BCCA3203C560630183A
:108110006621463087662F110C1D02C8CC5C5AD0F0
:108120007038CC9704624728707C3014FCE090666D
:10813000281C70381B2E28BC30EB33B898A8E00000
:10814000A383634323387C8338FC6B383C53387CEF
:108150003B387C2338083C8C1BADBC300670FCE0FF
:1081600048711C8C7F0C238914538C2B0441B02341
:10817000F8992C4C3F305166FB610044ED040CC76C
:108180000100D50CCC0F3008999C0CCFB83C580C92
:10819000D91C6000711CEB5924305006CC4F300CB8
:1081A000B19CA6CB091E201CE2153221460100E03D
:1081B000D50CCC3F300A999C0CBBB8F10C7CD80490
:1081C000884484D83C467CA8C46100CC4B30C306AC
:1081D000203C1C6ADB78EE30BF0E66267BA606705C
:1081E00038EE4B3EB75EF0FC56468B300770999CDC
:1081F00051844E7020B8BC588CC50284983CA8E0CD
:108200006D5820091EC8CC6046F070306906787C35
:10821000660FBC6670380EBAF038BA6EB7F04670AA
:10822000B858CCA03846BC30E660C4783C1C420A42
:10823000BD8E60A0587058585870707070E0DCA007
:10824000C44484C44404B1702DD91C610030FF0EB5
:108250004EF0E020F0AE70AEF0A6DB309C3C30A7D4
:108260003C309B685A2E28704E9C103020E84E708F
:108270009C90105C1010A8883006999C3069067894
:108280007CA63C68D5060ECC1F4CA038CC432E28CB
:10829000BC30B606E00C6B90662870387C1C0A1C5B
:1082A0004E70E06228E01908AE581C58F6BDBE4476
:1082B000F64348F62BF6603D02568C33841100B12C
:1082C0000EAE8E301EC63F4CC3301AC6A36E3008A9
:1082D000EE4E702E3C86F313EE66F3EEB8AE3D0222
:1082E000D588387E7E8953065E04467056607CA62B
:1082F0004708FCA627FCA64B3CED08E606E6E6464A
:1083000046FC06E01C8ECECC474C37784C1758E024
:10831000CC8338BC3AEEE2DFCE308E1A3C7E1E4E65
:108320001CAE3A30AEAA3CBECB133CEAF358AE6E5C
:108330001C53CE3A303C46FC6E1A3A3CEA38CA2806
:10834000E044E23349A459A41B49A4E5A43C1E4ED1
:10835000BE4F58E5A4D898D83CBB2550581CDD8C9E
:108360006EB858E065BC8C1BCCA0044841B0336D9E
:10837000BCCE992CF90C8C2F3C580C6765204670AC
:10838000B85888D3C4B83C5804987C58042B492466
:10839000B8587CD804D8FCD88404D87C8498A8E049
:1083A00085BC390C048CBBB85804ED04C4E0B01A89
:1083B00030E61B1C50BCAEC1B0AE4D14DDAC492440
:1083C00065205DBC651C4C752EB85888987C580893
:1083D000983CA81D02B85884987C5804A341B0F971
:1083E0000C3330A7C8CCF91E66DB2DAA8D08F681A8
:1083F0000B1C98B10A30FD70F0B8150A46A809BAEE
:108400008BA3ABDBB3ABA39B93FBA3F3032B23C9DE
:108410001230CFA663B51230903B1D140912309173
:108420000286061D146684E37330D04330CE0663A3
:1084300065169C021D1411B41DB4D884D81B30A835
:108440000629BF30AE06AF19B4D8D91C8C2330E052
:108450001B30D02D149388309C0613841D1411B446
:1084600006D91CA6D88C7384D884E6BD1C090E04DA
:10847000DD14661BD806163066066B1E7E8C177ED2
:10848000A1140CDDAC5D1E307006C7668B307466BF
:10849000D3069B3071463C301A7E3766EB305C4623
:1084A000E80B3065DB307A4636BB30689B301D0602
:1084B000CB3B301A06CF6667B8D8485CA2E2178873
:1084C000D8E88B266637DD1430053B302D23A61CFB
:1084D000D0E51411B46E5606D91C301D1C621F065F
:1084E000970C2B301FE5140912E6161D1411B46EFB
:1084F000060404CC13081C02A65A56BC1AD91CB890
:108500003007E8BAEF6E49241C0C2DB50CE5A46EBB
:1085100006D91CA675B0E9145B6E3DA41DB48E0689
:10852000D91C1C627330CF2D1449246E3DA46EAE4D
:10853000C512AA625830C02D14CCEF8CDBE0B8B85D
:108540003044E86914061ED91CA1143020E8F89CB8
:10855000E213A83060A820045330C848C8CCA066F5
:10856000E34404048449242DA806864C2BAD7043B3
:1085700093C1B01EA114C66FCC4F6914061ED91C3E
:10858000A11409123020E84924B80E41A41DB41CDE
:10859000EAE38E56063C3040FCE0BD1C2012050785
:1085A000204924785A0E43660E7038EE477A30C060
:1085B000661BAEA3AE3CE03020E80C57302006F836
:1085C000A85666A00879B2D91CA6063C30147C30A7
:1085D0001C50BC087A3056D84C1B36448C1B048483
:1085E000D8E80C8F3020E8E09E4EA0A60E3C266610
:1085F000EEEEEEEEE6A63C266606BEEEEEEEEE06ED
:10860000AEFC2E6E0E60DE77DC101E7CFE7FFCBEA4
:10861000FE5FFCBE437E9EBE1F3CEB7E3C1A9EFC72
:108620009CBE603003FCE8D34670CEED28041413E2
:1086300008AE58FECD7DE05CE0D460D0DC6202D7AD
:10864000629362E97CE0C2E223302C1B302ED4A07E
:10865000D57C33E97CE0D414030CA01C98E217D439
:10866000A03045D57C98F6CD7D7B1C38BC44137A70
:108670003076EF76DF7617483C0AE0CC1BAA7339D8
:1086800088E60952D5883ED74DA6251CD91C302036
:10869000E81538004C73B0E22F302DE813B8957C04
:1086A000D91C7B30C30E203C0A2365202B4E203C76
:1086B000D026E806303404661708B0C606C61CD0BB
:1086C0000C1BE21722E866F13A0E30410660304B8F
:1086D00006F3302506FCE61C0A301E6A23666A375C
:1086E000FC0E66813A30CD6A2F3C3E3EA366E030F8
:1086F000610660306606A0301ADBB03C0E660401ED
:10870000AC0C0F1CE22F0E16913E70012053AED818
:108710000C27B0B13E088BC1B0B1BC492444B0A114
:108720001CF93E589DBC981C1D88FC1EBEBEDDA4D5
:108730004E70E5A4D8B0D83CBEC32550704670B08A
:1087400068301E7CA11C0441EEB83CD844D8FCA87B
:10875000D91C78D884D8F04926410CA83080A6E6E8
:108760004EF070B858CC1F0C1B66664C17168C1355
:108770006E3C588C233080464C2F8C23767676BC0A
:10878000588C2B76767676BC56EE3C56EEEE4E3016
:10879000107030FDF0AEF046F070B858E07CD80CA8
:1087A000DD2F580C2B30844D320CDF890C4C3304F8
:1087B000B170434BF8E61F26E865144C19387DBCB0
:1087C000651CC8F84666E8B858F6F62B9DBC410C07
:1087D00004B898A859248C47C1B0302EA84924C1A8
:1087E000024E28E8A89868E0FC5C0AB8AAA8E0B0A5
:1087F00030E83AF6E3E030107030FDF0E0000000C1
:108800005AEEEEFCC6E6E6C63C06BC5CEA5A505C94
:1088100030662B22E399C63AC60E3006C3A6E67A26
:108820005ABC1A30F6F63C58FC0E3C3A301C0A3C56
:108830005AB03AE07AF30438BC585C98FE9526FCAE
:1088400010D0900EEE7E93EE0C31237EDBEE7EA3F5
:10885000FE13081C78221BDCEB1465238C27787E22
:108860006881228CAF88DB780EDC901E6F080CC705
:108870004E6E56DC5050087B0C5F0C1F0CE30C1F37
:1088800008330423780E561C561750DB7E63EE7EA9
:108890004B9C78221BDCEB9443E030D066FB20E05D
:1088A000D400980278A26838BC983C28E01CAE58E6
:1088B0000813044E6E56DC90688DB8B8580C2BC95E
:1088C0008C89B68CB551884EE80CDDB641A48A4936
:1088D00024DD20792419B46A1C0A301D623F0A2B5A
:1088E000AE9C58636E1DA4DD8CC1026E601CCB383B
:1088F000BC58780ED91CE9501C622B62BEDCDBA28E
:108900000C471437D4A250DCDC8C5BBE1FDCEB8C34
:108910001BD013D0DC4C9BD47F1EBE2F5467DCDBF6
:108920008C1BD013D0DC9BBE131EBE5EDC0C135020
:10893000BEE0DCA0760C831C6247A29C622FA222C0
:10894000230AA2501CE0169CE0D2D268AED2D228F4
:108950004EA846F070E0D91C78D808D8F0AB781C47
:10896000221BDCEB6206569C622BC6DC14DBA05695
:1089700013860EDC50BEDE774277FABEE3A6426F66
:108980007E07A6FAD31EBBBE2766EBE31E0C13BE02
:10899000AE0C83A550E854670CAD2355BC410C1DAB
:1089A000024EE860E078E05CA01E0C1B9C131C22C9
:1089B0002B62BEDCDB0C83144742F21F0404D00B95
:1089C0007676130456DBD45F8C2F543F3E63BE5340
:1089D0008483B8580C2B410CFD8A4EE8203077E098
:1089E000689D2244781CEA31B60EB8AAAE3C68F8FD
:1089F000AAAE3CA838AAAE3CE8387C4AFC2878FEEF
:108A00003B09B8B8D84C578C47D8DE3EFE31B8F396
:108A10004484D8063020665746F07038566637D9F9
:108A20001CA6E853D91C230841B0CE6DB81902B872
:108A30003C5806F804A0965C1427D4B6E30EF62B37
:108A40008C63DC541F66E333D4144FA6E32E8A3ABA
:108A50005B0E0A061C2A4F0E7E8E9C0ABA60E0AEA0
:108A600056E346A38C431B66239A3A370C1F4E737A
:108A700084762B0C4B069CA206BF1BEE608DB8CEF5
:108A800008D528EEE9502E0EA0B8BCEE7EE6C6FE54
:108A90001BDC508C752A5CF65B752C552CD4DABE29
:108AA00026E37B661FD4EB46BE3F752C552CD414B1
:108AB00047BEE3D4141FA2E39CE04C437E9EBE4716
:108AC000DCD4E3DCA07E83A28C1BD013D0DCA26BB1
:108AD000552C4C752DF3BEB6AE60EE5D1E5C4C930E
:108AE000063003562FC6FB462746FBC68606A6372A
:108AF000D4BEE31ED3752CD4143FBEE3A2D414EB32
:108B0000D61B1C501CA63033A6E00D2AC6A6C6A64E
:108B1000F306F6C70BE0DC201FD4EBA0E0A28C1B11
:108B2000D013D0DCA2E0A01E7E7E43ED28D91CEE3F
:108B30002526DC10FEE0DCD0D07C70D91CB07C7027
:108B4000061C4AD36A2775B0AB3020DE7E2320494D
:108B500026E8D309CA008CB3F12E461AAEBCFA1A25
:108B60003A30E63A303CC61C3CA2BC02F6F6DE6B5C
:108B7000F6277CD90E7CAE0819BCF90EF6CF75CA63
:108B8000AE5851000E389C0A983CBEAE2838FC26E0
:108B900084E6C67C287E7E677E01CBCDC63000EEA3
:108BA000CC4371CC66250E22C8EE66A30B000000F4
:108BB00000000000E55CBB6100A3E55C8838FC6652
:108BC000E6876B1CC4E666664B095010841CEE01F8
:108BD0003041A478901C8C476A550E4DA43DA49D4D
:108BE000A48C1F7CAAB18CC1B0041D1425FEA55015
:108BF000EED44B4670B87C588CED02B070EEF0E0CD
:108C00004EE8286AB3B83C58A020BC30C1FC1CE038
:108C100000105B504B903BF3D023BD8E103C064CB4
:108C200023308006708C83AE1CE2EEEEEEFC5C50CE
:108C3000303CE6E60E9CF83C5842A65844D91C301D
:108C40002006861CB86AF3AA6A37C6E8A8B8D3F823
:108C50007E60BEB03AE006B8588C233055737C581D
:108C60004C3305BCEEE91BB8580CDFB05A3C06305B
:108C7000667E679CD0FE431CD03EFE53FE470658DE
:108C80000ECD90EE87B00EB85830505E7C067C302A
:108C900076B1B5BCEEB85CCA46A80C2BE21B1C2210
:108CA0009C5858CEBC30147C301C50BC5870305985
:108CB000E2B858E0D8A686251CC1B030E02D1404D7
:108CC0001D1030E09C58BC0E66483D3A44251C1DE2
:108CD0003C984D14987A30F6453AF6F6167A3016E6
:108CE0003C5804D89CA298A2580C9321382B4C5184
:108CF000370C33BD386520A30CB5374CC9370CB7DA
:108D00008CCD378C8F5E7B3091AEFC9C425D1CAE6F
:108D10004D32C1B0711C9DBC110C1D028C1B0CB3DB
:108D20001538838C6B4CF53B0CF53B4CC9376520F3
:108D3000838C653BD32D38DB4C41370C3381346554
:108D400020A3203C0A30836A7F3031E82D383B0C69
:108D500081356520C3B8FB0C3B8C678C1B4924060E
:108D6000A6A6B8A6A803B8F8E806A6F13B4924B819
:108D70003C0E8CA730CD8C2FD91CD532AAAEBCA806
:108D80009858889858653A4C5330AEAAAEBCA80C97
:108D9000571B301E0C0B668CF39C98D844D8581C7B
:108DA0003001AAAEBCA8C1B030D02D14A83060E804
:108DB000D53649249C98D848D858D91CBD1C090ED2
:108DC000042021386B4C778C5F0C1BBD3865209BD1
:108DD0003030E81B30305E172EE83CBEFCE8953A98
:108DE000BEFCD056E82138430C1BBD386520BBB80B
:108DF000E04936BD1C1314201538BB3020A8A8A8A4
:108E00006D7CDC100E304C66CF21B0DDAC49249C6B
:108E10009858B81CD04C1B1CD0AE7CA2813A65205F
:108E20009B3057BE5E2B2666DF03305466E3834ECD
:108E3000BEFC1CD0E81538630C276520CB4EBEFC69
:108E4000D0E81BB8E0301F43301F23301FE8E8E8AC
:108E5000DDAC4924F81C98E8B83C58880898FC6DAB
:108E60001C61001106DCD01C0EB87E584CE706F8D9
:108E7000425646BE47A6E606E6E646A39C98584CF0
:108E80002330804686DDAC4924B80E8CA76686E682
:108E900083DDAC4924B80E30C8E0C8CC3B66E32083
:108EA0001938436D00C1B020492495BC110C9C9821
:108EB000D84C3B4C1FAEBCD1A6D84E5CD070AEBCDB
:108EC000FE6D076645023040E6C8CC6D0266DB04E5
:108ED000B1703C30E866FB59364924A5BCB8D88847
:108EE000D8A84E68D91C1538734CD13E957CB35D1B
:108EF0001C8498A84936492478EEAB7C4A68251C26
:108F0000D91CB81B0CCB6520E36D7C06251CB6BBB9
:108F10001C307F6A93303A6A73302E6A53302C6A61
:108F20003378EA1FAA0A3C68EED91C21B0B30000CE
:108F30000000000049248C931C78EE4B255068B843
:108F40005884986D1CB83C06300F6A291A86D91CC3
:108F5000DDAC492478E0DCA01CF2251866301E1C2C
:108F60006ACF78581598EE8FB858F83C9C580C5F2B
:108F7000B80E95BC110C810A4C37587C7048840C93
:108F80002B88B0A11C44B8D80C23584898589C583A
:108F90004C4B1D3C4924980E1DBCB80E86813A8C62
:108FA000537C560EB858AE444D32587CA11CB8586C
:108FB0001C98BC580C5B30E61BD03B3A30E617E0FF
:108FC0009010589C583532F8E6C1B04CA066664CFB
:108FD00013061EA1143020E8E060B0303360B030DA
:108FE0003A70EEEEDADADAEEEE7CE041A4584DA407
:108FF000EDA4D8E05CF84A0EBEBE175031020E8CCC
:109000002248E30130028C043EAEC242880480BE96
:10901000202C51C0202ECC0DA241A9AA84F902C453
:1090200050020D3384537FBC3F00000004DC78778E
:1090300077A50400DC4E0DC0AD804070097E441061
:10904000226323144F8CCCC30DC912942379D33FD0
:109050000030004100E45C480640200180840B3071
:109060003417E33B03614413D323C1903331FAF443
:10907000E4D2CA44F24DD4908823743880DFCFB351
:10908000F3BC6C759792E288CFD3CE4060C1562175
:109090001E168C74E8237655D4B87088323931D5D1
:1090A000D193F0E04D472E1FB82F2C89617420C258
:1090B00040844410A0363513834E847F64D84E55C7
:1090C000E88080D274124C1BE360A307800F28CC89
:1090D0001B31841C91DC3E01FC279EC001316D8256
:1090E0000FEEFF13DFCFFBFC27D90F9E1BC43013FD
:1090F00072813CF7F73CF743182F2EE388A4033C1A
:10910000000010D544483012D070C5713003B0173C
:10911000470C3C12C470CC030D8BCF8002470C4D22
:10912000F348CCC44C7888871F871EC715335F84EB
:109130008F2341C0084013CF4688CC00253840CD4E
:109140007512080A0D21334073C4044383C700F825
:10915000B1C44CFC72FC85BFDB87C4040C232031F6
:1091600023715CC00E193400C6848914C3703CD1CD
:10917000F3CF90E150CE6192DFF120A955A34A15BB
:10918000A82A166262403C8777F8480491C33833B6
:10919000C3400431F3B0F7C9C4E4C88DBBCB34700D
:1091A00038E013130741C43C7324232378D1C43D12
:1091B000215E141F13CAC53884C4AC737C7CC8B547
:1091C0001012024080D844C84417612520B33D20C6
:1091D000C623FCECD36EC8C1EC0B5420F944001537
:1091E0004F1534551823FBF73284FC4C018B8773E1
:1091F000E1F81727FF0113C760D19278AF17C603B4
:1092000094D754508F8FF450E4E5A41F659A3D8A9B
:109210006BDFCB3C02CA23A3CA8DC94D8842132001
:10922000668633F3ACFC18FE43A28D0B11A2CA83F1
:109230004813144140001733CC0C0CB26D33847DBD
:1092400003C74F3CC48314F3303D14CA20CED191E0
:1092500010CC3F3CC03EFD2EF2C6F1EE98127337A3
:10926000D673F4480C30CDC980CB3483D88F2072AC
:10927000CA2033DEF32003C48A6D1458608219A813
:10928000C5878C047931ACCCF07340CC1EC97667AD
:10929000F2355B43440B1D38CF7ED0C162733F0A69
:1092A00001630E80B8B3007C8E3C05B0F4D203108D
:1092B000BB0030CD0058885CC574351A37C3D2ED79
:1092C000E2D03010A2633C03F10C4D0CE1E8CF304A
:1092D000FD1107723C7012948ECB9025A18C23094E
:1092E0001C480F8A036AC214130FE30300A3388BD0
:1092F0002AA04C03C431CF0C0CC02C0200DE0AE2C1
:1093000038FC494000C0001D841057195F3DC44E11
:10931000C47FC3FF5DD64BD524CE0358C8CA19629B
:1093200081D117FB420808B2338443F5FC414CCC91
:10933000125328C634B952B9CE0350C400C846F2FD
:10934000CE7FE00932713233F100402233870C8C3A
:109350002CC5C40123EF0B0725F653843401339049
:10936000CC4C04E415AFCECC013931C710733303B4
:10937000188101C831313E1E080700F2C38071FC1C
:1093800063C5C8C4AC85332246E31F3B380720833E
:10939000DC0741FC13C33F6F88F8DDCC5050D57318
:1093A000444C18C04C58F8F883CC7132C3C10C0738
:1093B0000692BD78413BC4BD8F1304B3F810FA1870
:1093C000F3274ED1C7C7C7C7EBA48C080081ABE316
:1093D0007B48B13013223AC467233F437632168864
:1093E000C0F0303F32516308408F12F357B0804BCA
:1093F000F0CC0CD3C0C4DBD8567F5D34F2430503F8
:1094000041460000020103044247000027242120B6
:109410004348000028252200444900002926230053
:109420004540000F800000981E19B0456C63AB13D7
:109430000D08B0C964F0B8C9640EB01D6088C96475
:10944000CBAD130D08B0BEF053ABB063840F0DB0BD
:1094500071643BADB0BE001D606902AAB03560D337
:10946000A5A6A6B035603102B21E18B00EBBAFB0D3
:1094700061603B930201B05EE0930F030151848869
:1094800008080176008435928C031201595A860827
:109490001301215E8E0913015184338E1301A99E9D
:1094A0008F141301715E8E0114015184AB9705096D
:1094B0001601910E008883900505023007455A94E5
:1094C000130200418A940103012E8603355A810C50
:1094D000034E68A8E828E08F141398F0E0840C038A
:1094E000410C511E900C03318A87120C0308CD5E8B
:1094F000CE0C03C15294130C034E2868A82B980C71
:10950000034EE8090299100F039586922D04B005C9
:1095100066870504715E84011207995E84011289D1
:109520005E8C0504A18A0000BD8A8513047D5684E3
:109530000E05870E0548015A9E1205140E05B550FA
:10954000B8E81102981E05B0296A96040175BCE0BE
:1095500094030106B0B162BF0306AEAEAE2BB12DCF
:10956000181E0548B0296A833F030635586B9809D1
:109570000688015A940E098823831206B0ED66BF4F
:109580001306155A833F13063558C30065A68F147A
:10959000079208B0C966930D0888CB8713098481A8
:1095A000568C020C8E0CB0156E870F0C88CB96056E
:1095B000041341743B8E01050DF9709502902D1234
:1095C00051842574BB86060FE03009999C1508610B
:1095D000004106982F31B02D62922D105184080859
:1095E000D578CB8B0301100182880325BEBEBEB0A7
:1095F0001D606666B869603102851310CC2308EDE2
:1096000004B10E94100D0F1210810E842D12B03182
:1096100066900F1413A50E0000751E982B310E0CCA
:10962000B0CD6E981413010C38EE238C03128CB558
:10963000514E70EEE8B902930803B0FA1BBEE8B3CE
:109640008910A06964EE3A460BBE3C1898F01B8E58
:109650000412F552840E12BD2A8E14120D9E9E1213
:109660009552890313015A8613295AAB4E2172ADC4
:109670004E88DB8705124E655A930F0351846B8E1B
:1096800001145184438E091351848808E17A851AA4
:109690000913555E94121113B0F9629413130081EB
:1096A0008A8E0F4552AA14134950356043AB1413E8
:1096B00049501D60B92EAD141398A0BE589BAF142D
:1096C00013495061607B981E3031E16E850E0F1496
:1096D000795A97050916BD0EBF304D18455ABF1966
:1096E0004D18A55ABF303C18E956BF303D3C1825EF
:1096F0005ABF193D3C18055A993E3C18F8AEB8E8D7
:10970000AEA8B902BF193C18BD56BF303D18195A52
:10971000BF193D18515ABF303E18C556BF193E18E3
:10972000E156001D92910518830504482394030F08
:10973000B0E57E8E070913D13E8E0F0188ED0471CE
:109740001E86060F0184BB00009D7CAB0000201C20
:10975000E2E2E283B87CD84C1F481344D83C98A876
:109760004451064DBCE27F410C8C3B8498A8448553
:1097700006880CCB53410C04840C1F08830498A862
:1097800009B8634EE6BCAEB90C004A545C6FD6CA49
:10979000767D4D453C8C92989EA4AAB2BBC2C8CCA3
:1097A0003AD1E0E7EDF3F901097C0E2B14242D32B8
:1097B000353E4763545A6B717C82881A91993245C1
:1097C00093779E28A4A620ACB94F30C8A3DCE761EC
:1097D000EC4209FC600EC01F2E52575CB265696DE9
:1097E0007177883792989EB0B9A8C1DA1582D0D621
:1097F0000EDCE8EF1A14E208F6204CFC286B2A0075
:10980000C88C2409E71892C29EA3E7274DE0489E22
:10981000ECB83C5808987CA8E04E70F8E085B5E0BC
:10982000FFA0B0BE001D6070E0FA174EA05CF6A06D
:109830006636761B26E0F61B4E2B4A6A56D4D4E0D9
:109840004A545C6F0820F66D7132454F61ECDCC004
:10985000A66B982A3A47ACCA63887C82987DAA2B6B
:10986000D67654DC1A20E80E777C0E0E999357308A
:10987000F3FC42F96052280114E237EFB9B2B2E0CA
:10988000141F1A3E155CBBD192FCED453CC8094D36
:109890002EDAB0B9A8C19E2DD677A48C716535D0CB
:1098A000E7FDBCEEC10295BE69CC886B825A23F0FD
:1098B0009D585C0EAEF0AE6E70D494CBE0A55043D4
:1098C00032EC4E70783C0602E01CEA603CEB4CA4A3
:1098D00091EE6E98AE6150AEA0FEA03E337EE000E9
:1098E0002800D58818B550B902B550B5504E70381B
:1098F000AE7828B868F8A8AEE8E0A04E6E60EEE05A
:1099000047710E834140424348700E0078464567D8
:109910006075E00017141110534C0F00A8869C725C
:109920005259911C1815121A515CCF96A94E9D766A
:10993000565A901B19161305575DD085AC4F9E984B
:10994000505B08000C0C0C00555E07770C0C0C00EB
:1099500041460E4E5155593A617E0E5E2D2B2A2FEF
:1099600042474B0052565A2062257F00373431302F
:1099700043484C4F53573D2C631D9A0D3835322EBA
:1099800044494D5054583F05643C9B243936337E3E
:10999000454A08000C0C0C00653E07870C0C0C882F
:1099A000EE61501BDA26F6EF1D64989417D44AFA3C
:1099B000EE58AE0EF09C4A5CEA271C505C0E0A4A38
:1099C000EEEEEE5C262666421FFA06E247FC4626CD
:1099D000E21FFC468C13BE70981D60580E38A60618
:1099E000DA661FFAE7461AB160F08898AE8C5385A4
:1099F00050A0B0EED33E1BBB85508C97A0B03E7BF1
:109A0000CB8550EEAB630EB07BF8615070B0EE5377
:109A1000630EB0CBB8AEF86EB7CC6F4E70B8D84C02
:109A20003FD88C27AD7062C102B8AEF86E6760CCCB
:109A30004341A4E5A8BD8C834E70B8D84CA7D88C00
:109A40003FAD70641BCEB0EE8F2BEE702BCEAE0010
:109A5000B0A8AE58711C98AEE0B0A558B0AE4E702C
:109A600078BC46063C68E078BCAE300560061972EA
:109A7000EE38A02E6EFE433E2F385E3E537EF61B20
:109A800056765CE2174E60EE0EF0386E334C810B6A
:109A9000C90ACEF0AEE0CE7EFEBBA118CC60B858AD
:109AA0004C608CA00841B0B83C58084898FCA8E02D
:109AB00046705CA0D4D4542FCE58E09CD251B5A3AC
:109AC000983C98FC58B83CD88C132E0C1B2E2EBCFE
:109AD000F375583005755830087558300758B8BCBC
:109AE000D80CA0C4D8584E30FFD8BC0E7CA0BE60A5
:109AF000F1585B657387A1C90B3F8F15B01A30A66B
:109B00007E677E777E8F1ED8BEFBA6DBE0D8A6F3ED
:109B1000E0D800A6EBE0D80000A6E3E0A95C98BC82
:109B20006D1EA95C88CBA95C08ABB83C588404E0E6
:109B3000044E70783C5A70AE38EEAE0EF0386E605F
:109B4000EE0C134EF06EAE7BD55C542B1C52F0E045
:109B50004EF0D460AE7038DCDCDCDC93D55C544B6A
:109B60003CDC5010F070F03BD4C7AE7038DCAADC9F
:109B7000DC7C94E36B300870AEE0DCA05C38521CF7
:109B8000AEEE6FAE0E7038D494BB5CF260DCE09C3D
:109B9000D4D4F2EBE048A670851458C15C4E708EA8
:109BA000783CC6B0C67F08CEAE584E3CE6BCEE78D8
:109BB0005A7AAEC39806374C098348E07806BCEE63
:109BC0005A3AAE5878E62BBC1AEEF0EEAE0C3306DD
:109BD00033AE2E6366E3AE70FABC1A3CE638EE3C58
:109BE00070662FEEF098EE41A4CC17266E78063CF6
:109BF000063C063C686E4435BEB8584898A8E0005C
:109C00004E1B4EBE5C501B2E7AD898463E5ED81C2A
:109C1000D4763654E3EEEE6BD86EEE4B2687D86ED4
:109C200026DFAED80E23D8AE2BD8AED86E9E5E5BA4
:109C30008E1E263BD8FCD86EA66E264B66CEBE1E68
:109C4000D4D4C34EAE98EE2E76767600CB2E7AD84C
:109C500098463E5ED8065E139E0ED8DCDC8E132E30
:109C600062F354CB98AED898FE1B66CEAE5C4ABF6A
:109C7000EEAE5C0EE66B3A5BC62622DE6EFA604EF6
:109C80001EE0C6C36E63424F66EAE32EFAAE4ED8BC
:109C90004E5C50EEAED8AE332E7AD898463EFA23BC
:109CA000D8465E139ED85EAE6E2E2BD8EE66D85C7C
:109CB0004E13228EF32EEED4D4D3AE98C1622EFA78
:109CC000AE5E1BB5A23ECE6EEEEE0EEE5A0EEEE688
:109CD00013BA4E9C4217AE8E4E6EDC50CE5322CE3F
:109CE000F34EEE94C963D4CABBA63BC3FEB7F6A736
:109CF0000E8E1CEE8A5C4A9766061B36E04E22CE1C
:109D00003EEEC21BAA260EC223EE2EFBDE338A6E67
:109D1000262EFB6A626B7E5BEE865A5E2A4EBAE0A6
:109D20004E709ECE68B8A606A8E07E78EE68B8A60B
:109D30007EBB4E7078FED8B8DED8E01D648CB5626C
:109D400098941FD44AC9622EFAAEDCCED86ECEF6F5
:109D50006026E63B66EE1ED44ECF66E076FA3B36D2
:109D60007E13484623B6AE932EF0BEF01E06FA8E42
:109D7000FB2EEE66DB8EB0B5604CA0FAA00EF81D8F
:109D8000620E6964EEB03D60556469620E556435DB
:109D900060696475624E5C2650E04ED88564EECEF4
:109DA000E05C4ED01050D050105090D0D050D050D9
:109DB0005CE0FAA00E8E2626065C4647D4941BCEA5
:109DC000E066D34EDA8C93DCD4239D642BDC9D6457
:109DD000D4D49D640ECE95620E9564DCD417DC95C8
:109DE00064EE4EEE93CA0A0ACAEAEA4A8C330E06B9
:109DF0000E46E04ACAEAEFE0BE6E8ED8988E4E2735
:109E0000980EE026CB5C626EA5622EFAAE045E135D
:109E1000081E1A6ECEE673CE5E7FDCD494856B2668
:109E2000DBF568A3B9685C336E66AE333A8EF32E09
:109E3000EE66539CE22B62E24F225C23AEFAAEE266
:109E40006B4E5C6A0E1C500C13A66E0E4C1B096008
:109E50008C1BBE1E1162228EF32E543FEE66D4EE92
:109E60000BEE4C2B2968AE6EDC909CFA9BDCE23347
:109E7000628ED89883268E7E9BCECECE626E0E0CDE
:109E8000396153AE7EF32E7E982BD8988EEEEEEE8F
:109E90000E6ECEEE2798AEE066CB8ED82695626E1B
:109EA0005A5E0E0C1BE1644C1F0160416AEE5C902F
:109EB000D010905010501050905050100B4E54979E
:109EC0007A103AD4E7543F148F94CF54FF9CD05C5F
:109ED0006B9050D05010D050101050905CEEE000BD
:109EE000D0501050D050101010D0D09C8B1CD0D01F
:109EF000101050D0509010DC2B5CD0D0D01010D06F
:109F0000505CDB5CD0D0D0D0501C9B1CD0D0D09CFF
:109F10006B2EFAAE8964B861500EF85EBB06BAF6D5
:109F2000330D62E6EB66EE5ADFE64FBE1EFEFE1E06
:109F3000FE1388B85E2EFAAE08DA77D164FA1B9861
:109F4000FE072E11622EFAAE3E5EBFDAABA606E623
:109F500083461BA6080E5E5A5C8A62228ED8988BB6
:109F60005CCE62AE4E4D6E422766EEE3D8A5608BA6
:109F70000160B32EFA0EAE0E26E6B35E57AEE56470
:109F80005C4EA60E6E3B08CB54F7D43E26DB738E98
:109F90007EF3982EBE333E6EEED4940BAE8EEAEA7C
:109FA000EAAE9CD086C6E35C8EEEF568A56CFAE35B
:109FB000D4BB2E9C822E8EB5680C376E8E6E2E6EA4
:109FC0001CA56CFA3B8EDBEEDB8E235EEF665E0C2F
:109FD0001BBE00B5600CCBD164496098FE356AA603
:109FE000EEDB8E29686E5C1B2E62F34226DCE08C71
:109FF000A04ED8B968EE75620EB968B03D60EB004E
:10A00000000000B0094648167616810B70C15A014F
:10A010000C10080120040114010401140120051290
:10A02000120F120D050D0F1219200C0F13140E0F25
:10A030000E0518091314050E140E150C0C10120938
:10A04000160114050F1514200F062012010E070526
:10A050001001030B090E0714121920010701090E44
:10A060001905130E0F12010D120F0D08B060303AD2
:10A0700070BC5C50100EC1B0AE307A0656A856D3F4
:10A0800049240CA08DBCF10E2170B8F0B00E4C2309
:10A09000BD701BB57069708D70B00E356069704C05
:10A0A00023B9701BB17081704670F84C1F48EB0EDD
:10A0B000B835606970AD7081700E626970A9708D7D
:10A0C00070F04E70F8280D729D585CEE615060EE95
:10A0D0006670EE38D494B34E70138CA0BEBEBEE052
:10A0E00025601B1D60A550F05CE0D4D4D4D4D460AE
:10A0F0004E7078BC26DCD4EB667038A05CE0217032
:10A10000B5701D74F0BD700EA970EE4E70EE6162F8
:10A11000842170B1700EA970356081648C27B57090
:10A120001BBD700E3560BEBEC9643160A970696028
:10A130008164A9702EFA0E0960C9644D60FE89031E
:10A1400005608C60F088B9706BB0FA33FE238888A4
:10A150005EF00E35608964B80E3560D164316005FB
:10A1600060F00EB8AE6160FADF0ECB8C1F88E08421
:10A17000E0AE88FE13485EF0B0FAA00EEBAD74E3DB
:10A180002E0E7AFE4B480C338C238488445CA60642
:10A19000E6B177468FCECE235C62EE570C0785641E
:10A1A0000EA6AE3D7A0C0D633960AD746ECE5C5A6E
:10A1B0005E26E6433ED454D3EE3D7AD84E3ECE6B77
:10A1C000AED8221ED8AEAEBEEB1E2EAE8ECE93D82B
:10A1D0003ED86EEED454B3EEBD606ED8469CEEE130
:10A1E00078EE132E62F38E42FA1BDC9B0CE389643B
:10A1F0000160A9640960D16449601E0560B05ED841
:10A2000098464D60A606E6A176B176DC6654EB5E14
:10A21000B5608C3BBEBE696431608C2B6964316073
:10A220004C87696466660075608C3F4E5C66503D85
:10A23000604C13BE0C60F0E04E6E5E546F94EFD431
:10A2400027544F14679CD09CE0DC90901090509065
:10A2500010505050905CE09094F3631C5D789C50DB
:10A260005C109CE05C5D789C50DCE05C5D785CE0C0
:10A270001C5D781CE00808AE0E2EBAFE43880C1B4D
:10A280008C13485EEE4C457B8C2BAE0ECECE4E5CD6
:10A290001050EE66F62F661B268EEED898EEEEEE88
:10A2A000CEEEF69F8EFB2EEE66DB4EEE98EE4C1B4E
:10A2B0008ECEEE8E5B2EEE98EE4C0BE6F7EEEB8C30
:10A2C00047884C1F48734463840CC38C1B842B88C1
:10A2D0001B8564436E8E00AD743B26F6278EB32E2D
:10A2E0006600B5604C5F98EE66006960696449601D
:10A2F000D8AE0E263B6EEE3BD454B726E36E4EEE40
:10A30000E178EE133E8EF32ED4CEEE549BD88E8E93
:10A310004E5C50D89C90905B8A8ABEEB1ED8AE4EA5
:10A320002ED88E1E62ABAEFAAEFA0B7E661E8E9BE8
:10A33000980C4F8C3B396023B0D898464D60F0D1D3
:10A340006449608C13F08C13BEF00B5ED8AE98AEEF
:10A350000C1F8C1F866EDAC3D8A5600C7B8964D174
:10A36000644960016005600C8739604CA0BEE04E16
:10A370005C6A560E8E0CA02300ED64FA0D63B04C9F
:10A380009F0E1E4E5C66D01D604E5010D0D0D01077
:10A39000501090109C506960F60D62E01CA09C6EFD
:10A3A000138E26F34EAEEEEEEEEEFCA0A2E0CED47F
:10A3B00054AB139C42E60D63B0221FDAEBAEA24E03
:10A3C0002E5C105CEE22270D622EA2F3A637EEEE75
:10A3D000EEFA9BAEB04A1C5090B562B0064E3055B6
:10A3E0007C067C30E04924B83CD88C1F881384D884
:10A3F0007CA8E0302D9C58A051B698DCD0CB06C08C
:10A400001000000000800000000000048080042094
:10A410000020030001080CC41431000D320003CCED
:10A420002B28900210003314900130021028400CA9
:10A430004070A2015039980332900004800000005F
:10A44000C0000580000000005002420AC035003004
:10A45000300000DC000C8A04000068CC39000000E9
:10A460001AA031C1030230B9C040000C00008C00BA
:10A470001303C680088000B32100000850C80032D2
:10A480000800088000080800040001D9200C80C8DA
:10A49000A024933920000000C38D06083068000313
:10A4A0003000F30125000840009013900343A64DAF
:10A4B0008E0C307003190000000003000000000043
:10A4C0003000030000003000C3D0000004C0004290
:10A4D00000380C20153700F7CA89886FC8CB02F303
:10A4E00033840090D00300000240D95555555505DE
:10A4F00095657116695AAAA9EAAA2AAAABEFAE0312
:10A5000054285A3FEFFCE3C38B000BEE2A1E80FC5D
:10A5100000AF02542196A9C091EB95E5286ABB05CE
:10A52000550AC467A25A0A99872352F51188FE4F2B
:10A530008D13EF6E4D0CBA3833CCCC2000002CDAE2
:10A54000555555551500155515005555154055557A
:10A550001515551510001000000000000000100037
:10A5600000401040101560D50CEBD10C448A12123B
:10A57000FFDA8C88221341418B63680C8859206272
:10A58000800C302003C0083E2CC100AFC4C0F8BC12
:10A5900007B3CE204F11138087FC110AA08A8028B0
:10A5A000B820C938808C02FEECC17FFB38FF40C266
:10A5B000BBCFE3684E4C4CBCFF4E5CA80300953902
:10A5C0002292DDDB4B2FF470010F3FFFE12040F2C0
:10A5D00004C631E2C8C8FF310AC88CCCDF8720012D
:10A5E00009C9BFF3EF0B1220131124C40889E01B23
:10A5F000484322C4008F24003E46402C26233C3F83
:10A60000800314D0E76361134F1344343619314D7E
:10A610003B442A400129924FFE51D23C70212838F8
:10A62000CCFC3E400C04506029064CDB60F74E0128
:10A630000C002554D8F36063F7F187AAC1FF8DE3BE
:10A64000224BDC7136EE03C5084A8E288C927410BA
:10A65000CD0420812BCEEF8983040040B74FB00793
:10A660002010224988B04ED24F861258EFA11D0FFC
:10A670003BC0323C3F11CCF21C6F974072FB423D15
:10A68000B51F02300004E3844B12F4760BA2788CE1
:10A69000B30948006262173B0202862D52B8FF11CF
:10A6A000E25E5D50B2C46D0A100C403040866831E5
:10A6B0002658594D241452330029410718240720E5
:10A6C0002900A48002C0C4808CFB0B9522000B786B
:10A6D0008E00AC928400A75423CFF8092044F630B2
:10A6E00043C0B5EE5E298FF0735A2323CEB4001118
:10A6F0008C3CCC0B480C4442BC90393E9320082142
:10A7000000203D460000040040000010000004044A
:10A710000001000001400000410441B915376CFC04
:10A72000D1170304C3CC500C0C330860C4CCD0CC7C
:10A73000800411230A3FC6C80080FFBF78EE8A3F1D
:10A74000034C0322CC3401304C21002330108028EC
:10A75000C33062E2500005C01088C0FCA30438C5B5
:10A760008424B34DCDE02B2F043C123028DE40383A
:10A77000647D1374C6374208403EF6030000C140B2
:10A780002194C83E312220022085006B84CEC8046B
:10A79000599D5316097D7F71D8C532E1463B8038FB
:10A7A000133040C785224E5523DD0E054F4490CC13
:10A7B0001CDDBFB88B44A074125022129130970355
:10A7C00000767FF74C17DF8445CE98F2D949140202
:10A7D000C42012513222C900048C4A3B4BFC800336
:10A7E000050B0051482B0E31EC502DF0DF38C8130B
:10A7F000ECCCD8513D300451FBC73EF37F0CD00C5C
:10A80000441348AD7056390C51844E584488A18089
:10A8100095BCF0B3D5888A3E23E6D7ABAA0A704D23
:10A82000A47E7C81BC8D8CB0AA39887309504E5BA4
:10A830000CDF98EA2DBE0AFC4DA459A4AA0A582997
:10A84000A48A41A4CC57980647662F022762130AB0
:10A85000AEFCCA7004B00A8AB0CA70E5A47CE21FDC
:10A86000F6B362BF62ABF62BF61BF67F0C5B980A61
:10A87000468D8C59A498AA58081304B00A7C060F78
:10A88000662F02EF62DBF5A8B0AA70E5A4EA987023
:10A890001CA18C98622362626E6258B06A775582FE
:10A8A00046FC708A980A29A4BD8C6ADB20B07038F7
:10A8B0009C5898700E388E8E1CB63FB6DCDCDB02DE
:10A8C0007B4AF01C6A101C02BBA666700A4EF09808
:10A8D0007CAA698C70389C98F0467078A6682E66C1
:10A8E0000DBA6670EEF0EEC34670781C10701C0A4C
:10A8F00038E039883E37FEFEFEB183980A7CAA69AB
:10A900008CFC4DA4AA58B00A4DA4AA0A70E5A47CF8
:10A9100022DDAFE078E64E30C058708370383E9349
:10A920001CEA277CEA2371841B5584C606B0666F37
:10A93000E07EEEA0FEDC58B098701CB0FC6A6F7C24
:10A94000705584DE7985AB00000000000000000037
:10A950000000000000B0702E70380E3B55849870D7
:10A960002E58AEF0E07858EE8B1598EE810A4CEF39
:10A970000C27D588671CB1182BCCC3A918AEBC30E6
:10A9800076767627D588437AFA851406DA1A300661
:10A99000098366E64670787066BCFA38D884D8F0C9
:10A9A000BA3A301C62027CA23C0E3A300A7E27EE94
:10A9B000EECBEE3C7066EEAEF0EEBC663FEEAEDC8B
:10A9C000901C3B3C2606467078A6681C02C4BD8CD1
:10A9D00009B81D02B8463C584484B0E06259A66EDE
:10A9E000E0C461A4CAD844D885A43C0AED1ACCA01E
:10A9F000D5886A66A08CE746E000000000000000F1
:10AA0000386B3823380338E338C338A338FCE00008
:10AA100038E038933873385338333893387CE03C17
:10AA2000E07CE07CE03CE086EA667038CAE086E6DE
:10AA3000667038C64B42EAEAEA22E2E61FC61BC647
:10AA4000360A1B261B62620A707C3020FCE0AAC317
:10AA50007CD80CE92F758879A085140CCD071902D4
:10AA60007CD80CD12F758841A4F80C83E6DDA9654C
:10AA7000504C1346261366E8DD8CFBE61F26E8657E
:10AA8000144C1938655026E8E55C75067858EE8751
:10AA9000CC1F41A4A1A48584CDA8884E66480B157F
:10AAA000981CEE1B0C7B810AAE668F840C731B888E
:10AAB0004E704C47CCC98F41A4F8CD84E844B044D3
:10AAC00070198C4C27B066CB95A47CAAFC61A47C41
:10AAD0000A4CA9A76550E62398ADA01D0245BC11FC
:10AAE0000C711C2DA84CAFE0390C0860BC580CA0B0
:10AAF0000498DDD83BA188B030C570CC1F4C1B79C1
:10AB0000A055C42DA87BAA0A584888F5A898AA5829
:10AB1000334E59A48D8C986ACFE0AA8A700A7C3093
:10AB200083FCE0AE1C8A700E7C3080B31DA44BCC3D
:10AB30003F4E70F84666E8467038AA0ACC57E213D2
:10AB400022E21322E2132228E04CC98259A49DA4D8
:10AB5000AA0A29A4AA5839883E5F488C337EFEFE93
:10AB6000FEE3B0E098EE4DA4E5A41C6A4F06E64E65
:10AB70007005BC95BCCE581C0A59A43988FCEE98C7
:10AB80007C1D88EE7CEE6A461746363606277676BA
:10AB900013266A698C980A84F5AA584A174A4A23E8
:10ABA000666262E6E6E6E61322CA101C0A986D8C1D
:10ABB00098E0B9844C1187AE41A444F8E633E5A887
:10ABC0004C3748655026E8DD8E30DADADAEEEEE012
:10ABD000B02BB03A707A258CF3B02BB03A707A254E
:10ABE0008CA3B02BB03A707A258C53B02BB03A704E
:10ABF0007A258C3A3A3A7CEEEEE0B0703C467CE046
:10AC000066BC1C3A3076F6E7E23FEAC3666AAF03F9
:10AC1000222222227B9C229F224F3A3A301C22275A
:10AC20004E4C7F488EA9186EBCCB3A3066AF7A7A0C
:10AC30003C1CE044448641A4CC3FC6BC584C1B4D50
:10AC4000A4E5A47C82E2DFE237E2AFE223DDAC934D
:10AC5000F68384763CAEBC9C98161C66673C0E2935
:10AC6000A48C29A54E70AAE03C0EBB59A4A3E2E730
:10AC700036C736C739883EA74C2FED1848234C3BC2
:10AC800041A44DA4DD8C4E70E0E5A4884B7D9C98DA
:10AC9000CCBF4CAF4C9BCB5C42EE2B0E4E701C4A93
:10ACA00033AA7C8E8ED33C58681598EE9B0C1FC43B
:10ACB000934C7B8CA758B8E683B85898BC30E64BC9
:10ACC000E0C81C0A1DA4A37D9C8411007EFE4B8D50
:10ACD00008063064069B8D901C0AB8E6B38A636A46
:10ACE0008686A644D190EE60810A4670CC2FB85873
:10ACF0004C83B80A38AAFC0EF8FCAAE8AE0930ABBF
:10AD0000EA0130091E04CC7F4C6F06984C8D900CE4
:10AD1000870ABD8CC102CC330A0238BC3A30A6B6D1
:10AD20003A30FCE64738AACA0C4B8A3B384AD3086B
:10AD3000EE41A43DA43DA4AA0A559CEE530C3BEA67
:10AD400049A4E5A4D6E63342EAEAEA22E2E697C657
:10AD5000EAAD3CD86A8C8346425366985846704B9D
:10AD6000C63673A2A2B3AA62620DA48308AD3C8466
:10AD7000D8064891900AD8662702331B061B04AAFE
:10AD8000464223666262E6E6E6E61322CAE641A48C
:10AD9000EDA47CC63CFAFE8D8C59A4CE7C8D8CE54E
:10ADA000A4D8840C1388D88D8C980A7596190856E7
:10ADB000A08A16CCC3468B02A6588C3B84980638D2
:10ADC0004A4B0638AACA237D900A499646BBEAEA4E
:10ADD000868638E2AAE2270DA48B462222421B6611
:10ADE00053A2A23B047D905841A470986627023379
:10ADF0001B061B08AA0DA45697E6567FE68AB0AA42
:10AE00000C1322EAEAEAE63C8D8C9825961C903CCD
:10AE10001E98EE6A21B0001CF61B101CEEEA3CEAFC
:10AE200023BE2F7B3CEAF358845C4E7050FADA9CC8
:10AE300030583A30E6575CDA22A3E5E200D0881CAD
:10AE40003A308C97E63A30C61FE663E60EBC427C89
:10AE5000A67CCA70BCA6F6F6F6A33A3A0E303C1EA3
:10AE600078AE7E3A3A306A677E8E8EFE2F4A2F4445
:10AE7000E34A97BC631C06461F4EE030DF0647C618
:10AE80003C020ABC059AA6FCCA221C70BC0E98AEF5
:10AE90007A30EA8304D88C1B8408D86A3F8E8E0CE3
:10AEA0004F4A777C8C173C019A4ACF48B09C108C53
:10AEB0009F0E3C7A7AFAFAFADAFAFA9C98FAFA9C35
:10AEC000901CAA08E0781C101C0A70383CE6359AE1
:10AED000D5883ED37C62588ACAFCCA0E4DA459A4B8
:10AEE00098EE6E6E1CE5A46E1C6A578E8E986258A2
:10AEF000E24B4A871CCE7C0ABCA34ACF4670CE7C6C
:10AF00000444E0441CCC1F4C3BF80E38AA7CEAEB0E
:10AF1000C8E247C4EAEAEAE66FC628AE4A7CE8F827
:10AF20004666E8890AC6369B4E7048D3C44CA0F8E2
:10AF300046E8CC5795A43C0AED184435BEA918DB69
:10AF400036AF335836C7369903CC1F4CA349A43DBE
:10AF5000A41DB43C3E6B980E4670110C1B19088C56
:10AF600060D91CB8492676C321067858EE319EB8C0
:10AF7000AAA81598EEA19268B806FDBCEE3BB80EE3
:10AF80000801AC1B95BCB806EEEE787CEE0CFF78A1
:10AF9000AE3CEE1C4DA459A4C1A46E1C6AA06E1C4C
:10AFA00058EE8D8C1C98EAA0AE4670855201AC0C10
:10AFB000604ECAFCAA3C7EEE1DA0EE3F706E85502E
:10AFC0000982705838EEF0982606C3E08E85506EE0
:10AFD0000801AE41A4CC2F46CA4602B8AAA8E08C0C
:10AFE0009F061CC3300B0604B898A8A63CB0FC1CF6
:10AFF0001086BC5C221B29CA30E6D3E000000000AA
:10B00000382338F338C3389338633833387CCA3C34
:10B01000B3FCCA7C933CCA7C737CCA3C537CCAFC9C
:10B02000333CCA7C13CAF01CE03CEA7C23D588225E
:10B030003803389338633833380338D338A3730070
:10B04000385B3833381B38EB38BB388B387CEA3CFC
:10B05000EB7CC2D63CF0AA0A6E701C1BFCEA7C7327
:10B060003CEA7C537CEA3C337CEAFC13EACA47F0B6
:10B07000983EAE4670E011A0EED3A5A461A47C1D5D
:10B0800088E6132E698C980A3C1C2376DCDC76E378
:10B090004E70786E682E70E638E66670E6F0E6264A
:10B0A00066A7E6AEF04EAAAE38AEF09870384AF019
:10B0B00098A9A6980A4329A44685A47E58FEC74CA1
:10B0C00013C809824E1C70786E700638EE2F30C09F
:10B0D00006A04EE0CC8795A43C0AB18C41AA2DA8CD
:10B0E000669FE68BE841A4CC2FA1A4D84A2709503B
:10B0F0001B29A4EDA47CC4483BFCCAAED851ACD8F3
:10B100008AAE06B7662F02976A833CC9AABC08308C
:10B110007A76EF3C7E45AAA3583C0A4DA4EDA49C48
:10B12000D08D8C98E041A4AAD8A1803C1BD588D8AA
:10B13000063F6660021F62607C8ACAFCD83E67D800
:10B140003CCA7CD8447EFEFE1348E6170A4ED8E07F
:10B150004E70381CCC17E20AE01CAEE6BD9E5A26A3
:10B160008F263B301D7C44D1026666FC084DA8C585
:10B170000278101C0A703988E62709503BD5883EB2
:10B180006F4DA4E5A47CE21FF6D3B06ADB11A0EEFC
:10B1900009829C101C3020F0B070660A38D88408F0
:10B1A000D8F04E70786668C4B18C0180BD9CC10235
:10B1B000CC53AE0EBC30E04DA459A4AA0A707C302A
:10B1C00021FCE0C6C2A0BB1CCCB76262627186CC17
:10B1D0008F1C23A237A2A22FA2E0A2A2A2A2A2AEFB
:10B1E000E06EE0469C5845A4AE58707C9C98E61CE6
:10B1F0003084FCE0C98C8ECE5C581E99A49EFE5B08
:10B200003E3EBBF5A891A4CDA883FE95AAFEF75CAF
:10B21000224BFC261CE2CF8D8C8B22A70422170820
:10B220008DA4300F0C2391A453F5A82691A48DA4CE
:10B23000CDA841A459A49DA4698C7C698C0C63FCA5
:10B2400061A40A4DA4DD8CF846E8C502FEFE37CEA7
:10B25000DC95A4BB5C62439CE2B790FC5DAA628370
:10B260009CE26FD0BB8DA4FEFE33FC261CE20FD007
:10B270001DA45378EEA091A478CECE68C330F0AE72
:10B2800058782366CECEEEE798AEE0F8261F66E04B
:10B29000044E6EA05CE070CCA795A40C133C52D871
:10B2A0004A431BD5883E33E6DF09503359A4E5A451
:10B2B0007CC4488AD80EB0CA70AED851ACD832AE71
:10B2C000724B06AF662F028F627BAEE3A9184EAABF
:10B2D00058AA0C41A4B0AAD80E442BE5A84C3F7242
:10B2E00098121B0ABFAE707C066550A01C4C60A66D
:10B2F000E8B00ADD8CF8E0C41BC488CC27E5A403C1
:10B30000AABC3A30F6EB3A3076EF7A76E11B488CFD
:10B31000A91A7ABBA24BAA626266700A387CA27C28
:10B3200082E2FB2222A0F62BF61BF64FEACA8DAC76
:10B3300082E25322223BF6ABF69BF68B29A43CCA51
:10B34000E0E2EBE2FF36EF36DF8C258F8DAC8DAC83
:10B350002237484C6029A429A48C173988ED1AE2B9
:10B360008B8DACA253AA101C66700A38FCE0A27C3C
:10B37000E0E22FF66051AE7660EA8DACEA76DB0350
:10B3800004781C10581CFCCAEE30BF26AED8666B81
:10B39000D8AE7070383E437E1E1C6A237C6AE74A32
:10B3A0007F1C8A8AA6B63CCA087C7E137CF03B0CC4
:10B3B000234A3CB33CD84670D8E0B083D813AEFCE7
:10B3C000EE707C1C0A3988E6CBD5883EDBFCAA0EE1
:10B3D000584DA4E5A48A1CDA7C0AFC6AB74A574691
:10B3E0001CDA707C0EB0EE730C33466E8D8C3B987D
:10B3F00008231C980A7C8B3020061CF86AF3B8E0FE
:10B400007F61626364650060060405010C1D7E0DAA
:10B410004EF05C90308C3C0EE5A41CEA5730051CC5
:10B42000426AB7C1B06B3CC1B0E02B6E30051C4224
:10B430006A9F9E301F0C23E8BE3726BE1FE8EBE054
:10B4400020DE6DBA5E270C71B049241CE5A43C8E49
:10B45000D91C7C5675B0AB3080A330C08B0616303B
:10B460003A66AB302C66A3302E66F7304006B8D86B
:10B470004C5F8C4FD8DC101EDE7E3353D8E8302072
:10B48000DE237EBE7E70E8E0163020069730600630
:10B4900073A6D844D806B03070A646A0061B4E5CF2
:10B4A00090101C30663322E3303A5B3C56363B0E3C
:10B4B00041A4C1A41C426A60FC5C021DB48E9C586D
:10B4C00006164670307F66851DCE0E1C7C66DD8FAD
:10B4D000FC0E1DB48E9C58467051B473E0200C6075
:10B4E0004C3FC8CC37486D00CC603080E666FBE04E
:10B4F00030107030FDF09C4ADC909C905C901C9069
:10B50000282828E049246E1CCCE5A66EC9A6381C64
:10B510003CEA6D591C387C0EF87C0AAE28B87C0ACF
:10B52000AEE8787C0AAEA8AE9C9868E0E6251CE6FA
:10B5300056069C58B87CD804D83CA8F6F62F468707
:10B540008CE70C23300BE08C273077E03087E0303D
:10B550001C66273054E09D580CC92289BA84B898DB
:10B56000A82B88B898A80CA78CAB307F069C98E6CF
:10B570008D2666AF652083B83CD808D87CA8D92032
:10B580007924BD2025241D0239B478FE37FED91C4C
:10B59000B81B09B8469875B031B8638C41BB41A45B
:10B5A000198C4E70D92041A41E8EE5A41CEA2B6E86
:10B5B0008DA41E46700C1B29B8E05CA078A0FE7B11
:10B5C0009E60FEDE7E5B8C4BFE301A31B8B37E602F
:10B5D000FEE0D4577822AF145762DC5058D4A099BB
:10B5E000A4130C778CC37EB77EA7C314B794A70CA3
:10B5F000931CA0301B31B878F65329B83BA08DA41A
:10B60000042BA08DA4088D141D02301C9C5899A6F3
:10B61000307F66937846977EFE2F410CBD8AAE8DB3
:10B620008C29A44670AE68633E236520E3AE99A4DE
:10B63000BE008B1E41A459A4BE1EFC1CD08D8C7E66
:10B640000723781E9ED91C5EA0BEB8E3301FE830E9
:10B6500020DE7E6F1E3E5E23E8BEE346F07068E0AB
:10B660005ED3B8580C373CD888D87CA8469C98063E
:10B67000307F667F781CEA3FDC10FED91C1B09B8BE
:10B6800061B6851CDC10FEC1B051B6C98C9C9870A7
:10B6900041A41E30F19C5899A4B09C5899A4AE7E48
:10B6A0006815BA4E705C105CD0100EB8B03C06FA4B
:10B6B000FA7C4638BCA606583C28E0E6174E7009CE
:10B6C000503344A180AA70040A4DA4EDA4D80C27DD
:10B6D00004D8330804D88D8CB00E3988E603D58899
:10B6E0003ED7AA0A704DA40CEB08EDA47CA24BAA8D
:10B6F000626266700A387CA27C82E297E2EFE277AF
:10B70000E263DDAC4BB0E60F700C4B41A44E70E829
:10B7100028DD8CB8584CA0D5885FE27FE217365FF1
:10B72000364F59A4E5A47C22D7E38DAC0BEDA47C65
:10B73000563C8D8CE5A41C4AEECE8D8CCE7C63E508
:10B74000A41C4AEECE8D8CCE7C1BA6FC586E1DB47C
:10B750001C980120C3AEBCD91C0C733A3A3006A623
:10B760003C2EEEB9BC04D5124D140912D91CB9BC3B
:10B77000CE3C061EA114B81CD0E8661EA11463A618
:10B78000EE1C1084101C421F02889C1BDCDCB6EBF4
:10B79000E6161FDCD64E94602213E2B6F30EF88C48
:10B7A00017B858B0E0EE2798022398AE4EF0E0CEDE
:10B7B00070989801207B0C3FB858B0AEBCE06E4D3D
:10B7C0009CCE0592810A4404040C4745A4E5A45983
:10B7D000A42B6E2DB46E66E66ED91C4CD9B0D9126E
:10B7E0000C23EE58EE04D80C23080408D8E0BD1C46
:10B7F00018120F0D20E000000000000000000CB93E
:10B8000062204038238038C4F800C4039D1033D42C
:10B8100010D0CC0C0011802C2E122151C04411717B
:10B820003333809043A21A1F0035802093C1477F95
:10B8300020C4A3612032E2CCA3C838491C524981FC
:10B84000304443C8C64304224B1204F1EB003038A5
:10B850008431000000A00091869B8CE3321070D0F0
:10B860002A8348F420B806B3F836E2C90F0A92805A
:10B870003D86330033E3C94D03DC50C1832303000D
:10B88000440400300C00C07C373B280C0A5359CCD0
:10B890008A6892C4BDCC0431BD4C0C0E04E2A07881
:10B8A00038E00326143003DA203E180470483C4B7D
:10B8B00040E000002920CD9C84FC92EE2E4F87C0F2
:10B8C000804CE14430D00F461263E483E0384E10E0
:10B8D00086E1330334141258D131B2348A104D400A
:10B8E00004C0A0A20894D3206A153E053D0BE132A6
:10B8F0002138FCD7913944E6109943648E7A557209
:10B90000B4EBE27EAA2FAEEF8804E9AB701248C414
:10B91000C87675C4BED2C4D03CC8E4E8E2E1121ACD
:10B920003180CB4E02C258F8F06F8E0808A57D6DAD
:10B9300041C308EA1433A4015FE083F2604382004C
:10B94000C02C50CE0743710E6E4C8FF7C40C0D0601
:10B95000211895C54C4851A37B8DCE8DD7D40C139F
:10B960008A5A851332020C836C3854C8030C2CDEBF
:10B97000D1C404F37FC49C46D74D41334CCC3C0F1B
:10B980006195D01805C2D2A0C47A84C1E3121ECD3D
:10B990004EB838910C51A57DA23EBE8C3DD2704F61
:10B9A00060813B152E2DF67C3C70BC08A456179484
:10B9B000824F240AE00A40330108CF23F240F808FE
:10B9C000BA08D92008553CE038ECA8FA0C5021C43C
:10B9D000722208C7805E0808CFE1608E388E16623A
:10B9E0000B622F880833C20F01E7A0080328232227
:10B9F0006060FE084B0087B8C3913F2759227B0047
:10BA00000400008C00444400C820CB0DC4CC8C281A
:10BA1000C404008C0C4AFA0011110088093E06404B
:10BA200088508FEFB82BA0880F0260824D3180B90B
:10BA300008E01A12CF000522EE0741338C3C00418A
:10BA4000F0F3DFD43ACAD5C843078D40F3F3004979
:10BA5000515BECD038508380486C28C91C1132806F
:10BA60008C2CCE8CC094688C8B3B003040FD0C49F4
:10BA7000520D500D40145D55373324C34902C3188D
:10BA80004A4C50D8821B6449133184331103820419
:10BA9000D0C03C09CC4B0EE0394F8EBBB33EBE0745
:10BAA00049EFF1E22100414403880F230F051024E0
:10BAB000F3F30F015540C544CD03013C13FC0C4882
:10BAC000E4EEAE11E1816ADC861EE11086D2ED2340
:10BAD0008788181116CF704444301ADC878313B856
:10BAE0004C01847421983DCDF02034C9E0868D014D
:10BAF000008580438D30C40C208103604861F4FFD1
:10BB0000000000004C71B204FCE0180143C461BCA9
:10BB100013D30422336110447C7C4CF4217B0C1F32
:10BB200042FCC4C470D7F14CCCE3313821E310306F
:10BB300081F11008040CC2DEF228DFF9611C20300C
:10BB4000D50148E23A7B1D76D411D30434F777351A
:10BB500000B1C4714C2C48F0C74F128D33C2FD0D9B
:10BB60003131A0301310B1108010200B030A302A9D
:10BB70000A3204AC608A38CC3C23C2CC4C800A32F6
:10BB8000C1141333F18E22020C2222327131E443AC
:10BB90006ACCF771203937EBFCD4DF4C312DCE1055
:10BBA00032CE880C41CC30830236DF5B91D1B8C1F4
:10BBB000E4008D3C4D0F140E4A4C2007AA71DB5156
:10BBC0001DA342A0C3FB102632B21ACA083200BC21
:10BBD0000C008F0002D0805EC834233310F30F7343
:10BBE000DB2E0DDFCFF152F7D84B123A30000FC5E4
:10BBF0003043CBC810240C3341B4E43F000E004066
:10BC0000193F0097013B01C60A430AD2057C01D2C5
:10BC100001520A19008809B409AC0D5B0D630C16BA
:10BC2000016907F7037206B20E6205730E3606ACA1
:10BC3000080B0A7B0A85010303AF02B5068600B133
:10BC40000DE403490F530F5B0EC30EBA062D085FB8
:10BC50000E690E2F08050F2C0F350173035703C013
:10BC60000C0400AC009D03B809A300E306A20B2F4F
:10BC70000AFC00F7012001290132023C02CE066CC9
:10BC800000009319050B0C030B8045628432200ED3
:10BC90000306201418052D8D0F0F1213010B80556C
:10BCA0006A8E0306201418052018032D851A09131F
:10BCB0001001C870F868385C581C0E38AA28B044C7
:10BCC0005D5C385CD8284C9B5D1CCC274C09820DF0
:10BCD000FC0E0F20120F0F0DF1FE80BD6A981209A5
:10BCE000040D0581408001620DFC04151020060C36
:10BCF000F1FEBF0705124E78BC067CC6007DC68EDD
:10BD0000130110A9D09868F8F67B0DFC0B051903F8
:10BD10000F0405D9FE009D0E809D66BF0E0E3D18D6
:10BD20000B802D4ABF0E0E4D180B805D4ABF0E0EC4
:10BD30003C180B808D4A870E050C01F9C41379C499
:10BD40000C1B06434E3005EA6DCC66A606E0980F44
:10BD5000140179C40C1B2E53468D8C9C985606F505
:10BD6000C4B94A851A09130C068889E8B08BBF0547
:10BD70001A0913C15C4E70783CC62B0E1B841E3012
:10BD8000107046F0A1144E708C60DE9C7E7E2726DB
:10BD9000D4E30A061E5C422FFAA6E30E8EE0E1C44D
:10BDA0000459A4EDA456E63F3005426AAF089C58FA
:10BDB0001C38FCAA0A7C28E04E703830081C901C05
:10BDC0000A838D150E0179C40C600B801162940FEB
:10BDD00012010B80696660B0307CDADAFC3A307CA4
:10BDE0000B00E00B00E0D05C3066603AC60E300617
:10BDF000A075227E477E59F37E19637E0D4EEDDAE3
:10BE00003CFE4E66A63A5C105C223730C6E3692ED3
:10BE1000D05C30C6D7CC2B71CC66D3550E7C1C3091
:10BE2000060E7A30EA592FA6D3CCDD0E5D1C4CDF0E
:10BE300071CC66BFE92EBF0E0E3D3C180B80714AD7
:10BE4000F80E30E82BF80E3000E6AE6150600E566A
:10BE500037300306E3AE8D080626D3E07E7E895395
:10BE600060065E46FAA056607CA647FCA62FFCA69C
:10BE7000B5A2E10A814081C866BFE6856813A36662
:10BE80003168C66687E61568D34BD05C30E613E0B0
:10BE90007CE046E098E0D91C788C2B84D8842388F9
:10BEA000D888D8F0492660A0D91C783CD888D8FC1E
:10BEB0009B81130F100B80096A0B80F96A0B802598
:10BEC0006A0B00CD9E0286C6E0BF0E0E3E180B80A8
:10BED000C54AD91C30126A5F78D88C1F881384D861
:10BEE000F06330706A63411C30186A9D7E4EF00525
:10BEF0007E78E2D3411C4CC76100D1441BC17E193E
:10BF00007EC676C3A5D00C60C6762330EE13469667
:10BF1000864686AE0E7C0A85D026E61C4E8223A677
:10BF2000A2A2A21F26E386EA02AA0AEAEAEAAACAAB
:10BF30002AE0856813E0A6062658D944E0EB5D1C8C
:10BF4000214687010C060C0312B830FF3CEEB94ABB
:10BF500087010C060F14130B80FD6600203C56066B
:10BF60009CE23BA0005D1C21463087E099050B1444
:10BF700005070B801D6681408488ED64BE58300241
:10BF800089408808AD402570BE981D608CA7FE1FB3
:10BF90000E5B0E300555703BA00EAE00D164EE89ED
:10BFA0004C690208A140257088A393100C03100B64
:10BFB00080696E9807120C030B80C162863E3C18A4
:10BFC00015C845CCB87CAA3CA845CCF5C4CEE871D0
:10BFD0001E5CE6A616E61376A6E6E6E6C6A6D4142A
:10BFE000A3E09828C488C4FD7E3E4E302C5808300B
:10BFF0004070387CE0304070387C063CA6BCF0E0F5
:10C0000059A413A63040562B3001B6166660A5D051
:10C010000CA01C4A2A704E5CAA0A7C9C4AA606F018
:10C020007C70383CA606BCF0FBAE0E7C1CAAFC0E55
:10C030003040562B3001B6167030EF06383C662380
:10C040007666471C4A2A703866F308AE0E7C1630B6
:10C050000156BF0670F038665BA6360670F038668B
:10C060001B062B1C90D0061CE076173670383C66F9
:10C070008B3001763F2BEDA45626E66630075A1327
:10C080003AC6F306E6BCE2667CE62B4E2E1CEA8539
:10C09000D04666064B66861C82A0A2A27BC666A519
:10C0A000D046A063044E70F8EECE71C8700439D04B
:10C0B00006B0BCA6700C1F08B30C60783C06B03C00
:10C0C000063C068C3BB958BC70B95A3C70E06EA077
:10C0D0005627FAA6F330030C1B6608468EAE608D19
:10C0E0000A304056A03001B616E0041308081B04BD
:10C0F000044E7038DC901010102884444E5870386C
:10C100001CFCEADCD0BEEB59A4EDA48A1CEAAB0A05
:10C11000302C6A1F48B3885E5BBE980C23AA3C1B78
:10C120007CAA581C6A3005426AF78A985E630C2B19
:10C130003C58BEC37C1C9010CB2E5F1C38FCCA7CC4
:10C14000288C6F0C0B0CA0CC23D5886A41A47B0CE7
:10C15000A0986815980EEE734C670C771C9DA47C14
:10C160000E7C0AFD1A0DFC0E010D05D9FE83051289
:10C17000140507884B8305120C031201840B80A160
:10C1800052E54C0CA0983C063C4C3B0C17060C139B
:10C19000463CA63C9C4A0EA04E2F8C7B5C628E6671
:10C1A000665C1BFAA642EB8C13BE600D544924F862
:10C1B00028AEE8B5BCFD5A064C2B48B03C06CE7CF8
:10C1C000A6FCEEB0FC061C0201D08408CEFCAA0A34
:10C1D0007CEEEDA456E6C6762697CE7C4C1F261341
:10C1E0006603047CAA0ABCC6BCEE8CC3B07CA6263F
:10C1F0005F0C4FA646BC26BC703A4BA626E6EDD097
:10C2000063FCEEE626E6EDD00C604388983CAA7C01
:10C2100058E0CE7C0698E6B07C463C70B0FC70BC22
:10C22000A63C66063CF0E09301051601130B8099CD
:10C23000568891D04E70F80E300255701BB5A2AEE4
:10C24000BCEE514C4E70783C06F8C4FE1388CEF616
:10C250001348A67C9C4AFE1348A63C583154BCEEB9
:10C260008940A808B156BF0E0E3D3E180B80A14A6A
:10C270004E75F0EE600DFC0E0F200412091605F14C
:10C28000FE8C06130F1049F0F9C40B80E6E956BD89
:10C2900056585D1CCC604C6060B03AE08D0F0F12B8
:10C2A0000D050B809D5A8215131405074433901415
:10C2B0000507480B80594200BCA8E04E0070446856
:10C2C000780605BCEE59DE785E3E683C06660401E1
:10C2D000AC0EC1B01C0C0742271D145BAE012063DD
:10C2E0000C77AEBC4D14DDAC4924E304B1BCC36E85
:10C2F0006EC9A46E085346F059A4E5A459A4046677
:10C300008E060404D91078065830301C622B30B0E9
:10C3100062275613B6D91CB8B81C101C8C3342B80F
:10C32000302DE876B63CA23C3E1E7E7E8518492420
:10C330005DBC99C844785CE291DF3084CC2766EB21
:10C34000B371CC663F785C62683DDE309366FBC8B3
:10C35000CC2FC8CC0D541C101C02784CBB426F76FD
:10C360005B6267A21C10101C021776A268C34E5CA9
:10C370006244D302FDDA3668F6F65BE2E21FF6337A
:10C3800078562268E201DAFE435CE2234830F02B63
:10C39000C1B0BD1C03011420050D101419DDAC083B
:10C3A0000170650E4E9C90CC67601B7A1F7ACB881B
:10C3B00059C8550E1CA020E2F9CFD91C7858492441
:10C3C000300501ECC27012C38700233BB313BB0DD1
:10C3D000549B8CE378068605BC95BC66866608018E
:10C3E000AC4359C85B785C42688859C851DE8CEB15
:10C3F00048C393011405070B80ED520000000000B4
:10C400009805160113883398140507843DF0B0068B
:10C410003C2606F9FBE6C622BC70067CF03DD04EF9
:10C4200070F8AE708C2F38EEB94AAEF0E048F9C41F
:10C4300046C10238467CA65849F0DDD4B0E622FC5D
:10C4400006023DD08A983C0A05CC98420C172E0A69
:10C45000F9FB4EB07C5CD070FCE090051601130B2C
:10C46000803D6A4CE57A040D7CF57A0B80694606BE
:10C470007038F61366663C1EE0D09C30583A1C3A81
:10C4800030E63A30C64FE63F5C50D0D0F19AE60E27
:10C49000BC427CA67CCA70BCA6F6F6F6E33A3A0E1D
:10C4A000303C1E78AE7E3A3A306A677E8E8EFE2F22
:10C4B0004A2F440B4A97BC430E98AE7A30EA830465
:10C4C000D88C1B8408D86A3F8E8E0C374A77BCFD07
:10C4D000E24AE748B19AE6C532308306CE3C56665A
:10C4E00037B85CE2E2E2313238FC9CA262CF1CA297
:10C4F0003C28352EE0DCA0DCF2C156A00EAE1C724A
:10C50000CD564EEB514CD1C8E653D144E0C4F57E34
:10C510007D6813BB664670385C5228A658BDE0BEE5
:10C52000EF983CA6BCBE580948EEEB86983C7038A4
:10C530000EC67066E6386E33EE773A6E5F300406EC
:10C54000983A7EB75826371568A30DFC0E0F2013B6
:10C5500015030820010C0DF1FE266F29E60948EEAF
:10C56000DB33D1C8E62B4670F828B8EE4670CEF023
:10C57000F1688E1C527C706944E86E754CA8987006
:10C5800038F6274E70AB98267038463C05688D709B
:10C59000CE0EDC52BC702626694468454098803D2A
:10C5A0006A84050B800172840C0612038443930194
:10C5B0000C0612038801C8E6B5A2DC908C133E6815
:10C5C000BDD00881F08CA1C34E70780666263DC2AE
:10C5D0005AEEAE3C700698F00DD0A6065870CEF01C
:10C5E00070088C6366700201D030FF8D8CA658985D
:10C5F0000E0DD0A65870B0662F704EF09B0C234ED7
:10C600006EF0C102847E1788B0FC580670BC9C4A4C
:10C610001CBCF004738C060C033EA5E8B07E7E2B98
:10C6200089F63E8C1B78EE55F2BDD07DF20DFC12E2
:10C63000050320140F0F200C0F0E07F1FE920803C4
:10C640001010018408B5E00CAFCEBC06B07C8C2F76
:10C65000A63C707C26E6CEFC0AEDD0AE7C0E980699
:10C66000CEBC4630FF063B3CAA8D8CB03C0698E61B
:10C6700071D8849803920803130E09884349EA830A
:10C680000512130E0904B5E00CA7B03C51D8CE3CFE
:10C690000E889826587C9C0A7C1C0AAE7098E6EDA1
:10C6A000D0B0AA7C0EEDA4AEFCAE8D8CAE7C0E7C20
:10C6B0006A93846262901C622751EC02AE8C2FFC5C
:10C6C0000E888B987C0AFC66588C9BB383051210ED
:10C6D00010014404B9E049D8987C0EFC2BEDA45914
:10C6E000A4AE7CAE8D8C01D098663758AEFCAE738C
:10C6F0004C6030FF8D8E8C061A1305120B807D4A1C
:10C700005ABC1A203C06B0303AE62366DF461AE0EF
:10C71000411CF53E30EFB616666F3001B670387CBE
:10C7200006562306B66666E09819050B1405070B36
:10C730008005427924B5BCC10208D8284E2E687005
:10C7400088C4651C0488ED0600000000000000009D
:10C7500000000000000000000000000000000000D9
:10C7600000000000000000000000000000000000C9
:10C7700000000000000000000000000000000000B9
:10C7800000000000000000000000000000000000A9
:10C790000000000000000000000000000000000099
:10C7A0000000000000000000000000000000000089
:10C7B0000000000000000000000000000000000079
:10C7C0000000000000000000000000000000000069
:10C7D0000000000000000000000000000000000059
:10C7E0000000000000000000000000000000000049
:10C7F0000000000000000000000000000000000039
:10C80000810F1418F8EECE7EFE595A15C89C58397F
:10C81000B69209040D052E009170A56CBDCC06469C
:10C82000BCA63CF0BDCC26BCF0883E4E5859F08CDE
:10C8300053C1B01C4E901A987C5875B0BAD33020B2
:10C84000E8B03000E6E6C67EE3E8B0DCD00EA11426
:10C850004924385E285DBC8001529CC22B387C661E
:10C860003B0D54663002C61306F5C44E708CB551AC
:10C87000EEE8D5CCA6A62FB5BCFD5AC1B0BD1C04B0
:10C88000091220050D101419DDAC080170B902DC85
:10C89000901BDCD0FE84480453DC501BDCD0FE042B
:10C8A00044848404040E30407030BF0638661B0890
:10C8B000634C537C66B5F7EE7CE6FCEEAE0E3CA610
:10C8C0003C263C0E0C7F7038AED86E1788D8AE2E42
:10C8D0006F8C1B6E582DD00CE7A6067038FCA60690
:10C8E0007C7026E63DD00C6F4C278C5F83CE7C6637
:10C8F00037FCEE4B84AE0E3C06704E6EF00C278C6F
:10C900006B8485D0C6A686A6A5D0469330EEA62613
:10C9100086065C424F9B880C2FB0BC16DEBCDEF353
:10C9200076E30DFC060C2014191005D9FE0DFC064B
:10C930000C200E0F1420060F150E04F1FE1C3040C3
:10C94000704C57AE0EBC06387CA6BCF00CA04E2E28
:10C95000BC30BFF0E09208030C0504884383051245
:10C960000C05048449F08808E9D48CF9FB8C7B4ED3
:10C970007001C898A658CEBC06B07CC6E698A6063C
:10C9800027C6DB0686A6467098C60658CEBCA6C645
:10C990003CAA8D8C98E63C0AEDD0987C83B07C460E
:10C9A000707C707CF0CEFC0AD9D0CE7CAA0E84EDCF
:10C9B000A4F0664BB0561C2A13886A1CF0AE7CAEFD
:10C9C0008D8C8C60A293A63040562B3001B6166633
:10C9D0002F70383C06A2A2A28CAFAEFCAE88338C7E
:10C9E00006121510A068A5E88EB05A580881F09874
:10C9F0006E46262642EA4E7078063DC3BDCC46BC44
:10CA0000F0AE0E3C0A3DD0BA3CE6A670A638EE70F9
:10CA1000EEF0DA3C66A084A63040562B3001B61604
:10CA2000661FA5D0668C27887B981205160113888F
:10CA30003B9812140507843DF0B0588891D0B00699
:10CA40003CC61306BCA606BCD870E63C4626832628
:10CA5000E698A658B0FCA61C223DD098EEDB9214B6
:10CA60000507843B920516011388DC90FE95E8C10A
:10CA70005C4E70783CC6A660E6B006978C730DFCE1
:10CA8000050E04200F0620060CF1FE66A6C686BC25
:10CA9000A6BCFAB0FC060DD07AB0FC70BCC626BCB1
:10CAA000F0AE7084448C57A67CA63CA6700488B374
:10CAB00008849B90011713070512484B85160F0D2C
:10CAC000070512448491D0E6136670063C063C06C6
:10CAD000B958BCB958063C0627883C70B00E3CA635
:10CAE000BCA670840404B07C7038EEB07038EEF0F0
:10CAF0004C33B07C70CEF0B03C66603C048C7F8CD4
:10CB00001B661326700C600CEF3C080C9B700E2DFE
:10CB1000D0B0A68BAE7C0EB0E622FC06023DD08AD9
:10CB2000AE0E3C0A05CE94100B050513844B811400
:10CB3000100B0505138889E84E7001C8FCFA1E7EAB
:10CB40007EB0FC70BCA6063C463C7080C15A941076
:10CB50000C031284438114100C03128889E8B03C42
:10CB6000A6F5C4CEF07C06F5C46EA05A233003C6E9
:10CB7000B01D60EEB94ABD1C20051212DDAC0801E3
:10CB800070ED8AA188C1B0BD1E492404CDB4734E96
:10CB90005C90D0D010309C6262BDC06B49A43DA4B3
:10CBA0008A3DA4E5A4581C22071CAA588CDF6AED14
:10CBB0001898EA6DCC3010701EA114D91C7E9EBE50
:10CBC000B8BEF37EBAFC8518F90E46F070B85CE288
:10CBD000E2E24660E21BAE4BAEBC067CA63CA63C45
:10CBE0005EE0000000000000000000000000000007
:10CBF000000000000000000000000004320605E80C
:10CC00000000000000000000000000000000000024
:10CC10000000000000000000000000000000000014
:10CC2000000054000000009001000000042AD08899
:10CC300022282280008051018045028001C05504D5
:10CC4000C02422006024110054005001400500243B
:10CC50000204100D2002C05000000C0C00E0344F04
:10CC6000C8834F8A4F3C372C8E20C13B08E16810A7
:10CC70000D204E064065F3B8144DBFF48308922290
:10CC80000159C91D744FCC78E4452FC2F1020054FC
:10CC9000D450C1D8C430FD3A06FE876130164E41EB
:10CCA0008660434BC43D898BBBD1D3BB031011516C
:10CCB000D100034035312DE212133131D5C172500C
:10CCC00031E04C0005D10444151E50455D4C762FD3
:10CCD00003005C000000194207C9C4004066021648
:10CCE000F6460522501012B4CD460A001900740011
:10CCF000318F4F40384454F37F2B4147888714E0ED
:10CD00004331410F3C4A349009941140314166301F
:10CD1000CD2823514ECA60CAC01F8FC2E72F080119
:10CD2000B60501C2C8105D07FC2210301100FB04DB
:10CD30002244448C738748E0C4073D03A3064AA4F9
:10CD400080C1084B31C1142013044B03D60F1B02C2
:10CD5000023D0CC1E724E20051086000800000524F
:10CD6000D147842000923374CDFD6405C1111104B4
:10CD70000004F04020800661761402C404640012AE
:10CD80000012EE450D0511A0803900102148410028
:10CD90005238B18C40225015F70500549C0B0060AE
:10CDA0000020409A25CE660040050002205D3EA985
:10CDB0002686E8B534D00C004033C14149C223A3D4
:10CDC0007463C71333CDEFD27188521027BAD2E300
:10CDD000C4B84EF9F3B5A78448F623C2BAA24521D8
:10CDE000A28D6CF63300004E32C884B83260301D1C
:10CDF0000100104CE98608B7203B2AE10E0019001B
:10CE00000008804278001A0A820280078F442200BC
:10CE1000215410E1417004001D65155D2275F3B8C1
:10CE2000E322C140244354689FA88F2F638F854B12
:10CE30008B3D1F4FBCA244C05C357A9F2B0896D413
:10CE4000C515724F45A1214505910921A130E24444
:10CE500029BD290000603C981F8E04884668819196
:10CE6000089282470BA9C55401110002008620A236
:10CE7000833C683D40964089240204500189800724
:10CE80003A8A500A640200E8C0A48C0800006000DE
:10CE900080C1612444020555582C00146001800EA5
:10CEA00000040F80996110440009001073CD003C0C
:10CEB0007D840900500011C8000049C01D000074A5
:10CEC00094D4CA63114113480DD4000051DC70980A
:10CED0001913000000000000000000000000000026
:10CEE0000000000000000000000000000000000042
:10CEF0000000000000000000000000000000000032
:10CF000000804A0C00404613912302090D54171D5E
:10CF100053B58F34215E94A01611043630C5D10C60
:10CF20000080938C20000802F01246CC800200148E
:10CF3000482734878189904020227082815389025A
:10CF400031057041D43D5124230060080000601079
:10CF50000215828F8403800080427218468451C477
:10CF60004820514800511110204241B420B02C00FB
:10CF7000F0514CD008550B3C00094048A4803E03BA
:10CF800052098180487F314103FC038000A0104298
:10CF90000451019D4400480420002800E0D43022C0
:10CFA00000008640040480620208117C1F0000001B
:10CFB0000088488851C41004C14B02824022380CBA
:10CFC0008838C693C014400854000003000C184071
:10CFD00081124404C000C0000454E0440030809337
:10CFE000CCCC4406F5BF5A318CBC41400484CC40C3
:10CFF0003708C25EF501D4080C00000000000040B4
:10D000001A24005D0B6E08060F380B670B5F02D702
:10D0100002E202EA02F306340407010002C102C878
:10D0200001790089016E0122011701350B010423EA
:10D03000040F0B440CE5056009FB00EE09410054A8
:10D04000006902D0007A007100610000850D0914AA
:10D050002018032D83322020050D09142D9410175C
:10D0600013C5DA810D0C010C0341E68D0C010C0394
:10D070001289E6930D0C01120C03C9CE00000000CA
:10D08000000000000000970F0404A140F944694823
:10D0900063C1B0981E7E3570DDAC6564983102586E
:10D0A000300370C158CE6152814084D54CF88C1346
:10D0B000B86ED330200C3330188C1326E6A18804C8
:10D0C000B17022D91CB8C6E86564ED8A389C4AE084
:10D0D0003E3E3E8A1E4E62EFCECAD47EC31E4EAA8C
:10D0E000E05830107030FBF0E8E0850D0914D96885
:10D0F0008E7C5E61446948BB6ED9708B85140104D7
:10D10000D968754C694843C1B008F548656498EE24
:10D11000B94A97130C0312514C04E5449B86010C49
:10D12000031295445B514CF8BC6944FEA0DC50E00E
:10D1300097130E1512514C68E08940A838A0FE1BC9
:10D140005C8A0E9E1EB1644E46D95C5C19688D7077
:10D15000CE0E5C7CEACED95C5C4AFA1F4E5BA00E18
:10D16000665C1BFAA642EBAE0E60E099040DB8BCFB
:10D17000D844D87CA8E0990D04B8BCD848AB0E8E32
:10D180008EA04E5C504E4E9C3E3ED05C4140603C7A
:10D19000E00408E0DCA046F098067038F6136666F6
:10D1A0003C7E60BCA6BCDC100EC1B0AE5C900E46EE
:10D1B000F03C70380C435C04F2277CA2E370D91C6D
:10D1C0008EB07C7075B06E8E5E4B5CA2A39CA2AFDD
:10D1D0007AD30CE361009CD2BB9CD2A0C1B0DC101E
:10D1E000FE04041B300B3C0E1CF86A1FBEE3B8495A
:10D1F000243E616A856869547008A968E60670383B
:10D200001CFC6A6A1E6A337E7E98A658B08148ED7F
:10D210004E6954BE3E0165DB000045DA00000000A7
:10D2200000006954F693E0DCA01CEE982670380EDE
:10D23000A0F2A65EEBA6728940387C323200003242
:10D240001F12EF662792B2939260981D68A6049809
:10D2500070CE1C42F0861E81487E98C6BE6066EB8A
:10D26000F613263C5E9E9870380C134E7098532629
:10D270007038A670A6F066A60626AFC670B0F0BEDF
:10D2800033E0300870A6DCD09C1E387C4A3CEE604F
:10D29000A6BE60A6067038BB8940387C4666E6A606
:10D2A000260E4B361CE2172AA6496870383E607E6F
:10D2B0001C128B1C42F0935C0A6029FEAB05140122
:10D2C00004D9CE93190104048DCE980D0C010C03E2
:10D2D00011E6B2310B0C03DD48449828E0B4320B60
:10D2E0000C03DD4848AB940B0C03DD48846B8414BD
:10D2F0000B0C03DD488823514CAD72754C46178EDC
:10D3000030020C6BE01CA01C50509C30057217665C
:10D31000884884DD6C0C0BDDAC4E30200EB8B8B8FC
:10D32000662F7EB86623D888D8E8492438D91C9C53
:10D330004A9EF9447E3570492659CA85683389402A
:10D340004EA8E0454A93000099CA08C1B04944007C
:10D35000B9620058894068F858A8B80E4EA07A60A3
:10D360006E1F8CA0A84E2828A82828E8E828E8A83E
:10D370002828E8A8E04970136BDD48A00E3CAA7C81
:10D38000C6A670663004062B301246BA9A4EA6BC6A
:10D3900001700EB01A9A70DAA5709A7C2B816CA07D
:10D3A0000E0E4924389C0AAE284A7C0E4E5C50D0A2
:10D3B00010101090504E5CD0905090DC4140AEBCAC
:10D3C0000E389C4ABC70BAA57070BC0E4E1CD010B2
:10D3D000903A5C49404E5C100E2BCE7A1A23AE7CFC
:10D3E00006B0A6705A0170BC30120EB0BA5A7A66F6
:10D3F00006237AA646FCDA3C5CAA7C0EDD48694628
:10D4000094030512120F034843850D0914051344B4
:10D410004E7D4070CD6C49503C2EFCBB8514010400
:10D420001405134E7E708140EEB5A258CD6C448435
:10D430004950704570380EB0284CD3492478AECE90
:10D440003010956078AE68CEF0AE5C4E138A0A302C
:10D450001095607858B075604E3004583A3024BC4E
:10D460004960709544A0EE1FA01B2D60B02560EEB2
:10D470003961216CC4F57C856813E061481CCAF9E8
:10D4800072E0AEBC0EA01C30120A334A2356134A77
:10D4900016E004E0DCA005688EB03E777E4970138C
:10D4A000730950EA0A4BAE3C0E1C12D1501B84ABE0
:10D4B000D8EE271CD2D3D54CB540EE4D704E1C5043
:10D4C000501C0A1BCD4290901C0AD36E816C4E0EEC
:10D4D0008D70CE4EFD50A0980EE09ED95C4D70131D
:10D4E00063D95C8A8A4B30030455701B616A8A8A4F
:10D4F0008A1ED95CA04E9C909C0A931C3C0A73A087
:10D500005C99704E5CA5700E0E60E00E695013EBD6
:10D51000D95CDE7098067C6627B00E2B6670C15809
:10D52000CED95CFE23A03E2B6E6D50234C670BD9E9
:10D530005CDEA05CFE138A0EB0FE138AAECE5E6F78
:10D540009E2146307A66FB61020404981D5C5AE114
:10D55000080698467CA6BC58E01C987038E09713E3
:10D56000783CE64EC67CC63CEE514CC4780ED1E207
:10D57000B1640E681CE260CE3C58B96C6100CCED21
:10D5800057080C7F44E544CCCFE05CB5708C171C89
:10D59000D85346F0987CB95844CECC37FE2BA03EE9
:10D5A0007E538C2B2D548B234970630460B1702201
:10D5B00008D91C495C638ECC4FE01C214CCCF55C37
:10D5C000A0CCCF6089406C9BF89CE27B4970CC1D5D
:10D5D00070CC4F89403031E8F9561CF8EA23A8385E
:10D5E0000E98BC62EBCCAFA2023C580CAF0844AE24
:10D5F000F544CC47214CE05C115C3B6046F03013B5
:10D60000716487138474348575358676363718824D
:10D61000C21283C37300230B36363636363636369F
:10D6200036134B237BFBFB6B53306E66FBF1568B43
:10D63000030F0C039170E5EE995ABB05D40D5449C4
:10D64000248142115AB95A855A0DD49170A56CA003
:10D65000F9CE73AB8C374C73195C061C62131C42F9
:10D6600062315D33D38940F81C0CFFEABF4EA82815
:10D670009B4C8FB570A88C1B281368580C2555F34C
:10D680008C178C1F883B842B4CD73032155CA08CB8
:10D690002FA6FB415E66134660315C315488E54C31
:10D6A000AB8C9F4C8F0C1F0813042D5404434C3734
:10D6B0008C370CCF08A55A044C1F481344989C4241
:10D6C0001C4258C3155C044C374666B64893367600
:10D6D000DF1C862233A24C47C62B629C86A24431B3
:10D6E0005C4CCF3154BB4C778940A838700C255521
:10D6F000987CB958B004F544987C70AEF0C8CC7BE7
:10D7000008488C2D55C8CC3BE01CF55C46F0983C95
:10D71000A02660F61348315C7C26BC588CE54D6130
:10D7200000987C26167616577038AE98F038AEF012
:10D73000986E4971F9560CA04C43C8CC60A060208B
:10D74000E0CCED57E006983C0CA03CE03C0C173CCC
:10D7500058E0302E0C1B303DE830128C1B3004E8B2
:10D76000195CD95C065E3E4C1B3E234C17E63030FC
:10D770007CB6163C761B301FE8E67EABE0A0C1B05D
:10D78000600C495CD95C6EE00C2B5E4BD43B5E13A5
:10D790001C4C135C2BE01CA05E0EC1B03E04885CE8
:10D7A000421B3EC3EAE0DCA07EBB830491704C4F79
:10D7B000D8C9705C422F3E33D8885E3EFED91C78B3
:10D7C00068786860E0EAA09C9A5E339A509C029068
:10D7D000DEDE1790D95C13D07EF3D0D0D0D0D0D07D
:10D7E000D0E0DCD08C7F0A9417904C276210135045
:10D7F00050DC0210CA683828380AAE28A046F0E08B
:10D800009401030D0C017D681B796666A65E3E5887
:10D81000C4440D54E0C170843D6404CDB47B758C68
:10D82000E06564E04871682B65644164E04544EB61
:10D83000B068CDB42BE5AC88138478703D64E065A6
:10D84000443B8CE5AD3D6413208C758DE020843322
:10D85000985E580D54214C492498FE2BCC6F1568C6
:10D860004330FFCC3766EB235162203C560630181C
:10D87000662D5A308766D3309366FBC8CC6100FBB7
:10D880004E9C90CCA7601B7A1F7ACBF55A894858DA
:10D89000C17085641385644B1C20E2B78C73E54C22
:10D8A000300671643470C28412C300133383533B57
:10D8B000DBBBD14413037966E168E09C83016442D9
:10D8C00049621B985E3E4962E54C2B3008716480CA
:10D8D0003482C2848712C300CB033B3B6333538B38
:10D8E00073EB1568E365203BF168E05CE17084410F
:10D8F00062F168C1B008ED48B3447168008B294EED
:10D900008568668698663315C84D68CBC658E02092
:10D9100030F1CC256366E3E0E008017201EE884156
:10D92000DE9870C4F57CB058E0000000A09C4ED09A
:10D9300090CEFBE0B87CD88C6089028D0C011A195E
:10D9400018300289407D4070514CE83888084D50AD
:10D950007C46EE173A70842689400EEE6B8899500B
:10D960002B301AF1424E360ECFAE7C466860094825
:10D97000B0300446068C1B66367066A658851406C1
:10D980009806678826260613848568238C97A188C5
:10D99000C1B0BD1C0E0F20120F0F0D38F8214286AA
:10D9A000C626704E7EF0C6704EDC90901090F0044B
:10D9B000A96858B0C6260E2568869806B05568989E
:10D9C000A658A670660638D87066D8F026ABC67022
:10D9D0002658B0F65BF04670780E98702658AEF078
:10D9E000B09C629F0948EE173AD87026D8F0BE3F27
:10D9F000A6667006388BD152982B148140CD6C2EC0
:10DA00005899501BB5A2A0DE1B8E0E70984E5E3347
:10DA10000ED164AE734E9C501090D05010D090AE8A
:10DA20000E874570380EB00E286B8606B05568C656
:10DA30007038FC1CAA0C2F0A3967134A7CF026A602
:10DA400004A568A6A6E0A6496870381C3E607E1250
:10DA5000B3E0067038F61366663C46FC0606E051F5
:10DA60004C4EF0E0DCA030C0085C905C0E13664EBB
:10DA70007078067BA60670383EAF7E62A0FC5646E4
:10DA8000EE770CA0A398496870383E6F98A658E0CE
:10DA9000894833D144E07EA060B03AE06954F69BF7
:10DAA000982670383C05688D70CE0EBC555CD91C2C
:10DAB000B83B4C604EBB514C894038339870384667
:10DAC0003C0E0430059C5A109010DCDCDCDCA0FA23
:10DAD0005A13229AF33A0C534C2BC8CCA023CCED0A
:10DAE000576627D4BA73945BFA5A5CD0905CFA46B6
:10DAF00026139423FA10C3FCAA0E60E086011405D5
:10DB000013514CE838288140EE8349701B4E5BDC92
:10DB100050AEFC1E1B261FE6EBBC89403CA8E8E08B
:10DB20004EDC5050501090E084E80444D828E8308F
:10DB300029E8E0EE514CE8380E4E70AE68A0E09750
:10DB400013140513417013339E048D501BB5A24D61
:10DB50004C98DE1BA08E28E0B432050D0914018418
:10DB6000887B850D091401843B8514010401888498
:10DB700044417013CBB87C1C50600691704C23D884
:10DB80008813D8492430260213A222D888D88C7B47
:10DB90008662271CEAEA0604E948E2B308A3068C79
:10DBA0004FC9705C4267DC906B095060AE3C0E134D
:10DBB000FA4C47DCD0A25D6C6E4BD91C9C10D0A2F5
:10DBC0007CE89CA2BB8C608C603020616C30414C46
:10DBD0001B3050616C304D6E5851B6B6A31C8C7F13
:10DBE000A25390909C5D6C6E167693D090BBA2CFA2
:10DBF000302F0C4B664C73B8D848D81B4C3BE84BC5
:10DC00000EEE0E0EEECEEE0EE0CE30046944A0E035
:10DC100081400E3001A0A65C4636616B7606138A01
:10DC200066F3E0A0A01CE0DCA04EB2CEEE4EEEE02B
:10DC3000F16804E09C23E09C08A0C1B0AE707C5E5B
:10DC40000EAD5C0C60D91CF8F8B00EED4A7E7C1A63
:10DC5000FA5AA57013150E0D0F0E141505170504AD
:10DC6000140815061209130114B01A30E83ABEE37D
:10DC7000E09806C44924B8BCF6F6F6A088E004C5CE
:10DC8000703059D866F31BC570301E0C1BCC8766EC
:10DC9000DB2308C570302DD80C1BCC1F66D3C458AD
:10DCA000A60658E030107030FBF0A838238940F801
:10DCB000D8E0AE8444BC0E30121C0A776A53A0CA66
:10DCC0000A374A881B563348234ADF0660AE3C0EAB
:10DCD000E00E4E7078EE894078A0AE8E0E68E09728
:10DCE00013100F1413514C28E060FCB07CA0EE0E12
:10DCF0001CD09050A636369C133AA2F38E76E3AE33
:10DD0000BC0EDA3CDAB0BA5A707A9A4E5C109C417A
:10DD100040AE3C0E3C5A4E1C50D010509010AEDA23
:10DD2000CEFC70B01AE05D1C0C13C88498A8150CCA
:10DD3000711EE1688CD972E0C97020E0894038A07A
:10DD40002E2E60E000000000000000000000000037
:10DD5000000000000000000000080B6CBB8CAB0E44
:10DD60004E70B89CA2A8B5708C1B585B4C43C1B0D8
:10DD700048042BA16C044484617604588940594CB2
:10DD800038580CC76C2F4C517EDBE8F8D84C4D76D8
:10DD9000D80C1F4CC34670B83CD80C738C674C57DA
:10DDA000D80C7BC97491704898A828E8381CEA57A9
:10DDB0008CA30568EA274E907BF83CFECFFEBF603F
:10DDC0003D5BCC4B3B4E36682B854044E804D8A8DD
:10DDD000288940BD6C88044408844484608940F8E4
:10DDE000D88C3BD83038E8FD7E0C27D8D57E5848F3
:10DDF0003031E8757A980670389C62CFF613666603
:10DE00003C1EA6067038AE7E1B4E23267038AEE050
:10DE1000DCA05CEE5D7AF237B2EEEE7CD37C0630AD
:10DE20005EA61C6A873C5CB27C0E4EB2EEEE521BC4
:10DE30003CD31CEE25510E917004E6C61CEA4BE063
:10DE400008F174A8E8557E3C305E6A478E8E8CBF20
:10DE5000CC87A3FE97C68C7F4C6FD844CCD3655437
:10DE6000D0F0F9700D7EC6A16C49240C37B8D844A7
:10DE7000D8A8AE6841683B8DE2F174A8E8CC9974EB
:10DE80005D1C0C330498A809B8BC5884983CA87849
:10DE900058EE091E44D5420C676554D0F09888BCF2
:10DEA000983C589974E020F97098BC584C93C1B0D4
:10DEB000BD1C14090D051220010C01120D20534543
:10DEC000441333C17098BC5846F06666FB610098F5
:10DED000DC1044E05830F1CCFF66EB2030264C2BB0
:10DEE00008FD7046CC9F66EB987E4B4C1F482B4834
:10DEF0008C979170A56C6B2020441C583C1C0A49DF
:10DF0000CA30C36A8B2E4C4544000D54654400460C
:10DF100066CC3766EB0D54411C4C5F9C985606301E
:10DF200072665F4CFBD57E8C6B480D7CCB4168BB29
:10DF300098E3970F0E0D0C01514C88C4084860857A
:10DF4000684B2315684389400EDB6631687038E6FC
:10DF5000463C0E8940F9740E630C474C3F8C271CDD
:10DF6000C217D5764C43F8D88C1B58E058AEA8E8B9
:10DF70003038E84C60E00C132049244CA7CC091F32
:10DF80008C8B91704C37D88C53C502603D5BC97443
:10DF9000F90C9170048498A82860A05D1C98CD9E0F
:10DFA00058B8EE514C6C9B385888989CC2285D1C20
:10DFB000089842A84B4D4C38580484D91C783C89A9
:10DFC00040A8FE63084E2B00E080E02E6889CE4C0E
:10DFD000EBA56C33587D6813DBDC90F091708CA757
:10DFE0006148D6F970736576817ED968C97071BA57
:10DFF000D57EE976008B93CBD3DB0003320D14CEB4
:10E000000000000000000000000000000000000010
:10E0100000000000000000000000000004000000FC
:10E0200000006C454C54434D613076314C4C8C4C67
:10E03000C1CC34CAAAF4BD031FC60F60481110003A
:10E0400066C4781400404503401794EB00D4DF28E1
:10E050001B505047BB402060CD3D3930B30FCCDC66
:10E060004B45DA6707C225523BE40D172330723364
:10E07000300173171992E4E3C4793F7D6055402461
:10E08000A348451455922000508E404ADEC7B14245
:10E090007CF45845324211EDE291008482183D62D1
:10E0A0001F2246E435C9C708060B94B8FC3838006F
:10E0B0000400020000C07503700D700EC07999CD88
:10E0C0002144688C43D910FDD3B31F8E505448713E
:10E0D000300DD21847374FA8C3E0129BC4139A489B
:10E0E00043315140140AA790161A425812250507C9
:10E0F00029C05104E961838D01501188137A71564A
:10E100000080008018642B00006242E4C615594864
:10E110001122B05884214406012921804253B16D57
:10E120004D79CC4C3C7220125843C53149500611F0
:10E1300036063D6474670E11D01311F643423C3E1F
:10E140005190798704E5501A90281C3EE16288F4CA
:10E1500054B848C554429F0C0388D434242344F255
:10E1600025D28109C71972A2320444064DC1405D0F
:10E170009C371CB6DD05353DD50E91263405A61C11
:10E18000040000000050AAAA5645851700069754BF
:10E19000CC998911501ED521961D5B33B72DF316EE
:10E1A0003E7719A53409564948885810C210C00452
:10E1B000914520A1BF00E353659537581944293E86
:10E1C000393D501CAA504A92A43442826DD5F227A0
:10E1D0007F17CE091D12C7C44521481C9311EF3388
:10E1E00052043033002134C623334E16DB03830C34
:10E1F0008040CF1708042E12308010011F0004F059
:10E20000005050605B1294719219441A681820E40F
:10E210008111732E51556463F4782414576CF98B73
:10E22000C8843851445398464100C080724C06D18E
:10E2300054587410000004BC600A0664D978675C06
:10E2400015CDD4F479B92790C444030AF5B70B006F
:10E250008419356F23B2967C84E1336A844D124968
:10E26000CD3A57333300601F288AA82014585154E0
:10E2700084469A8F868896862C26A619685C8051DB
:10E280001DA01835109015047F850914C2808618CA
:10E29000554C09EE9F488D763112ED113E24EE4328
:10E2A000DE5422D1C4DD6625291E6D36DF5C0709E8
:10E2B0005684F52F6017F2F3C92F10050EB0E40055
:10E2C000D4644280818877CE08D907773035213AE7
:10E2D0000004744025CA00C000C0003010CE99C5AB
:10E2E00070D4E03F4F1F1610D8239810837030036E
:10E2F0007F3CC745C405403EC11F34DE01F237FCF8
:10E3000065BD1FE556C86AC2BE84C0D5260232204C
:10E31000990FD365550000000000E4DBDF31D55FC5
:10E32000A54E458C539531BEF4617C1C0F553C6362
:10E33000134C7C428772483200D44B0852E8D43BDD
:10E34000858100E561462545102EA32F6192F48753
:10E35000EA0000000000D44C786C333009D95757DC
:10E360009D83357303E17F541319DF2C724270488B
:10E37000F5601CF11D6D0B1ECF01C13581952C522E
:10E3800047828002B226FC5FF03B073FBE930987BD
:10E3900012DA311F4E3030565B05853C8F46104AED
:10E3A00002FCF4B3398AD6461379D53003000088CD
:10E3B00001D5AC4BA6C5F82D15E3B97866D406DCBB
:10E3C000C4805107BE57C0500C94531B0100D56246
:10E3D00081719009D8D108CB7EC0F383013B4738C7
:10E3E00063304C4561FE89344D7D7F24CE57FBE47C
:10E3F0001D40B70D9315ABF6665D665456FC0B8851
:10E4000000F8615044FE1348260E7676B5A3D91C59
:10E4100078D88484D88C1326F046F009C886E64B59
:10E42000309EA62BA058F142CC2766EBA3D91C78CE
:10E4300058203C56069CE21B4EAB3012664761C822
:10E440006686A568E330C4064FC64ED0A646263C75
:10E45000A3E6761C4E906AC6FB303162276A13A68B
:10E4600062AA3C26048C2B08A07E60585D1C98BCD8
:10E470009CE22B0602A2E6C602A23003622F1C42D7
:10E48000136230088C270C237B0C134630555EFC3E
:10E4900006BC30E61BF61B2E03068C2FC16813C387
:10E4A000A60EA05A7C1AFAFAFAFA56233C3AFCEE67
:10E4B0001A46BC26260E55C4604C61008859C8789F
:10E4C00028B86898A859C4EA005ABC1AB0303AE68D
:10E4D0002366DF461AE0BDD065F04C2FA18002DB39
:10E4E000CC3F4E70B8584C7BCC6795A43C0A59A4DD
:10E4F000E5A4D88C1744A180FD188A8514064E70B7
:10E50000CA685878A6C6026A6DCCB05E3C062B5D20
:10E51000C4C830DA7004B07C0E01D0EDA4AE3C6605
:10E520007F7098AE59A48D8CAE7C6606FC5843046F
:10E53000987C1666C3084E70980E78061BA66878FD
:10E540000E59A430C08D8C4DA4468D8C4E587078D9
:10E550000E4C23C4BD8C783C667BEDA4D884D88D4A
:10E560008C29A429A4AE0E584E70780EB8BC5884DD
:10E57000E0DCA0DC1050121C8AE5A43C5CF2CB7EEF
:10E580000F02FF1C8A4DA4EDA47C6A22D398AA69CD
:10E590008C0A588C574DA459A4468D8C980A29A4EE
:10E5A0001B1C6AF5A89B623C5888821B59A4468DA7
:10E5B0008C42D762101C021F023BA666700A4EF006
:10E5C00098AA698C7038989C50F09806467078A686
:10E5D000682E063B6670EEF0EECB4924F85A5EE8F2
:10E5E00030BF2684A80E78AE66CB70380E4670AE6B
:10E5F0003E8B1C8C137CEA330EFDBC95BCB88C1F83
:10E60000884B781C0A29A429A4B8AAA8A1801C397F
:10E6100088E68F0C2F59C4F0000DFC03080B13156E
:10E620000DD9FED5883E434670AA680A4DA4E5A4DC
:10E63000AA704670785816468386FDBCEE4B66B8C5
:10E64000FCEE0825AC1B95BC780EE3D1486E2B5927
:10E65000C42E1659C41916D1486ECFA3D1489D486F
:10E66000FE738BD1486E4BBBD1486E439D48FE2351
:10E67000FBD148CB4E3E304C0EB87E5B81C806784D
:10E680003C06B9586E63AE6E7F3A3A3A3A3C7038FF
:10E690000E8E844E70F8E030546E9B305A6E736666
:10E6A0006E53666E33B5A20EA04E3E7EC37E7EA034
:10E6B0007ECE7E574E43EEA0663346F6A0BEE04EB9
:10E6C0005EE76EE0CE7E1B5EE0E0DCA0DC5EEE1F6F
:10E6D000237CF2F3AE5EEE1F237CF2F30E03E0A583
:10E6E000CCBC0E4670AE6881F04E70789A66AE680B
:10E6F000304070AEF03E55F04E7084B07E7E7E2F7E
:10E700007E89F68801C8E6B5A286B0668DC61C066D
:10E71000A54FC678A6063DC358B0FC06707C26E619
:10E72000F002223DD0AED8E63C7006023DD0B0E605
:10E730000CC38604304006A5D00C49D1C676431CD4
:10E740000A6AA5D049D066B0E6C67038A670A6F0B1
:10E75000986666776651ECA606704EF09866BF8D97
:10E76000C68451EC8C276688D326E67022FC06020C
:10E770003DD0A658B026E6FC063DD098BCA6588CE5
:10E78000A3BA44DDD47AFA9A983C0698767FA60616
:10E79000BF0DFC060C2013091A05D9FEA5D00C9755
:10E7A00098762BA5D00C5F98E63CA6B0FC707CF068
:10E7B0005DC40A3EE6B006A63CA60667BC704E7075
:10E7C000F8FE2F66A6067038EE472DD0983C66AF4F
:10E7D000BB0000000000000000000000000000007E
:10E7E0000000000000000000000000000000000029
:10E7F0000000000000000000000000000000000019
:10E800009CC2FFCC574626FBCC2F5DC4243C71CC68
:10E810006653309066FBC8CC6100839C4262E2A5DF
:10E82000684E9C90CC5F601B7A1F7ACB5DC4E01071
:10E8300071CC664FA5689C228859C87BA568D91CF5
:10E8400078583012662761C8CB30C266AF46F08C6C
:10E850005B59C8BDCC66E627652073BCF05DC42952
:10E860003C26662F8865C82B49F08804E9D48C2B98
:10E870005DC47E3E4E70088C2B4540061BF9C430AB
:10E8800018A6C6B07CEEBCA686A6061F04A666988F
:10E890003CC658B03C0671D84E70B87CD8040C13F6
:10E8A00008D8BCA898668DC77C0EEDA4E601D0AE52
:10E8B0003C58C69C584E7051B41C53BDD0C1D85E54
:10E8C0003E2DE0DDFCB1C0BDD04C1BE9D071F0B0F5
:10E8D000FC700602385AF051FCAAAE3C58C9C099E7
:10E8E000C0980A01D098AA0A5841C480E68741C45A
:10E8F0004C5780E6AB708D8C987C0EB004D88C138E
:10E9000008D826CABFAE3C580AB066577001D0413D
:10E91000C4808D8CAB0C2341C4804B081304980A2F
:10E9200030FF8D8CA156C1D8BDD04CD9C85E7E7E3B
:10E93000FE39E098EEB5F604DCD01EB07E7E2F08DE
:10E940007E29E331F40C533E85E0B05E3E7095F0D5
:10E9500059C0B0CE46CE6E6E68BDD071F04E7078A4
:10E9600058B0FC060201D0EDA48A0456705C0A0679
:10E9700076265766D88C1B086AD86A6A98AACAE7AE
:10E98000AA581C4699C4B0A1C46AB0664F7001D0A1
:10E99000EDA4A1C4B30C7B46A1C45B0830FF99C4AD
:10E9A000640530FFA1C469D095DC0C554AF9FA38EA
:10E9B000BCA6BC288804E9D48C434E30913CEEE9D7
:10E9C0005ACEBC06B07CC698BC1ABCEE4E70385C01
:10E9D000AA581C06BC065F3C0EEDA459A4E6AEBCCA
:10E9E0000EEDA4AE5884C61C6A17881C987C66E697
:10E9F0001F8CAF8CFBFC580A01D098AABCDBE156F7
:10EA00003BB03C263C463C7098E63C0AEDD02E8458
:10EA100049D463BC6658CEFC0A01D0B07C263C7059
:10EA2000983CAA7C5806D3B0FC707CF05DC45E3F75
:10EA30007E2F06ABF0837E7E89F788480DD4CE58B2
:10EA40004E70F80E8C2BEEC3F9FA3DD00698BC063A
:10EA50007F0DFC050E04200F0620120503F1FE6653
:10EA6000B03C065DD8554AA5CC06BCA63CF081F06A
:10EA7000D5CC663002C61306F5C459C42E12000068
:10EA80000000000000000000000000000000000086
:10EA90000000000000000000000000000000000076
:10EAA0000000000000000000000000000000000066
:10EAB0000000000000000000000000000000000056
:10EAC0000000000000000000000000000000000046
:10EAD0000000000000000000000000000000000036
:10EAE0000000000000000000000000000000000026
:10EAF0000000000000000000000000000000000016
:10EB00000000000000000000000000000000000005
:10EB100000000000000000000000000000000000F5
:10EB200000000000000000000000000000000000E5
:10EB300000000000000000000000000000000000D5
:10EB400000000000000000000000000000000000C5
:10EB500000000000000000000000000000000000B5
:10EB600000000000000000000000000000000000A5
:10EB70000000000000000000000000000000000095
:10EB80000000000000000000000000000000000085
:10EB90000000000000000000000000000000000075
:10EBA0000000000000000000000000000000000065
:10EBB0000000000000000000000000000000000055
:10EBC0000000000000000000000000000000000045
:10EBD0000000000000000000000000000000000035
:10EBE0000000000000000000000000000000000025
:10EBF0000000000000000000000000000000000015
:10EC000081C8E6B5A2064540B9CCA6BCA63CF048F2
:10EC100085F08C5BB0FC2670381CEE77709BD5CCF1
:10EC2000A04E70EE59C4EA003CEAF30E4E70AE6896
:10EC3000B01E4E3E1CBEBE33501050903B10BE2B3B
:10EC400010105003BE2B5050D0D3B046FC06F5C474
:10EC5000A3F85E5AE8A878E630C0062663A60670D8
:10EC6000383E334E7EF066A3A1803CD5883E7B7053
:10EC7000AE0E584DA459A4468D8C980EB0E66F7018
:10EC80005DC414218A4E6E56DC90688DB8BC08981D
:10EC90003C28441C6A8AEDA45606303A067B303084
:10ECA00006AF3020469C58DD201C6A4E30056A5B5A
:10ECB00059A46A4C8FEB48783A87783A8DC7B83CAC
:10ECC000D808D87CA88CB5515DC4333B3045663F2D
:10ECD000783A27301B83302B66832666378C7F304B
:10ECE0001A23266627301CD32666678C9F4C435315
:10ECF000F8EECE71C8700439D006B0BCA6700839E1
:10ED0000D0E6172606B0BCA670783C06B03C063CA0
:10ED100006B958BCB95826703C063CE64EA670A60B
:10ED2000F0B02606C78DC60E66176629C6BC069CBF
:10ED3000E2D330901C02AB30316A8B30460217664A
:10ED40009C024B501C62276A136AA6A606C6E6A25E
:10ED5000065E233008465DC46A27F9C40C2F70157F
:10ED6000C8E68DC606F8FEB0C6FB46DE1BA6C6A6E4
:10ED70007079C4AA58B0665F701C980AEDA49C58BC
:10ED8000461C8D8C51B47B4E1C10CC2F6EEB4E4B21
:10ED9000203C56069CE21B4E5330C4064FC64ED054
:10EDA000A646263CA3E6761C4E906AC6FB3031622E
:10EDB000276A13A662AA3C26EE61005DC42E1230BB
:10EDC000FF06F8BC66470EB8A6AEA88DC6B8BC66EE
:10EDD000B5A3840895D0302B06B006273C061B81CE
:10EDE0000A06B8BC13EEA6F30EB03CE630A8AEEEB1
:10EDF000176668A69C583508B0063C260677BC7096
:10EE0000783BF87EFE5F5C10EEAB1C7CEAF33C3393
:10EE100015C83C9C4A7079C40C2F8AB058EDA4AE3A
:10EE2000D87C1C846A1788D8AE987CEA1F8CBF4EA9
:10EE300030051C6A538C2F6A59A40359A4034E70E1
:10EE400030913CEE3B79C46DCCF5C459C4EA00BDA9
:10EE5000E0DC101E46FCBE77E6A670066638EE7053
:10EE600066EEF0BEAB5DC4EE00307A66FB61027800
:10EE7000E8380E38D81CAA28E09CA01C380EF8AA46
:10EE80007CE8AE7C280EE0D4948DC7A0EA73E267DC
:10EE90009846AE283B48084EDDE04E300BAAA0FA5B
:10EEA00060E6133AA6CB3C30030E51C45DC42E126B
:10EEB000B87CD83C30300693302E66370C60A6A65E
:10EEC000E0300D664F302D06E0303A066061DAB171
:10EED000D0AE0E3CEECEFCEA6DCC666686664E3059
:10EEE00007A63AC6F346703CEEBCC66804044CE183
:10EEF000C4E9D00881F08C4BB07EFEA1C3A1F4839D
:10EF00004E70780666263DC2EE4E9CCA1C3E70AE20
:10EF10003C06027098F00DD0A60670B0F07A4670EC
:10EF2000CEAA7C0EE5A4E6AEBC0E01D0C68D8CB098
:10EF3000A626A67A2770AE5B7001D0B08D8C0DD05E
:10EF4000A6704E6EF05DC4F000492438FC7006389F
:10EF5000FCA67C70E04670387CAA0A3C28E00404D9
:10EF600084E9D4983C1C0A0451FC4A2A2AE0306007
:10EF70000698467004261C7C4A300AFC58B8A6A89D
:10EF8000E0D91C78D8E0EDA40616D91C303A6643C7
:10EF9000302C6623302E6661DAE0B1D08E0441A4B5
:10EFA00044CE0637662FA20217484ECA686A054645
:10EFB0000000000000000000000000000000000051
:10EFC0000000000000000000000000000000000041
:10EFD0000000000000000000000000000000000031
:10EFE0000000000000000000000000000000000021
:10EFF0000000000000000000000000000000000011
:10F0000088DCD0FE95E84E705C380AB0AA2845D856
:10F010001388D91C78468C1326F0256C88080404C4
:10F02000E9D40C5B44DDD4CE7C06463BA6265DD8F5
:10F03000705B7C0A556CB03C46BC70C57E256C0488
:10F040004670387C1C0AEDA4563CAA7CEE3BCEFCF4
:10F050001C0A556CDABC06B07C063B86BC065DD843
:10F0600070DA7CE6917AAE4670CE68C1B0E0B07CD2
:10F0700006300B0697300D46DA7C06333017C63E55
:10F080009306301806BBB03C061EA114F87E7E9E87
:10F09000066646F098A6581CB07C26E6CE7C0A048C
:10F0A000EDD098E67CAAFC58CE7C0AEDD098AA5800
:10F0B000CE7C0AD9D0DC101E9E9E1C98AA5804084B
:10F0C00093EDA48A06D91C79B01CCCE746F06A01FE
:10F0D000D0987C6A6F98DE586A8744D91C987E2F36
:10F0E000581EA9763020E805768A48196C4479B014
:10F0F00098DE1EFCDC901E1F5E1BBE5E3C5883ED3E
:10F10000A48A06D91CCC33D9B008357679B01C6AEC
:10F1100046F001D0986A63DE3FFCFE9B0C8BFEDE5E
:10F1200004F3D91C0CE37E9EBEC7F8BEF3A3D91C22
:10F13000B8F8568A063040C64B46F06A196C1B79FF
:10F14000B0980C37FC1E9E3C1E3C9CE2042030F024
:10F15000E6E09CA0443020CC697766E3C666797708
:10F16000E699C8D91C9C6282B8A2F34C1B98F3069E
:10F17000E094339C98A60658A0D88444D84C77C60F
:10F18000A69C58301F6617260698069CE8D09C025D
:10F1900082B8A2F34C5177485576203CF64BA568CF
:10F1A000711C5DC4E01078581A7A7A4E203C5A1CC3
:10F1B0005D001AE000105B504B903BF3D023000041
:10F1C000103C56063044668F788C1B84138884D894
:10F1D000F0A5680C6973517626669FB07C06668C34
:10F1E00023300B4686BC0646F05DD8C97A26667782
:10F1F000B07C0646268C1B300CC653064349247847
:10F20000FC5CEAEE9C300842A17CF6DD7B30088C89
:10F210001F4200957C068C47C1681BC17A7C5898B8
:10F22000A6588CBB796C4A57C1B0BD1C0E0F20127A
:10F230000F0F0DDDAC78D884D8F049246D586100EB
:10F2400030FF66675ACCE3203C0630C366DD7A693E
:10F250007288489806C96C25E8E3CEBC06B07C6687
:10F260002326E6CEFC1C0A04EDD0988D8C0666861B
:10F27000B03C0671D8C97A3008957CE6EFDABC0656
:10F280001C3001667FE6CEFC0AEDD030608D8CB07C
:10F290003C9D7EB07C667766C6E6A658BC065DD807
:10F2A0007C26E633C626E6A658CEFC0A04EDD098A6
:10F2B0003CAA7C58066611F4D3F6278C557B1C06B5
:10F2C000300825400E7E9B9A0507088700D36B3BCC
:10F2D000E3FBEBD323DBB17E75F44670387C0AED9B
:10F2E000A4567626A3617E056C8C1B8413883D761C
:10F2F0006520056C8498F0A568F572796C0AA17B8D
:10F30000B96CB0684829E84670787083BB843BFBD1
:10F31000796C0A5788CEFC0AD9D0B03C26BC70ED77
:10F32000A456768CEBE6556CC6263FAA7C5CCAEEEA
:10F3300083B96CB0FC5CEAC41C59E8056C8498F095
:10F3400046F01B056C8C1B84138898F0C97AB03C7E
:10F35000E6C17A6606265DD8056C8498F0A56869D2
:10F3600072267F556CB03C06265DD80B4666E68853
:10F3700059C804C1B0BD1C07140F201E7E7EC63CB8
:10F3800030033E1B30017EFCE8BEB3DDAC0C3B46D7
:10F39000F0C6E10803A5684E5C10901ACC4F26EB2E
:10F3A00099C8BACB7976300B01ECC3847434857577
:10F3B00035867636370023363636363636363636A6
:10F3C0005B65209300000000E080E006C61C224739
:10F3D0001C8622279C860882CD7EC61C222B1C22DE
:10F3E000DD7B02A29F8C174230555EFC06BC30E0EC
:10F3F000000005CAF3EBE3DBD3CBC303180D14679E
:10F40000308AA630BD8B72201165E34F0B1D10238F
:10F4100050C604A89C60C74C81496A521BF515F37D
:10F4200014124485B60825C6205B15EBA2262A0ACD
:10F43000400C50AD3C362203820F003532388184B7
:10F44000D80400CCC040819010038074D184F5B002
:10F450004DC000A409302333CC5068BB881F88FB03
:10F460000D8C8C84D4CC0035C0A803033C3181863C
:10F4700021F25B38338A1CC3A1362321B22485E8EC
:10F480002ECD8843480C08000638622380C71082BE
:10F49000B02066CDC040FD657EFDF5E6D61831D1C1
:10F4A00018C0A82221727CBCEF43E2F030E363BBBA
:10F4B000EF0C2320EC20ECFF10A2A0802122282AB0
:10F4C0008221C0C3953C412282101102821108CCD6
:10F4D00004002088310089FD0CCF0B1042084991AF
:10F4E0009D3055C3080018E00D7800880350F08166
:10F4F00034242AF102000000000000000000000097
:10F50000C9E0331053FE72482113E20331158A35E6
:10F510001D23C6B0CB28320EF88A423203980C4025
:10F52000102131411204B81BCE392500C520F0044A
:10F5300052D9C408182044D915449146A603153D54
:10F540006D50210009076954011693A150421A4ACF
:10F550001B050452C7AC8EA0418010409A4F5D112C
:10F56000040481004227644114441785A2244348BF
:10F5700061542468441EC98009CD33A1DC50106A4F
:10F58000821041C1B30601194525880333D6404393
:10F59000482331E50800000610D014294304310047
:10F5A000000000000000000000000000000000005B
:10F5B000000000000000000000000000000000004B
:10F5C000000000000000000000000000000000003B
:10F5D000000000000000000000000000000000002B
:10F5E000000000000000000000000000000000001B
:10F5F000000000000000000000000000000000000B
:10F600002134432432A02C3222037A488414111767
:10F61000C54108160E3BD19008DA2308D40C50B827
:10F620000320AAC428201417170E003183AAAE7332
:10F630007F3703F17A18EB40E8C42EE340E044E062
:10F6400088114C2046211420D24F22D41E7F7C8C5E
:10F650003FCF143D4D34004238019D1008E1503237
:10F660000030344E4207C404A89C60C74C81C84097
:10F6700045D3F0D0801231CC44D401412433841BD3
:10F680008E32F62E61200609FD73B40CC10CF38C8A
:10F690002108C44098186081620F848B9EC008279F
:10F6A00008C70FEEC5174060865D2403B731315C93
:10F6B000C744C7CB50005044642384930C32E88C79
:10F6C000683D00088509240A6002040084C0000027
:10F6D000880E841800A3512E4891801E8508048945
:10F6E0004F2F313131B13C1432C3085200000000B9
:10F6F000000000000000000000000000000000000A
:10F700000B801A2838215A84720934015C0504954B
:10F710006824000054180D059034E248C5443411A3
:10F72000140F3113C411249811405844587841C41F
:10F73000084D700CC447E3244571A11991368087A8
:10F74000D0CC54010C8D2B033B0371330F45304655
:10F7500034D6061D20F4E668C8003744C8516C4B07
:10F760004C8C214BDD14E55131D0141E6300C000D8
:10F770004931CDEC56540E954414C339144A34879C
:10F78000064767C5C435C67D44753300E0B41B2306
:10F790002DBC141F595580D10A901110105C9C612A
:10F7A000C4004500148D4105090941465124C9444E
:10F7B0007155591055508296A0968978626E514DB8
:10F7C00085094A4DF5430186E051080816C68CB1FB
:10F7D0009C01B0079E01E6167941C088F20C200515
:10F7E00021A1F70C331654E3D21600000090AAAA08
:10F7F000884077282F3FC5A2474B85F630FF3F88CA
:10F8000000000000010000000200000003000100F1
:10F8100005000100050101000800020109000201C4
:10F82000090102010A0000020B0000030C000004A1
:10F830000D0000050E0000060F0000060A0000077C
:10F840000B0000080C000009584E55543020005899
:10F850004E5554312000584E5554322000435846DE
:10F86000554E300054494D45522000435846554EA0
:10F8700031004164764C31200041647655312000DE
:10F88000416476553220004D6174683144005374F0
:10F89000617431420046696E616E63005A656E7232
:10F8A0006F6D005050434C20520050504355205231
:10F8B00000436972637569005374616E6461004747
:06F8C000616D657331006B
:10F8C600414C504841005052474D00534849465418
:10F8D60000524144005553455200444547001A1B07
:10F8E6001B1B1B1B1B1B1B1B1B1B1B1B1B1B1B1B62
:10F8F6001B1B1B1B1B1B1B1B1B1B1B1B19007C2009
:10F906004275696C742062793A204D652120202069
:10F916002020202020202020202020207C007C2049
:10F92600496620666F756E643A20696E666F407030
:10F93600617865722E6E6574202020207C00171B6E
:10F946001B1B1B1B1B1B1B1B1B1B1B1B1B1B1B1B01
:10F956001B1B1B1B1B1B1B1B1B1B1B1B18004255AE
:10F96600494C543A204665622031302032303235D7
:10F976002031303A35353A3030005645523A20304B
:10F986002E393034004A414E00464542004D415220
:10F9960000415052004D4159004A554E004A554CBF
:10F9A6000041554700534550004F4354004E4F56B3
:10F9B600004445430053554E004D4F4E00545545A7
:10F9C6000057454400544855004652490053415497
:10F9D600004D454E552000444953502000424545B0
:10F9E600502000434F4D20200053504545440049C8
:10F9F6004E464F2000534C4545500056494557202A
:10FA0600004D4F52452000524547532000464C4179
:10FA16004753004D4F445320004144562020005286
:10FA26004F4D532000434F4E462000532E494D471D
:10FA36000052414D20200050524F47200053495A52
:10FA4600453A0052414D204D6400202D2D2D2D208C
:10FA5600002D20202D20202D00726573746F726991
:10FA66006E672E2E2E0052756E20204379636C65CC
:10FA7600733A0044697370204379636C65733A0086
:10FA86004B657920204379636C65733A004465625F
:10FA96006F756E636520542E3A00426174742E2091
:10FAA600456D7074793A0050582D34314358004EE4
:10FAB600414D452020506720426B2047700042414F
:10FAC600543A00534E3A00020C010E0B00444953BF
:10FAD600500A00454F460A0057616974696E6720EF
:10FAE600666F7220646174612E2E2E0A004F4B0AD7
:10FAF60000505834310A0052414D0A004552524FC7
:10FB0600520A0044495350004245455000434F4D68
:10FB160000535045454400494E464F005649455707
:10FB2600004D4F524500534C4545500052544E002F
:10FB3600455849540044554D50004C4F4144000926
:10FB4600204F4E0009204F464600384D485A003196
:10FB5600364D485A0032344D485A0033324D485AD1
:10FB660000314D494E00324D494E00344D494E004C
:10FB76004E455645520058595A5400584100585956
:10FB86000058005245475300464C414753004E45E6
:10FB960058540050524556004D4F445300502E3095
:10FBA6002D3700502E382D46004144560055500042
:10FBB600444F574E00494E430044454300005447C6
:10FBC6004C00524F4D530041444400454A4543546E
:10FBD60000434F4E4600532E494D47004F4E004FAF
:10FBE60046460052455345540052414D0045784D16
:10FBF600454D0052616D4D640050524F4700314CE7
:10FC0600494E4500344C494E45003120534543008A
:06FC1600322053454300BB
:020000021000EC
:100000001640008F00A60299009E026600950247E6
:1000100003370309031E032602EC02F90451052FDE
:100020000557056A0577050C059104800485048A47
:10003000048F05B104630456045C046A047705A5C3
:10004000059A05D205A005C204E70504051204BE01
:1000500004C904A904DF04D004D7051604B0049E23
:10006000049704B704EF05CA054605290522054F84
:10007000056405710583058A05BA05360608066319
:1000800003B400008220160E0F03201604012DE099
:100090008E091805084830088B8E0914030F300F9D
:1000A000438E090E0902300244E6B83C5804CC1FC6
:1000B0008C2BC4840C5F04C1B0301F682668C668EE
:1000C0001E2B6520610049244E00309D3CFA7EB80D
:1000D0003C98FC6D1C3C587EFA7A6F605B0C2F08D4
:1000E0006B0B133C7A17FCCC8B0C67793C2E3812C7
:1000F000C6C3837711C08070301084743485753521
:100100008676363700E3E323DB53B300C3666666C7
:100110006666666666666666666666661B693CACAB
:100120004CE733FB300A06B34CA7DB5E23793CDE99
:100130002146A3B87CD84C1B441348D83CA8A34CF8
:10014000EF8B4C1B446B485B5E2F6100410EE0D986
:100150001CB8E6F8302006A8B8B856A66617B8A6A8
:10016000E826E8C6E8BE5E2B6D8CDF005D1C3C58BF
:10017000200BE066D91CB8569C5806E223E2E20642
:10018000A2263B66F8693C2403DC904C1B7E7E066D
:100190007E9BFEB806B8300A664623302F0626E856
:1001A0007E3E23C666E8E6E89C98E8EB5E6BD91CC9
:1001B000B8E63020E86606B8B8B8566613F866A602
:1001C000E8E6E84924793CC8B01A5A300CBC1A70E9
:1001D0008DBCF10E8498A8793CDE5D1C1106E0D937
:1001E0001C0EB89CE2337E7E4C137E7E302FE81CC2
:1001F00022A6F8B0E21B62DFA0FCCAF61F226656F8
:100200005ABCBADEFA7EF35AF8B0E2736263601E3B
:100210003009065C422FFAA6E30E6EC1B04924B83D
:100220003CD808D87CA8208CB55188EEE8E04E2058
:100230003C063018BC1AB0303AE62366DF061AE0F6
:1002400097050916180508F8AE6D8CDF8C3008008C
:10025000E66D8CDF3A5C005AD070088DBCF10E97C9
:1002600005091614030FF8AE6D8CDF8CAE0E9C00E2
:10027000E21B8902DCE2E7E2D7E05CA01C4EA202AE
:10028000E2EEEEEE3CBAF2BAA2DCD493300FE669AD
:100290003C51970509160E0902F8AE6D8CDF8C4EA5
:1002A00000BA1A3CFA1B8902E6EFE6DFE05CA01C0C
:1002B000BAF2F2F2BA42421322A2DCD4A33002E62E
:1002C000693C51B8AE6D8CDF8CAE00F06D8CDFE711
:1002D000A600F0EE3004EE465BCE1C58DC9886C3D8
:1002E000EE66F3BC463CE09918140F12793CC370DB
:1002F000793C43B0CBBF140902793CC33CD88C276E
:10030000D8B95AD8655A840E01793C43B0BC463CF2
:10031000BA6D8CDF6C6E008C9102A902920F793C51
:1003200043705B920F18793C4358AEB0D8AEAEB074
:10033000AED870D3940F0EF888AE6D8CDF8CBA00F7
:10034000BA005BF88458B8AE6D8CDF8CAE00D8AEC6
:100350006D8CDF8CD800E00B00A188C1B080B0307C
:10036000063000E6465D003CA6BC300656A87A562C
:10037000D3492408000170ED8A0B00C1020B00B9BB
:100380004A0B0089520B00B5A20B0089020B001921
:100390005A0B00810A0B0009828814010D201604F3
:1003A000012DE08D1614201604012DE00B00A1880C
:1003B00080E00440CC00F3004D50A631F27F3A6952
:1003C000111B1342A631F27F3D85C2032F0270C676
:1003D00000F600534952544EA605C8012F0470C6BA
:1003E00000F400535A3FF653495A453E3DA631A802
:1003F0001997738B9BF37585C8032F0000000000CD
:10040000050E04200F062001121201190E0F1420F0
:10041000011212011920060C0E010D052005121201
:100420000F120E0F20120F0F0D04090D20051212CE
:100430000F120E0F20182D0D050D0F1219150E0499
:1004400005062001121201199812140D201604013C
:100450002DE0AB14010D4EABAD14010D308073AA2D
:1004600014010D30203BAF14010D30A0D8793CD9D8
:10047000038D090414010DF86150753CD6CFAB090A
:100480003016F3AD093056CBAB0A3036A3AD0A3087
:10049000767B810A09130D30053B8A09130D301153
:1004A00058F86150EB8A09120D3013ABAB03130DF2
:1004B000301273AB12130D30323BAB03120D30927E
:1004C00058753CD606AD03120D30D2ABAB12120DEF
:1004D00030B273AD12120D30F23B810A09120D30A9
:1004E00007FB85160F0D0DC4483B900117130DC473
:1004F0008808F86150B80E785150753CD697BF0502
:100500000D010E0D793CDF22BF0D0904793CD62286
:10051000920DC433930DC4608848793CDFD0BF127C
:100520003E12C448C3923E3C12C493833E3C03C473
:10053000085B832B0319B86150C40888F8615075B3
:100540003CE5CE96091008048B820118010D1204B7
:1005500043820118010D030808844884F86150EBB8
:100560008D120E1204338D120E0308846B8D151339
:100570001204338D1513030888448404753CDFF19D
:100580008D1513883B82010D151384843B8D120E4B
:1005900006888844A3820118010D84845B8E090DAE
:1005A000882B98010D8488480804793CDF428D2A05
:1005B0000D793CE56793100E1214793CDF49960ED5
:1005C000090D793CE5259319130D793CE5EA94056D
:1005D000040D793CE58EB030CBB030F6F6366BB01A
:1005E00030F636F63BB030F636F636F61336F613FE
:1005F000363A70DADADA3ABC80E000000000000037
:100600000000000000000D50CA00F6004D454449AE
:1006100054A81B10A5AFCF66A90AA819A5AEAB199F
:10062000B6B2018BA5A8AC0AB6AA87A5BFA5A59BA3
:1006300073AC08B997F27F3FA9178EA5A57179A56C
:10064000AC9A73AC17A5AC0AA596B12A09A8157E79
:10065000BA0BCF6F06AC071DF34D5452A5A4C40CC2
:100660002F1F10C401F700434D45444954A81B07F0
:10067000A906A59283F74E4F542043505868124B59
:10068000638E75691A10101245A806AC06B1874B27
:1006900067B1838EB72701A90A73CF661242111A78
:1006A00010101141A819A5AEAB19D07D8F02AC0A6C
:1006B000D0778FE06683F352452EA5BFA5A59B7327
:1006C000AC08B994F27F3F8EA5ACAC06B98AA5966A
:1006D000A594A5ACA597A59509A815AC087EE03B07
:1006E00083F3494D2EA5BFA594A5A59B73AC08BA6D
:1006F00091F27F3F8EA5B0AC06BB8FA59554A5ADFA
:10070000BB880A7EA596AC06B25D0BAC0AD01A8FE8
:10071000AD06A596AD09A595B26D04A5A8111A1050
:10072000101140124385CF6FCF0FAC071DF34D540E
:1007300052A5A4CA1D2F2150CA00F6004D415452A3
:100740005801A902A81BF5524C2043588ECF68CF00
:1007500069CF6AB114CF67A802CF66F74F524445FC
:10076000523D3F8E616883AC024030511140A6215A
:10077000AB198E2083F152111B1C134240A59DC260
:100780000AF4004D5452CF6F02A908A907A815A872
:100790001BFC2041204920445420422053458EB266
:1007A0001904F152A5A0F44445543D9B737EB22830
:1007B000CF7BA808CF66F152BFB9CF67F152A5A28F
:1007C000B23ACF68AD02B4279F00B244CF6AE02DA1
:1007D000829A73F2522C9B73A5B2B254CF7CF15221
:1007E000AC029F00AD02A5BBB262CF7EA808CF6964
:1007F000E00B820FA807AC02A5BEA5BD03F152A570
:10080000926883511140A63175A819A59DAA198532
:1008100074401140A6218ED0926FC2162F3D30C079
:1008200001F4005A5E4E8030754F205371204271A2
:10083000054E01AC0485A815F2553D9B737EF2561A
:100840003D9B727E85C605F5004D41475A4FA81560
:10085000F2523D9B73AD047E85CC02F400655E5A76
:1008600081554E80B134CC01F4004C4E5A814F502A
:1008700080B141CC01F6005A5E312F4E8030131604
:1008800010714331754F20686053712068437104C3
:10089000E061049700B28185024F71214071B4116B
:1008A000C606F50053494E5A81325A7133E04C8ADC
:1008B00042225923E0518B4280B100CC03F5004322
:1008C0004F535A8132597133E0318A4254225A23AC
:1008D000E0358B4280B100C004F50054414E5A818E
:1008E0001242325A71124233E01D8B4023E00C8ACF
:1008F0007143762259714380B1000B83835871553F
:1009000043715840BD850C558360400D124385C02E
:1009100008F400615E5A7532717450427622421DAD
:10092000F3655E5AC003F5004C4F475A5034758149
:100930004F5024957195727580B100C403F6005A2A
:100940005E312F57327533753151713051402071FE
:100950004354762171432322C204F4005A5E578126
:100960004F504F75754F7175427540744E554E809E
:10097000B100CA03F300432B71067540754074B192
:1009800000C202F300432D547154B613C801F500A0
:1009900043494E56E00482B100034F607154714EDA
:1009A00085C003F300432A4F75754F757571754205
:1009B0007540744EB100C003F300432FE024021DC4
:1009C000F2432ACC012F5B70C600F400504C591240
:1009D00013A621AB198ECF6AF84445475245453DD1
:1009E0003F8E1245D00F6A71121146D0166A71A857
:1009F00000A903A905A9069116911506E04B8C974D
:100A000015B608E0448CCF6FA815A81BFC465820EB
:100A10005254202020204E45578ED0156FCF66A906
:100A200006901691157183838397159096AC059562
:100A30007342E1E18E9073909642AD0571F4463CAD
:100A4000583EE18B8FD0406F0DF1619015A631F3C8
:100A50007F3D3F778E919585CF67A619D0576FC898
:100A600015F40052545312141A11AC069117AC0528
:100A7000BB9390161141911590960C95959715BCC6
:100A8000079500A8050B2036213722382339243A50
:100A90009016121040A819AE73F34E3E358E85CFD6
:100AA0001911101A10101691149115E12E902DE0C5
:100AB000DC842A11E17191E16E91E16B91E1689121
:100AC000CF18289112543827911129911342269159
:100AD0001014424137901214429013514190104229
:100AE0009011514136A900E06397AA038503AA0239
:100AF000B1882D29453D2D2A453D0190133C129585
:100B00000C950D2D51901041661000111B1C1845BD
:100B1000E0358675523F2C2D4290111243416711EA
:100B20008361433E2C519012412D12424052940E4B
:100B3000A800E00287082C2E543E40372D2F543F4A
:100B40004036E02796850771777185CF17181A1000
:100B5000101691149115E08390AC03852DAC00E044
:100B60002C842811E0C191E0BE91CF162754124386
:100B7000838351264166B1A2524039AC00E00E8415
:100B80007476413AAC00E00584A9028505F4524F21
:100B90004F54E03B8F77E02C8D850154523B742BF2
:100BA00054AC00E00586A802850774F155E0208F5B
:100BB00074F156E01A8F74F155E0148F74F156E019
:100BC0000E8F850EAD068591979617917385CF0F81
:100BD000E00E0DF27F3D9B737E85CF10103D268386
:100BE0006167B4D0433E7690956140566811405796
:100BF0001146713C0A1110950C2E543E092D2D2CD6
:100C00002E42403D78858383E00B8E67852E4266B9
:100C1000B916BA200F909540429715BF099095409C
:100C2000901491157585CF119715012D424090951F
:100C30007191958504A803103D27362837E0D41616
:100C4000B300C0452F2320C201F600444946455158
:100C500019A621AB198EA815F54E414D453F8C8E36
:100C60009A07F74F524445523D3F8B8EA901977327
:100C7000A801FB535445502053495A453D3F8E121D
:100C80004331F458303D3F8E32F459303D3F8E337E
:100C9000AC01E02D800A2322E0958135E06B84369B
:100CA000E06784920683402340222183403440E061
:100CB0007E81254026834040134324E05482BA2B92
:100CC00001F559302E3D3F8E340B242322E0608104
:100CD000353021E0498636302120244025E0448506
:100CE0009206834030218340E034862683404025AD
:100CF000401343244034762625401343402183404B
:100D0000354276E00C82BB3F052340222140B29E53
:100D10000392027192038F980298037F8507202423
:100D2000402006124324407442234022744002AE05
:100D300087082142CC212F3A50CA00F3005643A91C
:100D400004CF6FA815A81BFC4450204350200D2051
:100D50004D2055568EA627D0176FCF7EA62DF16455
:100D6000CF14F27F3D9B737ED0286FCF7DA62FCF0F
:100D700068A62CF10DD01614CF6BA62AD03C6FCFED
:100D80007BA629D0068FCF7CA628CF0FAC04D04EEF
:100D90006FCF7FF2583D9B737EF2593D9B727EF27E
:100DA0005A3D9B717ED0656FCC0FF60043524F5376
:100DB0005383CE023042CE022342CE01947171940D
:100DC0000342742042234121744190712241CE712B
:100DD000A62785CF67A623D04E0FCF6DA624D09E21
:100DE0006FC208F300565361686877139474967461
:100DF0000F7591F496740F7591F496740F7591F4C4
:100E0000757585CF6EA625D07E0FCC05F3005652A2
:100E1000686175A627741342134090F3977290F29D
:100E2000977190F185CF66A626F3444F54D0CE1427
:100E3000C605F400444F54214271224240712342BE
:100E40004085CF6AA62BD0BD0FCF69A62B74F14D7C
:100E5000D0F114C005F30056453175327533757500
:100E600085C002F300562D1C11A62EC601F30056B4
:100E70002B920175920275920323222185C802F4F8
:100E800000565859CE0175CE0275CE03757585C8CA
:100E900002F30055564F90714F917077114ECE70FE
:100EA000754E85CC02F300560DA62BA62AA62BA6BE
:100EB000265D85C402F3005644A628A62B7485CA75
:100EC00001F300562A9470947142C8012F2030C05B
:100ED00001F30054521117A621AB198ECF6AA91B3A
:100EE000FA5A302C59302C5830203F8E13A62477D4
:100EF000F5524F540D3F8EA90567B198A805911082
:100F00007311CE71F7632C622C61203F8EA62B12D9
:100F1000A624CF6F01A81BA815A901FC5E4E205E78
:100F20004F202020204E45578EB117CF7DA622CFCF
:100F300066A801A630D008FFCF67A901A630CF7FF1
:100F4000F2583D9B737EF2593D9B727EF25A3D9B57
:100F5000717EB140C013F3004354AD01B38813A6B2
:100F600025A628AD058503AD05B2B611A62412A6A7
:100F700025A6239010AD015459A62E1130A6259018
:100F8000105A9300A62EA62914A62412A62511A64F
:100F900025A6269400A62A20A62E14E00783AC01DD
:100FA00085021304A625A629C00C2F00000000000E
:100FB0000000000000000000000000000000000031
:100FC0000000000000000000000000000000000021
:100FD0000000000000000000000000000000000011
:100FE0000000000000000000000000000000000001
:100FF0000B00D19E000000CBC30000311604011885
:1010000000000000000000000000000000000000E0
:1010100000000000000000000000000000000022AE
:10102000020000C0001800100010F223E3F3C4CE49
:10103000201214C16F3C5888FFE6EF080000000042
:10104000006804545555554D1CF1EC4CE30DC03D62
:1010500006CC23E2CCD14F333B3713F22B3353541E
:101060000D4FAB28CF1D48E80DCEB33713DBCF1C97
:10107000734C456417FC24E2F05112F1F2F2BA28E5
:101080000479EF2FD173C3C4FD7D138C14D5CA63CB
:1010900000004C444C10D705000013542274334018
:1010A0005513ECC10800C0041122DD0C5430B20706
:1010B000234C101304C12CD07530002333008C3C1A
:1010C000C300CC074CD033303F30E7E1B4003341AC
:1010D000220713141335CDD4650D74EC47C9D01015
:1010E000D0109010D01000003000C0348D0110419D
:1010F00041111462000011620010004444512100AB
:1011000001000001000001001000040010000004B4
:10111000000000000C0000014000104F02003301ED
:10112000114410410440001033000400014000103D
:101130004F00C40031400C4008C001C0CB1033093F
:10114000009300D330B0330D70000CC002C02CCC23
:10115000246000800080910C00022000088064134D
:101160000000800060008000024839054C0330090F
:101170003005300530D9744967746618DA6F050098
:101180000080010044111111511151444404515483
:1011900044441145114500116200004411050054FA
:1011A00055014544455114154011111441101011B9
:1011B00011411111111145140444444404454414CF
:1011C00051115104111151045015110144880100AD
:1011D00014110045444444004055541551454045C0
:1011E0000010454404000050141140141111111155
:1011F0001111111144101111111111114111114549
:10120000541545445551106200505555551441141C
:1012100044050014414405005511005445000015D3
:101220005455555541445515010055055541450046
:10123000405541554145004055554105555551557D
:101240005551555500505555000100555544450020
:101250000055555555550140555555551100555595
:1012600004401501004154550540555555110041A4
:1012700040880140441401005441515044444441C9
:10128000441011010000144444544544144414050E
:1012900010044544404511410010101111155144EE
:1012A00044545555114504540440445050411004D1
:1012B00051545154544545455145101551555554B7
:1012C00044454540415545555515551511545555FD
:1012D00015545504101144455041105555155504E9
:1012E00055114405101454554510550445500445F6
:1012F00050514414411015551555545555455455E4
:10130000555541551145454411155115454555054E
:1013100011620000451401501100501111000050DD
:1013200015400550115441414154555550555510E3
:10133000054055055550550551554155555555557F
:101340005510551545514455555555555421064090
:10135000444400000045101111444144440411412B
:1013600044101111441005511005010014151551B8
:1013700054551515514410110440551115511115AE
:10138000554410005554151111450404014055559C
:10139000151144144100545505404400445154056E
:1013A000005114550014451555004444540044544C
:1013B00000441462004444110100404501501411DE
:1013C0001501004511454400000045444404111135
:1013D000411444411401105144544451444445457E
:1013E00014114551444451105511210000000000D2
:1013F00000000000000000000000000034C003E016
:101400001839F738F77FF3A2007B00BC00CAF3CF8E
:10141000F81FF845F859F866F873F8A0F8BBF8D744
:10142000F90FF924F93BF958F972F981F98CF9A10E
:10143000F9B6F9C8FA5FFC470DDE0E280E3F0EB470
:101440000ECF0F5CF3DFFD39FDA8FDE1FE0AFE3093
:10145000FE53FE61FE6BFE7DFE8FFEA3FEB3FEBF5C
:10146000FECFFF540FB7F3AB0B900C350CA40CC19F
:101470000CE40D21000085160C0F1308793C2C6834
:101480004670F87030C070381CD0F0A04E68A8B01C
:10149000E80E4924B8AE4EEED74E9F30C7704E5C72
:1014A000229CD08628E806706048658C015C621B2F
:1014B000A2A230C770AE738705140E0904793C2CC4
:1014C000A8898C00900F0F0C0913CC37793C92C47B
:1014D000E0793C3BEEA038588C4F0C27693C924C8D
:1014E000E733784C270CB3B846FC064924F81E7E37
:1014F0007E37793C92895270A6A687A647A6B7A6E2
:10150000BF898C5DEE3B0E658C32EE2F58658C21C9
:1015100070658C3A898CC5898C50793C92793C1ADB
:10152000120503151213090F0E898C881E7EF87E92
:1015300023B87E37793C92895244793C3BEEA338FC
:10154000580C270C63AB8C9F884844CC13488843C5
:10155000084404CC13080898F04670B87C588C876F
:1015600088983CA86D8C9F580C1F04138498F04CED
:10157000471348300B0C1F301E06793C65E6534C70
:10158000C36D8C9F580C174B793C92793C1A0E0F07
:1015900020120F0F0D898C884E58793CD36AF3DCEA
:1015A000901E1C793CE5E698E6D63C58BEB31C98E4
:1015B000EA1F3CEB58681598EE1B4C33793C92813E
:1015C0000A5C420A0C23AA62231C29A430C3704E71
:1015D0005CAAF04D9CCC67B8584C474EE8380E0AD0
:1015E000AE28B80A30C370387CAABCF04E705C10CC
:1015F0009050105090105050D058681598EE1B4CD9
:1016000023693CBCC80C17C40E1C1DA4BD8C4D9C8A
:101610000E30C37038BCAA7CF0E0A18888C1B0BD90
:101620001EBA60A67066A638E67066E6F0A3BA60D9
:10163000A67026A638E67026E6F0A3E0DCA0467089
:1016400078E630C0067026CB38EEB33E8F7E5C1253
:10165000DC90905C726B5E725BFC560643A6262B98
:101660004EE0E026E046704EA668793C3BEE43A68D
:101670000670264338EE2BFC5606B3668646707815
:101680003CC6BC68860630C070383C1CCA60164632
:10169000A0A6262746E02B66E6C60A3C0A7CF03662
:1016A0006630C1464670783CA6C6A65ABC1A783C3D
:1016B000066626A666A6793C21A6E066866D8C9F06
:1016C0003E13664670783CC6BC682626C61B46E0BC
:1016D00030C00670383E23A626CB30C01E7EC646DC
:1016E0001F661E46707826467CA63C66683C06A6A9
:1016F0008630BF46BC265E1726463C5ABC1A667921
:101700003C21467078E67C0630C0704EDC9090FC40
:10171000A6B606167CE6F67CF04E68A830C00666D3
:1017200070383E274E7EF04626E0044460793C3B0C
:10173000EEA038588C13488CE30C8B084C3F0448BF
:1017400098F0B833844498F07858FB7858C44C1318
:10175000C88CBF6B0C1F4EE0B858C40C13C80C5794
:101760004670B87C5884983CA84670987C1CEAA0C7
:101770000E6D8CBAB858259E4924B0E888793C2A69
:101780000C27793C954C534924B87C588C1F450252
:10179000C502793C2A793C3BEEA0A6067026433868
:1017A000EE2BFC5606B38630C00670383C56062633
:1017B0000670385CEA273E1366A6066686A65ABC03
:1017C0001A6630C0E6793C2E662643A67026064E81
:1017D000F0C3E04E1C909C101C0AE5A456E6603055
:1017E00005426ABFE01CEDA43C3005426A1F1E1B87
:1017F00059A47CE000000000000000000000000090
:101800004408918C6B30C170385CEA1CBC0A46708D
:10181000793CBA5C6AC44213C81CBD8C4C091FC118
:1018200002793C95F858793CAB6BB058793C9558A7
:10183000793CAB793CA2F0418C78793CA8EE2769E1
:101840003CA10EB05EFE23693CAF1EA0BE1D6160D0
:10185000FE1FEE27693CF3793CA5EE63793C9F1CA3
:1018600002D0761613B6F0793CA86838E8F828B0AC
:10187000A8B80E793CB53A356060793C1D793CF2E8
:10188000EE9B793C6A0E793C1A793CB52626BE253A
:101890006160FE574E5C2226260E793C1A793C99EF
:1018A0000E38AEA0BE1D6160793C1D793C79793C53
:1018B000A2A0256060793C1D793C56D85EFE6B790C
:1018C0003C52A04E3E6EA03D60A5500E60793CFD9E
:1018D000EE9F793C56793CA2A02560A550600E7918
:1018E0003CFDEEFBF8700648693C00793C524E5CCA
:1018F000223AA3793CA5EE37B068693C71793C9FE8
:10190000F627693C6A76F0793CE7793C1DB00E79A0
:101910003CA8A0BE1D6160793C52A04D6060793C3E
:101920001D793CF2793C1D793CEC793C06A0BE1E49
:1019300060793CE3793C81793C990EF8AEA0BE1DFC
:101940006160793C063ECE63793C0EA0BE1E607994
:101950003CDF23793C5A793C87EE67793C5A793CE5
:1019600087EE27F8E82BF84EEED7793CA858793C5B
:101970009558793CAB793CA2F04670B0E8498C2A86
:101980000C27498C95B95AA04E5C66503D6030C812
:1019900070382560A5500E30C770AEE80E384E6026
:1019A000E0B0A84E68793C99E8064870693C00B8F8
:1019B00068380E793C99AEE884B0A8F8280E793CD6
:1019C00099A0BE1D6160793C1D793CA50EB8A0614F
:1019D000604E5C223ABE256160793C060E793CA2DD
:1019E000A01D60A5500E60793CFDEE87793CEC7936
:1019F0003CA2A05CFA37BEB626228B5E37FE373A91
:101A00005BBBFEE762FA1B2213667A00A5500E60EC
:101A1000793C99AEE84EEE27693C2A7870F80E7949
:101A20003C994EEE27B08C53AE0E06664870693C6A
:101A3000000E793CA85EFE23693CAFA0B8AE6160A1
:101A4000096060793C1D793C990EF8A0BE1D61606B
:101A5000793C52A0496060793C1D793CE7793C6A49
:101A60000E793CB5BE1D610E60793C99AE680E7969
:101A70003CD3BE1D6160FE9B793CA55E680E793C3F
:101A8000D31D6060793C1D793CA50E793CB51D6085
:101A900060793C06793C1D793CD386BE2561FE7396
:101AA00060793C52B0A0BE3D61BB793CA50E793C4B
:101AB000D386BE1D61FEBB30C970380EB0BE356125
:101AC000A5500E60793C99AE6888693CB9B026266D
:101AD00026BE77793CB5666666E0A0316060E07945
:101AE0003C5AC3793C56A3793C99F823793C990E2A
:101AF0003833793CA50EB8A0BE1D6160E0793C99F1
:101B0000AE0EE8384EE0793C52A0756060E0793C5A
:101B100056C3793C352B793C52E32E7A0B30C0709A
:101B20003868F828CEBE1EE8B8BA9CEAEAEABAA835
:101B3000AA8A8A8AE330C070EED8B81A9ABABABABA
:101B40001CEAE6A8F8EE38E87828BA463CFED8EE5B
:101B50005CE030C39C4330C41C2330C59C7038EE1D
:101B6000D8B8D4CE14EBFEAED83B793C52A0756009
:101B7000A55060E0AE0E58CE23793C56A049606077
:101B8000E030C070B83CA6BCA830C37038BE5CEA78
:101B9000F0E07038E0793CAB0E30C7BB30D0A330FA
:101BA000C08B30C87330C95B30CA434E707828B8D8
:101BB0006898A85CE04E5C22A0E01C38AAFC0EF8F5
:101BC000FCAAE8AE28E0B0A0FA274626765C5A5E6A
:101BD00050EE4670B87C0E9CA2467C60E6E6A0AE55
:101BE0001C2666E21B4213A6B67FB66F58860646D1
:101BF000B6504626561B26986E466030D070E000E0
:101C00004924F870B80E30D0704EF0F0586D8CAB9F
:101C1000AE5830C07098E8A0BE1D616030D0704EE4
:101C200028E8DA2F58693C3E793C5B30C070F825D3
:101C300060706006481344666630D07038F0EE5825
:101C40004670B028EE7004793C6B30C270658C0829
:101C50006D8CC6AE68F8F0E80666693C506D8CC6BF
:101C600078A01D6068B80EB86160AE0E58CE4960AD
:101C700009604EBE50503D60606D8C1D30D0707854
:101C8000A03D6030C070B82560A830D070F80E302C
:101C9000C07038F01D6060793C55B0FED830DE7001
:101CA00038FED83160606D8C1D30DE7038A6F07E55
:101CB00030C070CE284E900E30D070B8A01D60A8F5
:101CC0000E60693C0A30D0704EE86D8CC6B068304A
:101CD000C070AE6830D0705C4E90A830DE70385E58
:101CE00046F030C0704E28A830D070F80E78A01D95
:101CF000602830C070F80E30D07038AEBE1D61382C
:101D00003D60A550F05C4E22A80EA0B8AEBE1D618D
:101D1000FE2B60693C55B86960AE0E58CE4960E84C
:101D2000B80E1D60B82560F83D60B869604E6690D9
:101D3000503D607030C070F80E60793C62B03D601C
:101D4000700E30C070F81D60F00E60793C62E806DD
:101D50006660693C36B80EA0BE35612830C070B8E8
:101D60000E30D070B86160F030C070780E30D07036
:101D700038616030C07078BE2561B0256060793C04
:101D80005B78256068606D8C5230D070F870B8A0B8
:101D9000696078BE2561B02560606D8C1D30D070A3
:101DA000780EF0A01D60386960606D8C35A03160E0
:101DB00060793C5BF02560606D8C1D30C070787080
:101DC00030D070B8A0FA23DA50260EA8356009602A
:101DD00058606D8C95B0AEA06160B0256068EE462D
:101DE00070B80E78A846703868EE2E7A606D8C0652
:101DF0006D8C52A03160709E30C070CE2830DE7085
:101E000038A606F0B0BE256158380E30C070AEA8B6
:101E100030D07098E8780EB0AEBE1D6128B06888EA
:101E2000084E6830C070B84AFC0E4E1C50A8901C7A
:101E3000029C48021BAE44F08C1F04138430D07007
:101E4000780E4E5C10A035604ED0256068F80E30DC
:101E500007E66030C070B8AE26AE7038A0BE1D6117
:101E6000382560A830C070780EE0DCA01CF2525E0D
:101E70001B669230D070B85EBE1D61FE7384083060
:101E800007E66030C070B80EB09C02EB26AE70AEB4
:101E900038A0BEAE60267038A01D60783D60B8697D
:101EA000604E90BE2561FE1B88083007E66030D08A
:101EB00070F80E30C070B8A626A670AEF0B80E78D6
:101EC000A06160F82560E83007E6C66030C070B8F1
:101ED0000E0C33B0AE9C22A80227693C38B80E4CD9
:101EE0005730D070F826AE70AEF030DE7038A03EBD
:101EF000137E46F060693CE2F858606D8C9530D0F6
:101F00007038586D8CABAEA0BE1D6130D07078704B
:101F1000F858606D8C81980EB0A01D6060793C55BA
:101F200070606D8C521E30C07078A03D60B0FA4376
:101F30005A5E5066D414EB2560A550F05C58606D75
:101F40008CABB0A0A550F060D44B30C07038D888AE
:101F5000D8F0418C786D8C52A049624EA05C6650DE
:101F60003D6230D07038AEA0BE1D636630C10C1724
:101F7000267038FC9CA2023CF0A0B0A550584670D8
:101F800098F068A8E87060E0DDAC0170ED8A5470EC
:101F9000C600F40054564D1110A621AB198EA900AD
:101FA000CF7F773132333435D00BEF0FA815F27F66
:101FB0003D9B737ECF6FA81BA916FF204E2C204996
:101FC0002C2050562C504D542C46F27F568ED01B50
:101FD0006FCF7B111242CF66F14E31AB16A634BFE4
:101FE00036CF7C111243CF67F14932AB16A638BF0A
:101FF00046CF68F2505633AB16A635BF52CF69F3C1
:10200000504D5434AB16A636BF5FCF6AF2465635F4
:10201000AB16A637BF6BCF7EA815F3454E44AB0079
:10202000A800AC00F5424547494EF67F204D4F448D
:10203000457ED07F6FC817F2004E2267B49B111BFC
:10204000124336E02F8864BBA32864B29705F624B8
:102050004552524F528ED0A36F042325402467B5BA
:102060001443B18402E0068A015431850B6526656C
:1020700043318509E0118938E00D8939850CAC00C0
:1020800011AD001042850A2383CE05334026543615
:1020900061E0150B114024422623424067B55243AC
:1020A00026425485CC0FF30050562267B189E05484
:1020B0008727254226B2830125210224424054333A
:1020C00085C204F400504D542267B18BE036872757
:1020D0002542234026B28501232540210267B50011
:1020E00043543485C005F30046562267B18BE01493
:1020F00087244223402743B2860124214223400201
:102100005435850822111B124365214254553776F8
